:020000040800F2
:10000000B0DC0020990300086D520008854D0008FF
:1000100059520008C12F0008855E0008000000004A
:10002000000000000000000000000000CD020008F9
:100030005B3100080000000011030008D5570008DC
:10004000B3030008B3030008B3030008B3030008B8
:10005000B3030008B303000879310008B3030008B4
:10006000B3030008B3030008B3030008B303000898
:10007000E9300008F5300008013100080D310008B2
:100080001931000825310008B3030008B303000844
:10009000B3030008B3030008B3030008B303000868
:1000A000B3030008B3030008B3030008B303000858
:1000B000B3030008B303000849580008B30300085D
:1000C000B3030008B3030008B30300083D5600085B
:1000D000B3030008AD5C0008D55C0008195D00089A
:1000E000B3030008B3030008B3030008B303000818
:1000F000B3030008B3030008B3030008B303000808
:10010000B3030008B3030008B3030008B3030008F7
:10011000B3030008B3030008B3030008B3030008E7
:10012000B3030008B3030008B3030008B3030008D7
:1001300000F002F800F0BAF80AA090E8000C82443F
:100140008344AAF10107DA4501D100F0AFF8AFF21C
:10015000090EBAE80F0013F0010F18BFFB1A43F0A5
:1001600001031847C8750100E87501000A444FF003
:10017000000C10F8013B13F0070408BF10F8014B06
:100180001D1108BF10F8015B641E05D010F8016B4B
:10019000641E01F8016BF9D113F0080F1EBF10F8AF
:1001A000014BAD1C0C1B09D16D1E58BF01F801CBD2
:1001B000FAD505E014F8016B01F8016B6D1EF9D555
:1001C0009142D6D37047000000230024002500266A
:1001D000103A28BF78C1FBD8520728BF30C148BFAA
:1001E0000B6070476E2900F0E685702900F03582BB
:1001F000662916F06D86652916F06A86672916F05D
:100200006786612916F0668603681B0A28BF41F0DD
:100210008001692900F0A681642900F0A381752975
:1002200000F0A0816F2900F0E686782900F00182B5
:10023000E92900F08186E42900F07E86F52900F0A6
:100240007B86EF2900F0E386F82900F0008203683E
:10025000DB0928BF41F08001632900F0F085732994
:1002600000F0F585E32901F08D83F32901F09283F5
:10027000002070471FB59DE8030002F0DDF800F094
:10028000CEFB00F025FD04000020002116F0F4FD57
:10029000401C60600020002116F004FEE06001F0C8
:1002A0003BFD1FBD10B501F0A0FD10BD01F0F0FD3C
:1002B0001146FFF7DFFF0AF003FE02F091F803B4E6
:1002C000FFF7F0FF03BC05F09FFE0000224B19680A
:1002D0000868B0E8F00F80F30988BFF36F8F4FF024
:1002E000000080F311884EF00D0E704700000000F2
:1002F00006480068006880F3088862B661B6BFF3FC
:100300004F8FBFF36F8F00DF00BF00BF08ED00E02D
:10031000EFF30980BFF36F8F0F4B1A6820E9F00FDE
:10032000106008B54FF0500080F31188BFF34F8F75
:10033000BFF36F8F15F0F8F94FF0000080F31188CC
:10034000BDE8084019680868B0E8F00F80F3098834
:10035000BFF36F8F704700BF78000020EFF3058078
:10036000704700000B49D1F800C04A685CF8043BB4
:100370001068184442F8040B8C4528BFA1F1DC0C2E
:100380008A4228BFA1F1DC02C1F800C04A6020F017
:10039000004070474CCF002009488047094800477B
:1003A000FEE7FEE7FEE7FEE7FEE7FEE7FEE7FEE725
:1003B000FEE7FEE704480549054A064B7047000082
:1003C0004758000831010008B0D00020B0DC002000
:1003D000B0D40020B0D400207047000010B500F069
:1003E00077FC001D10BD00BF916A0100B2F120032F
:1003F0000AD5C2F1200320FA02F001FA03F321FA30
:1004000002F140EA0300704721FA03F04FF00001C7
:10041000704700007CB51D4616460C00009001D0C8
:100420002044401E074B7B442A46694601903046D3
:1004300000F0DBFC05461CB10020694600F0E8FC3A
:1004400028467CBDF10900000FB4044910B503AA89
:10045000029800F001FD10BC5DF814FBA8CF00204D
:100460000FB41CB5084B06AA7B446946009005985A
:1004700000F0BBFC04460020694600F0C9FC2046A1
:100480001CBC5DF814FB0000A50900000FB47CB58E
:100490000C0009AA009001D02044401E084B7B4468
:1004A00069460190089800F0A0FC05461CB10020A8
:1004B000694600F0ADFC28467CBC5DF814FB0000EA
:1004C0007909000070B5044685690068C10601D548
:1004D000302600E02026C00707D070BDD4E90121F6
:1004E00030469047206A401C20626D1EF6D570BDD4
:1004F00070B5044685690078C00707D170BDD4E99E
:10050000012120209047206A401C20626D1EF6D5F4
:1005100070BD70B50C460546012A05D028788006C6
:1005200000D5EA69002302E0012305E05B1C934249
:1005300002D2E05C0028F9D1A869E618C01AA861C7
:10054000286A184428622846FFF7BCFF04E0D5E972
:10055000012114F8010B9047B442F8D32846FFF765
:10056000C7FF70BD2DE9F0410646002410687529CB
:10057000314616A510D000F0B3FB002802DA404245
:1005800013A507E031688A0701D512A502E04907E3
:1005900004D511A5012401E000F0ABFB00210A22E3
:1005A00006F1240709E0B0FBF2FCB0FBF2F302FB1A
:1005B0001C00303078541846491C0028F3D12346DB
:1005C0002A463046BDE8F04100F09CBB0000000028
:1005D0002D0000002B00000020000000F0B40D46AC
:1005E0000188090502D5214C7C4402E01F4C7C4463
:1005F0000E34002100F1240608E002F00F07120972
:10060000E75D42EA03721B097754491C52EA03076B
:10061000F3D102780023120704D5702D06D009B15A
:10062000022311342246F0BC00F06CBB01231034CD
:10063000F8E770B504460D462146106800F059FBF6
:10064000024629462046BDE870400023C6E7D21D79
:1006500022F00703D3E90023C0E70368126843F0E0
:10066000200303600823C3610023B7E7E46A0100A5
:100670002DE9F05F894604464FF0000ADFF874B1B7
:10068000FB44C0F820A02046E1688847002874D0C9
:10069000252806D0D4E901219047206A401C206219
:1006A000F1E700265F462046E16888472028054696
:1006B00007DB312D05D2781910F8200C08B106435C
:1006C000F1E7B00701D526F00406C4F81CA0002706
:1006D000C4F818A02A2D09D0284605F08CFC38B3A0
:1006E00004EB8708303DC8F8185019E059F8041B8E
:1006F000204604EB87029161E1688847012F054697
:1007000018D1E069002820DA26F020061DE0D8F88C
:10071000180000EB800005EB40003038C8F81800E6
:100720002046E1688847054605F065FC0028EED1C3
:10073000012F0AD02E2D08D12046E16888477F1C62
:100740000546022F46F02006C4DBA069002803DA24
:10075000404246F00106A061F00701D026F01006E5
:100760006C2D0BD0682D09D04C2D39D06A2D35D089
:10077000742D35D07A2D33D016E038E0E1682F465D
:1007800020468847B842054609D16C2F26D04FF441
:100790008060E168064320468847054604E06C2FE8
:1007A0001AD04FF4807006430DB3A5F1410019280B
:1007B00002D8203546F400664A462946204626607F
:1007C0004E46FFF70FFD80B101280BD0F61D26F035
:1007D000070000F1080956E74020E4E78020D8E749
:1007E0000020D6E706F104094DE7284652E7206AC3
:1007F000BDE8F09F746A01000FB400B58DB010A978
:10080000099000910B904FF0FF300A9000200C905F
:10081000064878440690064878446A4607900F993F
:1008200009A800F013FC0DB05DF814FB5708000098
:100830006F0800002DE9FF5F1D464FF0FF3B91461A
:100840004FF000085F46D5E90146A96901987F1C71
:100850008847296A824688470028F6D1BAF1FF3FC7
:100860000CD0002E24F4C06419DD600614D5BAF152
:100870002B0F09D0BAF12D0F0ED103E0584604B06A
:10088000BDE8F09F44F48064A96901987F1C884703
:10089000761E8246002E02DDBAF1300F03D0B9F188
:1008A000000F26D032E0A969761E01987F1C44F41F
:1008B00000748847002E824605DDBAF1780F06D015
:1008C000BAF1580F03D0B9F1000F10D01EE0B9F102
:1008D000000F02D0B9F1100F18D1A969761E019846
:1008E0007F1C24F4007488478246102002E0082010
:1008F00000E00A20814609E0A96908FB0908761E84
:1009000001987F1C44F4007488478246002E05DD60
:100910004946504600F086FB0028EDDAE969019867
:100920008847A00502D46FF00100A8E7E00725D1B1
:10093000600613D5600502D5C8F1000000E040460E
:1009400029680A1D2A600968220501D5087015E08A
:10095000220701D5088011E008600FE02868011D1A
:1009600029600068210502D580F8008006E0210793
:1009700002D5A0F8008001E0C0F8008038467EE78C
:100980002DE9F05F93460F4680460446002600F0AE
:10099000A3F9D0F80090824614F8015B2DB1FFF75F
:1009A0001DFD0068405DC007F6D12B2D02D02D2D16
:1009B0001AD0641E0021CAF800105A463946204653
:1009C00000F074FB014627B13868A04201D1C7F896
:1009D0000080DAF80000022809D0CAF800907005FB
:1009E00005D54842BDE8F09F46F48066E2E7084638
:1009F000F8E700000B4910B5A1F17C020A4CC2E9EE
:100A00003712372106E000EB104342F82130074B44
:100A100000FB03400B1EA1F10101F4DC10BD01201D
:100A2000E8E70000ECCE0020E119D666CD0D01000C
:100A300040EA010310B59B070FD1042A0DD310C85B
:100A400008C9121F9C42F8D020BA19BA884201D9AD
:100A5000012010BD4FF0FF3010BD1AB1D30703D0F5
:100A6000521C07E0002010BD10F8013B11F8014BAB
:100A70001B1B07D110F8013B11F8014B1B1B01D1C7
:100A8000921EF1D1184610BD10B5431C02E010F8BB
:100A9000011B71B18107FAD14FF0013202C88C1AE3
:100AA0008C4314EAC211F9D0C01A0A0603D0C01E42
:100AB00010BDC01A10BD0A0401D0801E10BD09026D
:100AC000FCD0401E10BD032A40F2308010F0030C11
:100AD00000F0158011F8013BBCF1020F624498BF91
:100AE00011F801CB00F8013B38BF11F8013BA2F12E
:100AF000040298BF00F801CB38BF00F8013B11F0A9
:100B0000030300F02283083AC0F0088051F8043B48
:100B1000083A51F804CBA0E80810F5E7121D5CBFB5
:100B200051F8043B40F8043BAFF30080D20724BFE8
:100B300011F8013B11F801CB48BF11F8012B24BF7C
:100B400000F8013B00F801CB48BF00F8012B7047CB
:100B500002F0FF0343EA032242EA024200F002B835
:100B60004FF000020429C0F0128010F0030C00F0D6
:100B70001B80CCF1040CBCF1020F18BF00F8012B54
:100B8000A8BF20F8022BA1EB0C0100F00DB85FEA22
:100B9000C17C24BF00F8012B00F8012B48BF00F8EE
:100BA000012B70474FF0000200B51346944696465D
:100BB000203922BFA0E80C50A0E80C50B1F1200170
:100BC000BFF4F7AF090728BFA0E80C5048BF0CC01E
:100BD0005DF804EB890028BF40F8042B08BF70477C
:100BE00048BF20F8022B11F0804F18BF00F8012BEE
:100BF000704710B5044610F0030F08BF11F0030F43
:100C000040F015804FF0013E121FC0F20E8051F8E7
:100C1000043BA3EB0E0C2CEA030C1CEACE1C08BF11
:100C200040F8043BF0D0A1F1040102F10402521E8D
:100C300008DB11F8013B002B00F8013BF7D111460E
:100C4000FFF78EFF204610BD4FF0013C50F8042BFB
:100C500051F8043B9A4221D1A2EB0C03934313EACF
:100C6000CC1317D150F8042B51F8043B9A4215D1FC
:100C7000A2EB0C03934313EACC130BD150F8042BD3
:100C800051F8043B9A4209D1A2EB0C03934313EAB7
:100C9000CC13DBD04FF00000704700BFD01A01BA70
:100CA000B1FA81F101F0180122FA01F0CB40C1F153
:100CB0002001DBB2C0B2C01A2CFA01F3D11A914361
:100CC00011EAC311E6D1704770477047704770470B
:100CD0000048704770D000200048704750D0002076
:100CE00009684A0501D540B27047C905FCD500B274
:100CF000704709684A0501D5C0B27047C905FCD5DF
:100D000080B270472DE9F0470D4699469246044659
:100D100000F124080168880604D5E06921F010017B
:100D2000216000E00120A84201DD471B00E0002710
:100D3000A1697A1902EB0900081AA0612078C0069F
:100D400002D42046FFF7BEFB002608E0D4E90121CB
:100D50001AF806009047206A401C761C20624E4517
:100D6000F4DB2078C0060AD52046FFF7ABFB06E08F
:100D7000D4E9012130209047206A401C2062381EAF
:100D8000A7F10107F4DC07E0D4E9012118F8050018
:100D90009047206A401C2062281EA5F10105F3DC63
:100DA0002046FFF7A5FB2078000602D50220BDE80B
:100DB000F0870120FBE711680268006A530501D53E
:100DC00008700AE0D30501D5088006E0130603D5B4
:100DD000C217C1E9000200E008600120704700006E
:100DE00001694A1C02610878704700B58FB0CDE9EF
:100DF00001310021059105497944CDE903101146DF
:100E00006846FFF735FC0FB000BD0000E5FFFFFFAF
:100E10000A6802F8010B0A607047D1E900239A4280
:100E200002D2531C0B601070704710B5436913B1A8
:100E3000AFF3008001E0FFF76CFB012010BD1278DA
:100E400000F124010A7000224A700122EDE71168C6
:100E50004FF0FF32E9E70000074B70B50D467B44C9
:100E6000FFF7C3FF0446284600F052FF10B14FF0D1
:100E7000FF3070BD204670BD538300002DE9FF5F39
:100E800015468A460446DFF8AC80F8440027D8E9C6
:100E900000103E46CDE9001010E03AF816106A4600
:100EA00002A800F0D5FF411C07D02178890603D5A0
:100EB000E269391891420DD80744761C20788006E3
:100EC00002D5E069B84205DDAE42E6DB3AF816002D
:100ED0000028E2D1A069C01BA0612046FFF7F2FA0A
:100EE000D8E90010CDE90010002017E03AF81810FA
:100EF0006A4602A800F0ACFFB0F1FF3F81460BD07C
:100F000000250DF1080B05E0D4E901211BF80500CF
:100F100090476D1C4D45F7D308F10100B042804663
:100F2000E4DB206A384420622046FFF7E1FABDE89E
:100F3000FF9F00007E6201002DE9F0418046D21D36
:100F400022F007020025D2E90002F52915A614D0E7
:100F5000011E72F1000106DA0023D0EB030063EBFF
:100F6000020211A608E0D8F800108B0701D50FA6E1
:100F700002E0490701D50EA601251146002408F11B
:100F8000240704E000F018F930323A55641C50EAA6
:100F90000102F7D12B46324621464046BDE8F041DA
:100FA000FFF7B0BE000000002D0000002B00000085
:100FB0002000000030B4002100F1240408E002F019
:100FC0000705D208303542EA4372DB086554491CF4
:100FD00052EA0305F3D10468002310A2250707D5C0
:100FE000A40600D421B1C46901230DA2641EC4610A
:100FF00030BCFFF787BE10B5044621461068FFF7E6
:1010000078FE02462046BDE810400023D2E7D21DFC
:1010100022F00701D1E90023CCE700000000000026
:10102000300000003A2800D2303820F02002412A57
:1010300001D3A2F13700884201D34FF0FF3070474F
:10104000026811441378016018467047D160054961
:1010500079445161044979441162002111611146BA
:1010600000F09CBCEDFFFFFFE9010000426842B1C7
:10107000016811F8013B23B1521EC0E90012184665
:1010800070470121C160881E704742685AB1C36829
:10109000016843B983688B4205D0491E521CC0E9E0
:1010A0000012002070474FF0FF3070472DE9F05FCD
:1010B000824615468B4600270AF10104B94600789E
:1010C000302801D09DB113E014F8010B01277828D6
:1010D00003D0582801D045B10AE00DB1102D07D139
:1010E000002714F8010B102502E0082500E00A256E
:1010F0000026B0460EE005FB080005FB06F10127BF
:101100001FFA80F801EB1046B6F5803F00D3B946D0
:1011100014F8010B2946FFF785FF0028EBDABBF135
:10112000000F05D00FB1641E00E05446CBF800401C
:10113000B9F1000F06D0FFF7CFFD02210160C81EF4
:10114000BDE8F09F48EA0640FAE710B5203AC0F043
:101150000B80B1E81850203AA0E81850B1E81850B8
:10116000A0E81850BFF4F5AF5FEA027C24BFB1E8F5
:101170001850A0E8185044BF18C918C0BDE8104066
:101180005FEA827C24BF51F8043B40F8043B08BF6F
:101190007047D20728BF31F8023B48BF11F8012B36
:1011A00028BF20F8023B48BF00F8012B7047000021
:1011B0000048704750D0002030B5B0F10A024FEA25
:1011C000900E71F100034EEA817EB0EB0E0061EBF0
:1011D00091014FEA101E4EEA017E10EB0E0041EB2A
:1011E00011114FEA102E4EEA016E10EB0E0041EB8A
:1011F00011214FEA104E4EEA014E10EB0E0041EB6A
:101200001141401841F100014FEAD00040EA41701D
:101210004FEAD10110EB80054FEA810444EA907453
:1012200044EB01046D1944EB0404521BA3414FF03D
:10123000000348BF0A3200D530BD401C41F1000117
:1012400030BD10B50446FFF7C9F80068005D00F036
:10125000010010BD70472DE9FF4F0C461E464FF0B0
:10126000FF378BB0D2E90001DDF860800A908A4632
:10127000C1F30A5505B93D46002108464FF000006C
:10128000BAF1000F00F4400005DA00EB80004FF4E3
:10129000400101EA50004FEA9059B9F1010F00DD19
:1012A000B9460A9850EA4A000ED044F61050A5F20A
:1012B000FF3545432F14B8F1000F1ED07542291E8B
:1012C0001EDDC9F100021CE0B8F1010F4FF0000073
:1012D00001D0302103E0F24305E02154401CB0422C
:1012E000FBDB30460022002121540B99C1F8088015
:1012F000C1E900200FB0BDE8F08FBD1B6D1CDEE71B
:101300004A4600DA694206A800F04EFE06AB93E8B2
:10131000070003AB83E8070050460A9901F088FAFA
:101320008DE80700A0F500501F3800900398002DAD
:101330000ADD42F21F014A460844002303A9039034
:10134000684601F0F1FC09E0A0F500504A461F385C
:10135000002303A90390684601F0FBFC8DE8070019
:101360000004000C03D04FF0FF30410800E01046AD
:10137000B8F1000F03D00022009215461EE0751E42
:1013800005D4FFF719FF303262556D1EF9D5B3460B
:101390000122084302D000227F1C04E0207830287C
:1013A00001D100227F1E002A099784D01DE0112D53
:1013B00007DAFFF701FF303262556D1C50EA010277
:1013C000F5D1084302D00098C8B10EE00021681E94
:1013D00005E0235C625C63542254401E491C814238
:1013E000F7DBAB46A81B401E0990002004F80B0059
:1013F0000B98099AC0F80880C0E9002B7AE71126FB
:101400004FF0000857E72DE9F04F88460446D21DFB
:1014100022F0070191B0D1E90001CDE90A0104F001
:10142000C6FD02460B98C00F01D02D2007E02068B2
:10143000810701D52B2002E0202101EAC000032A08
:10144000099001D0072A05DB03464146204600F0FB
:101450006BFD0BE12078800601D5E06900E00620F5
:10146000B8F1650F814606D0B8F1660F18D0B8F113
:10147000670F70D131E00020B9F1110F009001DB4E
:10148000112301E009F101030AAA01A90CA8FFF741
:10149000E2FEDDE90C70002609F10105834647E014
:1014A00001204B4600904FF000470AAA01A90CA862
:1014B000FFF7D1FEDDE90DB00C995D46002610B9AD
:1014C00009F101000D18B9EB050003D4C0F1FF3696
:1014D00009F10105A5EB09002BE0B9F1010F01DAD3
:1014E0004FF001090020B9F1110F0090484601DDCD
:1014F000112300E003460AAA01A90CA8FFF7ABFEDE
:10150000DDE90C704D4600268346207800070AD49A
:10151000AB4500DA5D4601A8012D04DD411911F843
:10152000011C302907D04F4502DA17F1040F04DA05
:10153000012082460FE06D1EEEE7002F02DCED1B5E
:101540003E4403E0781CA84200DD7D1CB81B00F17E
:10155000010A4FF000472078000703D4AA4501DBB9
:101560004FF0FF3A0021B7F1004F0DF143088DF81D
:10157000431024D002202B23002F01DA7F422D2399
:101580000A21021EA0F1010000DC5FB197FBF1FC13
:1015900097FBF1F201FB1C7C17460CF1300C08F8AC
:1015A00001CDEEE7A8F1010003702188090501D5FE
:1015B000452100E06521A0F1010800F8011C09980F
:1015C0000FA9A1EB0807FF1D00B10120411901EB94
:1015D000EA70A1693844081A401EA0612078C0064C
:1015E00002D42046FEF76EFF099828B1D4E9012104
:1015F0009047206A401C20622078C00622D52046F1
:10160000FEF760FF1EE0002E04DBB34502DD01A8FB
:10161000805D00E03020D4E901219047206A401C21
:101620002062761CAAF101005FEA000A0AD1FFF7E6
:101630004FFBC0680168405CD4E901219047206AF3
:10164000401C2062281EA5F10105DCDC07E0D4E97E
:10165000012118F8010B9047206A401C2062381EB7
:10166000A7F10107F3DC2046FEF742FF032011B08B
:1016700041E600002DE9F04F04460D46D21D22F050
:10168000070089B0D0E900974846394604F08FFC3E
:101690000246F80F01D02D2307E02068810701D50D
:1016A0002B2302E0202101EAC0038DF820300BB18A
:1016B000012000E00020032A824601D0072A04DB33
:1016C0002946204600F030FC3FE12078800601D416
:1016D0000D2500E0E569C7F30A560D2D49DA002112
:1016E0004FEA175B08464FF00000002F00F440005F
:1016F00007DA00EB80004FF4400100EBD07001EA04
:1017000060008115012901DD4FF0FF3100224FEA11
:10171000850CBCF1180F06D31346ACF118004FF03E
:101720008052C24003E04FF4801323FA0CF30CF113
:101730000C0CBCF1200F04D3ACF1200C09FA0CF016
:1017400001E007FA0CF000294FF0004801DD18B95C
:101750000FE00ED140450CD319EB02095F4121B9CE
:10176000404502D19F4329EA0209BBEB175F00D035
:10177000761C2088000502D57B48784402E07A4830
:101780007844193808AA302302F80A30037C0AF199
:101790000101002E0AF1020A53546A4602DC4FF09E
:1017A000300101E04FF031014FF001088DF80010D9
:1017B00002D0A6F2FF3603E059EA470100D06B4E93
:1017C000002D02DC2178090704D54FF002082E21F4
:1017D0008DF80110C44600210BE0C7F303433F011D
:1017E000C35C491C6D1E02F80830052908F1010888
:1017F00001DA002DF1DC00210CE000EB1973491C2B
:101800001B786D1E082902F808304FEA091908F103
:10181000010801DA002DF0DC21688B0602D516E004
:10182000A8F10108E04505DD02EB080313F8013CCF
:10183000302BF5D0B8F1000F09DD02EB080313F8E7
:10184000013C2E2B03D1090701D4A8F10108002D7A
:1018500005DD3E2102F808106D1E08F10108407CEC
:10186000002E02F8080008F1010804DA2D20764263
:1018700002F8080002E02B2002F808000A214FF4C9
:101880007A70864208F101080BDB96FBF0F33033E7
:1018900002F8083096FBF0F308F1010800FB13662C
:1018A00001E0642E0CDB642096FBF0F3303302F889
:1018B000083096FBF0F308F1010800FB136601E025
:1018C0000A2E06DB96FBF1F0303002F8080008F132
:1018D000010896FBF1F001FB1060303002F80800BF
:1018E000A16908F1010808EB050202EB0A00081AD9
:1018F000A0612078C00602D42046FEF7E3FD216AED
:1019000008AE01EB0A00206204E0D4E9012116F8D8
:10191000010B9047BAF1010AF7D22078C00602D530
:101920002046FEF7CFFD6E4609E016F8010B3E2873
:101930000FD0D4E901219047206A401C2062B8F101
:101940000108F2D22046FEF7D3FD09B00320BDE81E
:10195000F08F206A2844206203E0D4E9012130207E
:1019600090476D1EEBD3F8E7A959010002FCFFFF79
:1019700010B5436913B1AFF3008001E0FFF77EFAC1
:10198000012010BD128800F1240182840022C2844B
:101990000122EDE711684FF0FF32E9E72DE9F34F3F
:1019A0004FF0000A0C4656468DB001200C9001F114
:1019B0000C000B9062690B9801219047051E2DD0F9
:1019C000252D2CD0216A8847C0B162690B9801216E
:1019D0009047216A88470028F7D16269411E0B9819
:1019E000904700E0761CA1690D988847216A8847D6
:1019F0000028F7D1E1690D988847DBE7A1690D98C8
:101A00008847A842074601D1761CD3E7E1690D98C3
:101A100088477F1C02D1BAF1000F6FD06CE1626978
:101A20000B9800273D46394690472A2804D1626921
:101A30000B98012190470125DFF8D08262690B984D
:101A400001219047A0F130010A290AD24745E5DC7F
:101A500007EB870100EB4107303FDFD445F010056D
:101A6000ECE7E90601D46FF000476C280AD04C2857
:101A700014D0682815D06A280DD074281CD07A2874
:101A80001AD01DE062690B98012190476C2802D0A2
:101A900045F0040514E045F002050DE045F0200591
:101AA0000AE062690B9801219047682802D045F04E
:101AB000080505E045F4006562690B98012190472F
:101AC000C4E9015765283DD019DC58287AD00CDCD0
:101AD000452837D004DC252826D041289ED131E086
:101AE00046282FD0472899D12CE05B2877D0612851
:101AF00028D063287CD0642823D15AE0F7E06F28EF
:101B000048D008DC66281DD067281BD0692821D062
:101B10006E2816D127E0702845D0732868D0752824
:101B200047D078280DD14DE0A1690D988847252828
:101B300005463FF469AFE1690D9888476D1C3FF495
:101B40006AAFD9E00D9923466A466FF00100AFF302
:101B50000080C6E045F0400023464FF00002606080
:101B6000A80736D43EE0E8077FF447AF2068011DA0
:101B700021600068290501D506701BE7290701D5FA
:101B8000068017E7A90703D5F117C0E9006111E73F
:101B900006600FE745F0400023464FF00802606002
:101BA000A80716D41EE040F60E0125EA0100606089
:101BB00016E045F0400023464FF00A026060A80797
:101BC00007D40FE045F040006060A80708D5234621
:101BD00010220D996FF00100AFF3008081E007E063
:101BE000102223460D996FF00100FEF723FE78E0E6
:101BF0004FF0000963284F46C8464B46CB4602D0FB
:101C00005B2807D039E02079C00601D40120A0600C
:101C1000012732E06269D4F80CB00B98012190479B
:101C20005E2807D14FF0010949466269D4F80CB02B
:101C30000B989047216939B900210A4603AB43F854
:101C40002120491C0829FADBD8B3216949B308F1DE
:101C5000010862690B98012190475D28F4D1B9F120
:101C6000000F09D0002003A951F82020D24341F8E9
:101C70002020401C0828F7DB03AB206900282079CE
:101C80004FEA40701ED05B462246CDF80080CDE979
:101C900001970D9900286FF0010020DAAFF3008062
:101CA0001FE0C11703AA00EBD1614B1121F01F0106
:101CB00002EB8302411A136801208840034313603A
:101CC000C7E719E00D99224600286FF00100009740
:101CD00002DAAFF3008004E0AFF3008001E0AFF37D
:101CE000008000280ADA401C06D10C9820B14FF081
:101CF000FF300FB0BDE8F08F5046FAE7E90701D199
:101D00000AF1010A064400200C9053E6CCCCCC0C1E
:101D1000007B00F08000704710B542485421FEF768
:101D200041FF41485421FEF73DFF40485421FEF752
:101D300039FF3F493B483C4A3F4B08603D490A60F8
:101D40003A491960531C0365481C10650120086559
:101D50003B48344A39A1784400F0A6FA20B9384803
:101D600078440A3800F045FB37482F4A35A17844BB
:101D700000F09AFA20B9344878440A3800F039FB68
:101D800032482A4A2FA1784400F08EFA20B92F4811
:101D900078440A3800F02DFB40232248DC00002163
:101DA000224600F05EFA20B125487844543800F00D
:101DB00020FB1D4822464023002100F052FA20B1AA
:101DC00021487844543800F014FB18482246102368
:101DD000002100F046FA002806D01C487844BDE8EF
:101DE0001040563800F005BB10BD104870B5006DAE
:101DF00020F001040B4800F0CDFA0B4800F0CAFABD
:101E00000A4800F0C7FA09E0206D20F001052046DD
:101E100000F0C0FA204600F060F82C46002CF3D108
:101E200070BD000054CF0020A8CF0020FCCF0020C0
:101E3000C4010020C8010020CC0100207200000075
:101E40007E510100770000006A51010056510100E7
:101E500070B516460C460546FEF7C0FA036893F8BF
:101E60000101012806D0FF2C0FD8185D68B10120B0
:101E70002C7070BDD3F807013246214603F20713D8
:101E800003442846BDE8704018474FF0FF3070BD4E
:101E90007546FFF78DF9AE4605006946534620F0BA
:101EA0000700854618B020B5FEF784FABDE820404B
:101EB0004FF000064FF000074FF000084FF0000B06
:101EC00021F00701AC46ACE8C009ACE8C009ACE8B9
:101ED000C009ACE8C0098D46704770B50446051FBF
:101EE00000F08EFA0068002C14BF446870BD002C0E
:101EF00018BFAC423CBF20466468F8D301680A189A
:101F0000AA4218BF456003D12A6805461144016002
:101F100028684119A1421CBF6C6070BD616869608E
:101F200021680844286070BD2DE9F0411F46044631
:101F300003260168072A01F4006004DB08B116A536
:101F400005E016A503E008B115A500E015A521F0F0
:101F500010002060A069C01EA0610FB1401EA061EA
:101F60002046FEF7AFFA4FB1D4E901213846904739
:101F7000206A401C2062C01C206206E0206AFAE74A
:101F8000D4E9012115F8010B9047761EF8D22046BE
:101F9000FEF7AEFABDE8F0814E414E006E616E0074
:101FA000494E4600696E66002DE9F04781461646A7
:101FB0008AB0354878440DC88DE80D003248784421
:101FC000801C03AC0DC884E80D0041F69B3008442A
:101FD000372190FBF1F290FBF1F5A5F1800501FBB3
:101FE00012041B3C02D56442012000E00020DFF80F
:101FF00098A080460027FA44AAF1BE0A0EE0E00746
:102000000AD03246684607EB470101230AEB8101FB
:1020100000F09FFE8DE8070064107F1C002CEED1BD
:10202000194F7F44AE3F19E0E80715D007EB0410C5
:102030000DF1180A90E80E008AE80E00C068F04220
:1020400001D1981908903246012306A903A800F08F
:1020500080FE03AB83E807006D10641C002DE3D104
:102060004FF0010332466946B8F1000F03A802D0D1
:1020700000F05AFE01E000F06CFEC9E90001C9F869
:1020800008200AB0BDE8F087005201002DE9F047B2
:1020900005460C46C86820F4201040F48000C86053
:1020A000800602D5084600F0F8FAE06841F28201A5
:1020B0004FF0FF390140022903D0204600F096FA84
:1020C000B5E000F42041B1F5004F0FD1C00306D5B3
:1020D0006168E06A884200D80846606006E02069CE
:1020E000E0626060606903F090FFA061A068002278
:1020F000EEB200280DDAE1688B050AD4C043A06077
:1021000041F490302260E0606068411C61600670BC
:10211000A5E0E0689046226040F40050E06020694D
:1021200068BB606903F073FF012704F12405A0B1C7
:10213000A08910F4407F08D0E06900F0ACF920617C
:1021400018B1E06840F4006016E0E7612561E068DE
:1021500020F4407040F480600EE0E06900F09BF9EC
:1021600000282061F1D0E06840F4006010F4407F66
:10217000E06002D140F48070E06020696060E06857
:1021800025696FF0010AC1051FD56168E06A8842C0
:1021900000D80846411B04D02246284600F030FAF9
:1021A000F0BBE068010203D5E562C4E9015854E0E0
:1021B000691CE1626160E16940F48030491EC4E954
:1021C000021030462E70BDE8F087010202D500F4FF
:1021D00080320AE06068411C61600670E0680A2E87
:1021E00040F48030E06006D00022E16A60688142FD
:1021F00003D90B4602E00122F7E70346A7895B1BE0
:102200007F0503D4E7699F4200DDE2B1814200D837
:102210000146E5620F1AC4E90158002B09DD00E010
:1022200005E022461946284600F0EAF908B148467A
:10223000C9E747B1A069E5626560C01BA061E068BD
:1022400040F01000E060E068000208D56168A06915
:10225000E562491B08446560A0615046B3E730461B
:10226000B1E770B5C468A50713D0650211D4B2F503
:10227000807F09D0B2F5007F06D0B2F5806F08D11B
:10228000012300F1240106E05D1E6FF07F46B54298
:1022900001D3012070BD0161C361416024F470610C
:1022A0001143C160002070BD2DE9F0410C46074686
:1022B0001646104600F06EF82078611C61280AD09E
:1022C000722802D077283CD102E00125002405E0E5
:1022D0000225042402E0082448F2020511F8010B4B
:1022E0002B2806D0622809D011F8010C74280AD0D6
:1022F0000BE045F0030544F00204EFE745F0040568
:1023000044F00104EAE744F010043846214603F0A3
:102310008FFE411C15D00021316171604FF40071B6
:10232000F560F1617061200704D53046022200217A
:1023300000F0E0F8306D40F0010030653046BDE857
:10234000F0810020FBE72DE9F0410D460646104CD8
:10235000206DC10704D0410804D020F00104F7E744
:1023600022460EE0542000F096F807000ED0206DB3
:1023700047F001010843542120653846FEF712FC5E
:102380003A4629463046BDE8F0418DE70020D6E7C1
:1023900054CF00202DE9F04704464FF000094FF0DC
:1023A000FF37C568D4E90486A80707D0204600F0A7
:1023B00051F9304603F026FE002802DA3846BDE81F
:1023C000F087280502D54046FFF787FD4C212046BF
:1023D000FEF7E8FB206D20F0010020654846EEE79F
:1023E00010B50446AFF300802046BDE81040FDF76D
:1023F00066BF10B500F078F9BDE8104000F06EB986
:102400000048704758D000207047704770477047A9
:1024100038B504460A4600206946AFF3008000281C
:1024200008BF38BD02460099204600F085F901201A
:1024300038BD012000F072B9F8B5AFF30080054651
:1024400000200C46102000BF0646A819A0420DD956
:10245000324669460020AFF30080070008BF00F055
:102460005DF90098A04218BF0546C419FFF7C8FFE0
:1024700005600746F01D20F007004619284600F0C9
:1024800054F9B44208BFF8BDA21B31463868BDE814
:10249000F84000F051B970B50646FFF7B1FF056886
:1024A00006F10B0020F00704B4429CBF002070BD71
:1024B0002B466A68BAB11068A04210D304F1080133
:1024C00088423CBF5068586007D35168101941607A
:1024D0001168091B016058601460101D70BD13461F
:1024E0005268002AE7D121462846FFF791FF0028CD
:1024F000DED170BD2DE9F041044616460D46476910
:10250000007B80072ED0384603F081FD50BB3EB3E0
:10251000012E02D0022E25D104E0204600F026F93B
:1025200005441DE0384603F070FDE168002841F0E5
:102530001001E16005DA204600F058F80120BDE8FE
:10254000F081C9030BD56268E16A914200D8114657
:10255000A26911442269891A814200DD08460544B6
:10256000002D01DA0220EAE7E16A6068E268814250
:1025700006D29103E06203D522F4003141F010024B
:10258000A6690027AE4213DCE16A814201D90B46FD
:1025900000E0034603EB060C2369ACEB030CAC45EF
:1025A00006DD814201D98C4600E084469C4505D178
:1025B000A760276042F02000A5620DE0AD1BE66930
:1025C000AE1B8142A66000D90846C01A281A2060B6
:1025D0005819606022F0200003490840E0600020A4
:1025E00084F84870ABE70000BFCFD7FFC16821F483
:1025F000001141F08001C1600021816001607047DD
:102600002DE9F047814614460E464FF0FF38324818
:10261000D5685769054209D03846A16903F022FD03
:10262000002811DB2C48C0430540E5602B463246AC
:102630004946384603F019FDA16920F00042B21A5C
:1026400011440028A16103D02046FFF7CFFF404688
:10265000BDE8F08770B504460569C06A61688842C4
:1026600000D80846E16821F42011E160C90312D5C1
:10267000A84208D02246411B2846FFF7C1FF10B1EF
:102680004FF0FF3070BD0020E562C4E90150E06802
:1026900020F48030E060002070BD10B50446C068B2
:1026A00020F02000E060A16AA06988420DD0204699
:1026B000FFF7D0FFE06820F4405040F01000E060E9
:1026C000A06AA0612069E062606044F24001E068B5
:1026D0008843E06010BD000010000200002801D017
:1026E00003F092BC7047000010B5014602A000F054
:1026F0005EF8012010BD0000534947525452454432
:102700003A2052656469726563743A2063616E278A
:1027100074206F70656E3A200000000010B500F064
:102720005FF8BDE81040FFF7D9BF00210160C0E9A4
:102730000110704710207047034640688C460028FF
:1027400018BF88423CBF03464068F8D31868184455
:10275000884207D00CF1030020F00700001D411A49
:10276000521A0146081D0A60FFF7B7BB10B50146B3
:10277000C268900703D0900607D5886A0AE0FEF782
:10278000ABFA01210160881E10BD8B6948681844AE
:102790000B69C01A91F848301BB191F84910401AE2
:1027A00010BD1103FCD50028FADD401E10BD70B528
:1027B00005460C460A2000E06D1C03F063FC35B1B1
:1027C00028780028F8D102E0641C03F05BFC14B107
:1027D00020780028F8D1BDE870400A2003F052BCF0
:1027E00010B5012805D0002103A0FFF7E0FF01206C
:1027F00010BD09A1F8E7000053494752544D454D1B
:102800003A204F7574206F662068656170206D6591
:102810006D6F7279000000003A2048656170206D8C
:10282000656D6F727920636F727275707465640084
:102830005FEA400C08BF91F0000F4FEA8C234FEA8B
:10284000C12243EA51514FEA1C5018BF00F5F04035
:102850004FEA300018BF41F000415FEA6C5C00F0C5
:102860002980BCF1FF3F08BF40F080407047130C47
:1028700006BF12044FF0100C4FF0000C130E04BFF3
:1028800012020CF1080C130F04BF12010CF1040C1E
:10289000930F04BF92000CF1020CD30F04BF52003F
:1028A0000CF1010C11464FF00002A0F11F00A0EB4B
:1028B0000C00704711F0004F08BF704731F0004125
:1028C0003FF4D5AF0B0C06BF09044FF0100C4FF0CE
:1028D000000C0B0E04BF09020CF1080C0B0F04BF17
:1028E00009010CF1040C8B0F04BF89000CF1020CE0
:1028F000CB0F04BF49000CF1010CCCF12003A0EB7D
:102900000C0022FA03F302FA0CF241EA030100F18F
:102910000100704720F07F4C80EA030023F07F47DE
:10292000ACEB070303F57C5300F0004003F1FF0319
:102930002DE980494FEA154B09B44FEA144325EAC3
:102940000B4E24EA03480FF2042606EB132749082E
:102950003E785FEA320203FB0667C7F5000707FB14
:1029600006F64FEA54374FEAD64606F1020607FB51
:10297000066CCCF1005C4FEA1C472CEA074C07FBC5
:1029800006F40CFB06F504EB15464FEA961634BF29
:1029900000204FF000404FEAD13706FB07FC4FEA1A
:1029A0001C4C0CFB0BF7D21B03FB0CF761EB070174
:1029B0000CFB0EF7B0EB074072EB17420CFB08F76D
:1029C00034BFA2EB0742B2EB074261EB17414FEA7B
:1029D0000C444FEA910706FB07FC4FEA1C4C0CFB2A
:1029E0000BF7B0EBC74072EB573203FB0CF734BF69
:1029F000A2EBC742B2EBC74261EB57310CFB0EF7BB
:102A0000B0EBC70072EB57720CFB08F734BFA2EBB8
:102A1000C702B2EBC70261EB5771039F4FEA8161B6
:102A200041EA921104EBCC044FEAD1374FEA8262BB
:102A300006FB07FC42EA90124FEA80604FEA1C4C0A
:102A40000CFB0BF7D21B03FB0CF761EB07010CFB34
:102A50000EF7B0EB074072EB17420CFB08F734BFE0
:102A6000A2EB0742B2EB074261EB17414FEA8C55EC
:102A70004FEA910704EB9C2406FB07FC4FEA1C4C31
:102A80000CFB0BF7B0EBC74072EB573203FB0CF7B4
:102A900034BFA2EBC742B2EBC74261EB57310CFB2C
:102AA0000EF7B0EBC70072EB57720CFB08F734BFA0
:102AB000A2EBC702B2EBC70261EB577115EB4C25D5
:102AC0004FEA816141EA92114FEA82624FEAD137BF
:102AD00042EA901206FB07FC44F100044FEA8060D2
:102AE0004FEA1C4C0CFB0BF7D21B03FB0CF761EB02
:102AF00007010CFB0EF7B0EB074072EB17420CFB23
:102B000008F734BFA2EB0742B2EB074261EB174173
:102B100015EB1C154FEA813141EA92414FEA8232AE
:102B200042EA90424FEA80304FEA0C7644F10004CA
:102B300048EA03434EEA0B484FF0000EB2EB080C94
:102B400071EB030724BF624639464EEB0E0E4FF081
:102B5000000B0018524149414BEB0B0BB2EB080C38
:102B600071EB03077BF1000B24BF624639464EEB45
:102B70000E0E4FF0000B0018524149414BEB0B0B6E
:102B8000B2EB080C71EB03077BF1000B24BF62462C
:102B900039464EEB0E0E51EA020718BF46F0010609
:102BA00016EB0E7655F1000254F1000103D5BDE895
:102BB0008901BDE80088BDE88901BDE80048B61973
:102BC000524141EB0101A3F10103704780807F7EF8
:102BD0007D7C7B7A79787776767574737271717093
:102BE0006F6E6E6D6C6C6B6A6A6968686766666545
:102BF0006464636362616160605F5F5E5E5D5D5CD3
:102C00005C5B5B5A5A595958585757565655555543
:102C10005454535352525251515050504F4F4F4EA3
:102C20004E4D4D4D4C4C4C4B4B4B4A4A4A494949F1
:102C30004848484747474746464645454544444433
:102C4000444343434342424242414141002B9C465C
:102C500030D477002BD01CB54FEA370703B44FF0C0
:102C600010004FF01001BAF1000F06D0BCF1000FB8
:102C7000DCBF40F0080040F008014FF000000FBC3E
:102C8000BDE810400BF1010BBBF1010F08BF5FEA7B
:102C9000170722BF12F1010211F101014FF00041AB
:102CA00043F1000300F0004043EA00007047F9D30D
:102CB0005708D0E746EA064613F1400F4FEA16469A
:102CC0001FDD13F1200FDFBF16430A46002120331A
:102CD0005B42BED0C3F1200746EA064602FA07F778
:102CE0004FEA164646EA0706C3F1200722FA03F226
:102CF00001FA07F721FA03F14FF0000342EA070255
:102D0000A7E746EA020646EA06464FEA164646EABC
:102D10000106BCBF46EA0646360C4FF000034FF0F2
:102D200000024FF0000194E72DE9804C9A4693464B
:102D300070B491E8380007C831EA400C48BF34EA63
:102D4000430C03D5FFF7E6FDFFF780FFF0BCBDE8BD
:102D5000008C2DE9804C9A46934670B491E8380077
:102D600007C810F0804F08BF13F0804F03D100F068
:102D700005F8FFF76BFFF0BCBDE8008C20F07F4743
:102D800080EA030023F07F4C07EB0C03A3F57C5390
:102D900000F00040A3F1FE0392F0000F00F0B380BA
:102DA00095F0000F00F077802DE901494FEA1140BE
:102DB0004FEA144621EA004800FB06FC24EA0647D5
:102DC00008FB06F607FB08F800FB07F718EB0648B8
:102DD0004CEB164C4FEA124B18EB07484FEA1546DE
:102DE0004CEB174022EA0B4E0BFB06FC25EA06478C
:102DF0000EFB06F607FB0EFE0BFB07F71EEB064E5F
:102E00004CEB164C4FF000061EEB074E4CEB174BED
:102E100018EB0B0840F1000018EB0E0B58EB000804
:102E200040F100008F1A4FF000013CBFC943661B00
:102E300014BFB5EB040C00213CBFC943F61B4FEA9D
:102E400017444EEA8E0E27EA04454FEA1C4704FB5E
:102E500007622CEA074C05FB07F70CFB05F604FBA1
:102E60000CFC16EB074642EB174216EB0C4642EB06
:102E70001C421BEB060658EB0202414146EA9E0645
:102E800001D5BDE80189B619524141EB0101A3F119
:102E90000103BDE801894FEA14454FEA114724EACE
:102EA000054621EA074C05FB07F406FB07F70CFB78
:102EB00006F105FB0CFC11EB074144EB17444FEA0C
:102EC000124711EB0C4144EB1C4422EA074C05FB72
:102ED00007F206FB07F70CFB06F605FB0CFC16EBEE
:102EE000074642EB174216EB0C4642EB1C456A18AC
:102EF00054F1000148BF7047B619524141EB01013E
:102F0000A3F10103704795F0000F37D04FEA11424B
:102F10004FEA144721EA024624EA074C02FB07F174
:102F200006FB07F70CFB06F402FB0CFC14EB074452
:102F300041EB17414FEA154714EB0C4441EB1C41A0
:102F400025EA074C02FB07F506FB07F70CFB06F624
:102F500002FB0CFC16EB074645EB174516EB0C463F
:102F600045EB1C42121951F1000148BF7047B619D8
:102F7000524141EB0101A3F1010370474FEA1445AF
:102F80004FEA114724EA054621EA074C05FB07F101
:102F900006FB07F70CFB06F24FF0000605FB0CFCE6
:102FA00012EB074241EB174112EB0C4251EB1C4173
:102FB00048BF7047921841EB0101A3F1010370472C
:102FC00001A000F0CBF8FEE76275736661756C7462
:102FD000000000001CB5002427A0019404F025FD8A
:102FE00004F07CFB29A004F020FD2D4E2D4D01A8FE
:102FF00004F074FA32226946306813F057F8012859
:10300000F5D101A804F06AFA00984188A02901D3FB
:103010009F2141808AB281682348FDF754FD0098C2
:1030200021494FF4007240880C54A0311E4803F02F
:103030009BFE1D490746A031009804F079FA052F40
:1030400003D11AA1009804F073FA00980BF014FB56
:1030500028780028CBD02C70642012F077F8BFF3CA
:103060004F8F1F4801681F4A01F4E061114301605E
:10307000BFF34F8F00BFFDE75B4346475D207461A0
:10308000736B2D656E7472790D0A00005B434647C1
:103090005D207461736B2D72656164790D0A0000A7
:1030A00004000020B801002028B100204E6F746594
:1030B0003A205573652041542B534156452074687E
:1030C000656E2041542B524553455420746F206146
:1030D00070706C79206368616E6765730D0A00001B
:1030E0000CED00E00400FA05014800F0C5B900004D
:1030F00070040020014800F0BFB900002C0400203B
:10310000014800F0B9B9000060030020014800F058
:10311000B3B900001C030020014800F0ADB9000065
:10312000A4030020014800F0A7B90000E803002034
:1031300030B590F840500124AC40C56B6C60046819
:1031400063604368102B036803D099600068C26015
:1031500030BD9A600068C16030BD7047F02201A1A7
:1031600004F020BC2E2E2F436F72652F5372632FF5
:103170006D61696E2E63000008B5002000900B4859
:103180000168C90711D0012101600948694600683A
:1031900012F0C0FE0098002807D006494FF080507A
:1031A0000860BFF34F8FBFF36F8F08BD1404014059
:1031B0000800002004ED00E04FF4897202A107A08E
:1031C00004F0F0FB72B6FEE72E2E2F436F72652FD0
:1031D0005372632F6D61696E2E6300006572726FAA
:1031E000722D68616E646C657200000006490020F3
:1031F000C8610648016941F004010161016941F0BB
:103200004001016170470000B80400200020024026
:10321000064A0021D16106490A6942F002020A61A8
:103220004861086940F0400008617047B804002018
:1032300000200240044B0022DA61044A136943F083
:103240000103136101807047B80400200020024090
:1032500014480022C168CB06134904D5CA6942F05C
:103260000202CA611022C3685B0705D5CB6943F02F
:103270000103CB6142F00402C369DB0707D0CB69CD
:1032800043F00403CB61C16921F00101C161A2F5E2
:103290008071013901D0C2607047C16921F001011C
:1032A000C161704700200240B804002070B5054697
:1032B00000F04AFC0646114C09E0681C07D025B115
:1032C00000F042FC801BA84201D9032070BDE068D9
:1032D000C007F2D1E068800601D52020E060E068F8
:1032E000C00605D4E069C00702D1E068400703D5F5
:1032F000FFF7AEFF012070BD002070BD002002402E
:1033000010B590F821100022022905D00421816314
:1033100080F82020012010BD01680B6823F00E0307
:103320000B6001680B6823F001030B6090F84030DC
:10333000C46B012101FA03F3636080F8211080F867
:103340002020104610BD00002DE9F05F90F82110FC
:103350000024022903D004218163012485E001684F
:103360000A6822F00E020A6001680A6822F001026F
:103370000A603F4E3E4FB215DFF8F4C0DFF8F09020
:10338000DFF8ECA0DFF8E8B0DFF8E4E00168783FB0
:1033900013011502ACF1640CA9F15009AAF13C0A21
:1033A000ABF1280BAEF1140E4FF48018B14227D9BF
:1033B000B9420ED0614512D049451DD0514518D0B3
:1033C000594518D0714501D1424615E0294EB14208
:1033D00001D1012210E0274E1436B14201D1102252
:1033E0000AE0244E2836B14206D0224A3C329142AD
:1033F00001D11A4600E02A461E49091F0A602BE047
:10340000B94213D0614517D0494522D051451DD04E
:1034100059451DD0714501D142461AE0B14202D151
:103420004FF0807215E0134EB14201D1012210E03D
:10343000104E1436B14201D110220AE00D4E28364A
:10344000B14206D00B4A3C32914201D11A4600E00B
:103450002A46074980394A60012180F8211000215D
:1034600080F82010416B01B188472046BDE8F09FED
:1034700080000240080402402DE9F05FC16B0A6839
:1034800001680B68046C4FF0040808FA04F8844DD6
:10349000844E854FDFF814C2DFF81492DFF814A2CF
:1034A000DFF814B2DFF814E218EA020F65D05FEA21
:1034B000437862D50A68920603D40A6822F00402AF
:1034C0000A60DFF8F0814FF48062016808F11408A7
:1034D00013011402414524D9A9420DD0B1420FD0A5
:1034E000B9421AD0614515D0494515D0514501D191
:1034F000120312E0594501D104220EE0714501D1B9
:1035000040220AE06D4D1435A94206D06B4A28329C
:10351000914201D11A4600E022466749091F0A601C
:1035200029E0A94213D0B14215D0B94220D061455B
:103530001BD049451BD0514502D14FF4800217E002
:10354000414502D14FF0806212E0594501D1042279
:103550000EE0714501D140220AE0584D1435A942D0
:1035600006D0564A2832914201D11A4600E022463E
:103570004B4908394A60C16A71E04FF0020808FA05
:1035800004F818EA020F70D05FEA83786DD50A68F4
:10359000920606D40A6822F00A020A60012180F825
:1035A0002110DFF810814FF40072016808F114084F
:1035B00013011402414524D9A9420DD0B1420FD0C4
:1035C000B9421AD0614515D0494515D0514501D1B0
:1035D000120312E0594501D102220EE0714501D1DA
:1035E00020220AE0354D1435A94206D0334A28324C
:1035F000914201D11A4600E022462F49091F0A6074
:1036000029E0A94213D0B14215D0B94220D061457A
:103610001BD049451BD0514502D14FF4001217E091
:10362000414502D14FF0007212E0594501D102220A
:103630000EE0714501D120220AE0204D1435A94247
:1036400006D01E4A2832914201D11A4600E0224695
:10365000134908394A60002180F82010816A002946
:103660001CD0BDE8F05F0847FFE70825A5401542DC
:1036700014D01A0712D50A6822F00E020A6090F8D8
:103680004020C36B012101FA02F25A60816380F885
:103690002110002180F82010016BE0E7BDE8F09FC9
:1036A000080002401C00024030000240440002407A
:1036B000580002406C000240080402401C04024012
:1036C00030B560B11A4B026814219A4209D2194BE5
:1036D0001344B3FBF1F18900016417490AE00120AA
:1036E00030BD134B5B421344B3FBF1F1890001641D
:1036F0000F490839C163022180F82110136843F68D
:10370000F0718B43F0E901142143D0E902452C43C9
:1037100021430469214344692143846921431943B6
:10372000116000214163012242770177084630BDD4
:1037300008040240F8FFFDBF0000024070B50446D7
:1037400090F82000002501280CD0012084F82000EA
:1037500094F821600020012E06D084F82000022574
:10376000284670BD022070BD022684F82160A06347
:103770002068066826F0010606602046FFF7D8FCA0
:10378000E06A00282068016802D041F00E0106E0DE
:1037900021F0040101602068016841F00A01016024
:1037A0002068016841F001010160D9E770B5044665
:1037B00000F0CAF90546601C02D0044800780444B1
:1037C00000F0C2F9401BA042FAD370BD680000208F
:1037D0002DE9F047054626480F460126017E0129BE
:1037E0000FD00121814601762868DFF888804CF2ED
:1037F0005034022808D0A2462046FFF757FDA8B152
:1038000031E00220BDE8F0872046FFF74FFD08BBFE
:103810000120FFF7EBFC2046FFF748FDD8F8101019
:10382000064621F00401C8F810101CE04FF0FF30EC
:103830003860AC6811E02046FFF7EAFC5046FFF71D
:1038400035FDD8F81010060021F00201C8F810105C
:1038500001D03C6007E004F50064D5E9020100EB0B
:10386000C120A042E7D8002189F818103046C9E7E6
:10387000B8040020002002400348016941F08001A3
:103880000161002070470000002002402DE9F05F38
:1038900007461C4888460024017E15461E4601291D
:1038A00009D00121814601764CF2503A5046FFF78B
:1038B000FDFC18B122E00220BDE8F09F012F02D0EC
:1038C000022F00D00427D346DFF83CA0220128466F
:1038D0003146FCF78BFD81B208EB4400FFF7AAFCF0
:1038E0005846FFF7E3FCDAF8102022F00102CAF88C
:1038F000102018B9641CE4B2BC42E7D3002289F856
:103900001820D9E7B8040020002002400649002012
:103910000A69120607D5054A4A60054A4A600969DC
:10392000090600D5012070470020024023016745A9
:10393000AB89EFCD2DE9F84FDFF8C8910024A9F14C
:10394000040B23460F2709F1040AABF1040ED1E062
:103950000125A54006EA0502AA4276D1DFF8A8C1F2
:103960004E68A6EB0C0866452BD00DDC032E34D038
:1039700005DC36B3012E19D0022E2FD11BE0112EFB
:1039800016D0122E2AD119E0B8F5881F19D006DCFE
:10399000B8F5803F15D0B8F5801F1FD111E0B8F5FC
:1039A000001F0ED0B8F5041F18D10AE0CB6815E04F
:1039B000CB681B1D12E0CB6808330FE0CB680C33DB
:1039C0000CE08B682BB1012B4FF0080303D045614D
:1039D00004E0042302E0056100E00023FF2A01D88F
:1039E000064601E000F104064FEA840501D9A5F17D
:1039F0002005D6F8008007FA05FC28EA0C0803FA2F
:103A000005F548EA0508C6F800804D68ED0070D558
:103A10003E4DAE6946F00106AE61AD6924F0030685
:103A200005F0010500953A4D06EB050CDCF8085051
:103A3000A607360F07FA06F825EA0805DFF8D4804E
:103A4000404503D14FF0000825E052E0DFF8C88080
:103A5000404502D14FF001081DE0DFF8C08040452D
:103A600002D14FF0020816E0DFF8B480404502D1E1
:103A70004FF003080FE0DFF8AC80404502D14FF073
:103A8000040808E0DFF8A080404502D14FF00508A7
:103A900001E04FF0060808FA06F848EA0508CCF8F5
:103AA00008804D68D9F80060ED024D4601D51643F7
:103AB00000E096432E604D68DAF80060AD0255468E
:103AC00001D5164300E096432E604D68DBF8006098
:103AD000AD035D4601D5164300E096432E604D6868
:103AE000DEF80060ED03754601D5164300E096430D
:103AF0002E60641C0A681646E2407FF429AFBDE8D8
:103B0000F88F00000804014000001110001002406E
:103B10000000014000080140000C0140001001407D
:103B20000014014000180140001C0140C26821EA55
:103B300002030A4043EA0241016170470AB1016190
:103B400070470904FBE700000148806870470000E7
:103B50006800002070B5040013D021684CF6CC40FA
:103B60000860216845F255500860D4E900014160C1
:103B70002168A0688860FFF7E7FF054641F23C3600
:103B80000DE0012070BD00BFFFF7DEFF401BB0421B
:103B900005D92068C068800701D0032070BD206867
:103BA000C0688007F0D121684AF6AA20086000208A
:103BB00070BD00684AF6AA2101600020704700002D
:103BC00002488168027811448160704768000020D3
:103BD000074810B5016841F010010160032000F0B2
:103BE0009BF80F2000F006F800F044F8002010BD0C
:103BF0000020024010B504461B4888B0C16941F05E
:103C00000401C161C06906A900F00400059068467E
:103C100000F02AF900F048F9039901B14000134976
:103C2000B0FBF1F01249401E0860091D40F2E73078
:103C300008600F490120143908600D481C380168DC
:103C400041F0010101600A482838016841F0010192
:103C50000160002221461E2000F03EF81E2000F0E8
:103C60002DF808B0002010BD0010024040420F00A7
:103C7000280800400F4808B5816941F001018161C1
:103C8000816901F001010091C16941F08051C16178
:103C9000C069002200F0805000900F21901E00F0BB
:103CA0001BF80548416821F0E06141F00071416076
:103CB00008BD00000010024000000140002809DBA0
:103CC00000F01F02012191404009800000F1E02036
:103CD000C0F8001170470000F0B40E4B1B680C4692
:103CE000C3F30223C3F10705042D00D90425191DD0
:103CF000072901D2002300E0DB1E012606FA05F1A8
:103D0000491E214099409E40761E16403143F0BC2A
:103D100002F061B90CED00E0064900F00702086806
:103D20004FF6FF03184040EA0220034A10430860A0
:103D3000704700000CED00E00000FA052DE9F047A7
:103D40000F46050061D0434E306800F00700B842CE
:103D500009D2306820F0070038433060306800F046
:103D60000700B84251D128683B4C810712D5400763
:103D700003D5606840F4E06060602878000703D5F0
:103D8000606840F4605060606068A96820F0F000EE
:103D9000084360602878C00728D06868012810D0E0
:103DA0002168022810D0890700292EDA616821F0E5
:103DB000030101436160FFF7C7FE804641F2883985
:103DC0000DE021688903EFE78901EDE7FFF7BCFE0D
:103DD000A0EB0801494502D90320BDE8F0876068DF
:103DE000696800F00C00B0EB810FEFD1306800F093
:103DF0000700B8420BD9306820F007003843306024
:103E0000306800F00700B84201D00120E5E72878CB
:103E1000400705D56068E96820F4E0600843606009
:103E20002878000706D56068296920F4605040EAC8
:103E3000C100606000F058F86168084AC1F30311DE
:103E4000515CC8400649086006480068FFF7D2FE8A
:103E50000020C2E70020024000100240F66E010878
:103E6000740000206C0000200F2202600C4A53688E
:103E700003F003034360536803F0F0038360536867
:103E800003F4E063C36052684FF4E06303EAD202D4
:103E900002610448006800F00700086070470000F5
:103EA00000100240002002400448054900684968AB
:103EB000044AC1F30221515CC840704774000020DD
:103EC00000100240066F010804480549006849686F
:103ED000044AC1F3C221515CC840704774000020FD
:103EE00000100240066F01080E4A51680E4801F0AA
:103EF0000C03042B11D0082B0FD10C48C1F38343C2
:103F0000C903C05C0AD55168084AC1F34041921EFA
:103F1000515C054A5043B0FBF1F0704704494843F7
:103F2000704700000010024000127A00E66E01089F
:103F300000093D002DE9F84F040070D02078C04DF5
:103F4000C00749D06868C0F38100012807D06868BD
:103F5000C0F38100022809D16868C00306D528682B
:103F6000800339D560680028E7D035E06068B0F597
:103F7000803F0BD010B1B0F5A02F11D0286820F4ED
:103F800080302860286820F4802002E0286840F40F
:103F900080302860606890B1FFF7D6FD06460AE0E1
:103FA000286840F480202860F0E700BFFFF7CCFDD0
:103FB000801B642873D828688003F7D50CE0FFF7CE
:103FC000C3FD064605E000BFFFF7BEFD801B642869
:103FD000F0D828688003F7D420789A4E80074FF0F5
:103FE00001094FF0000839D5686810F00C0F07D0B0
:103FF0006868C0F38100022809D16868C00306D44C
:104000002868800714D52069012808D110E02069AC
:10401000B0B1C6F80090FFF797FD074605E00AE14A
:10402000FFF792FDC01B0228C4D828688007F7D587
:104030002868616920F0F80040EAC10028600DE0BE
:10404000C6F80080FFF780FD074604E0FFF77CFD1F
:10405000C01B022823D828688007F7D420780007DF
:104060002CD57948A169D9B1C0F80090FFF76CFD53
:10407000074604E0FFF768FDC01B02280FD8686AF6
:104080008007F7D571484FF4FA510068B0FBF1F0A2
:10409000009000BF0098411E0091FAD20EE080E02F
:1040A000C0F80080FFF750FD074604E0FFF74CFD25
:1040B000C01B022875D8686A8007F7D420784007AB
:1040C00060D5E8690027C00008D4E86940F0805056
:1040D000E861E869012700F0805000905C480168C1
:1040E000C90513D40168834641F480710160FFF76C
:1040F0002BFD824606E000BFFFF726FDA0EB0A007D
:1041000064284ED8DBF80000C005F5D5E06801282A
:104110000AD008B1052813D0286A20F001002862CF
:10412000286A20F0040002E0286A40F001002862BA
:10413000E06841F2883B98B1FFF706FD82460BE04C
:10414000286A40F004002862EEE700BFFFF7FCFC9D
:10415000A0EB0A0159455AD8286A8007F6D50CE029
:10416000FFF7F2FC824605E0FFF7EEFCA0EB0A0148
:1041700059454CD8286A8007F6D41FB1E86920F069
:104180008050E861E06988B36968C1F38101022960
:1041900044D00228C6F8608004D0FFF7D5FC04465E
:1041A00038E034E0FFF7D0FC074604E0FFF7CCFC32
:1041B000C01B02282BD828688001F7D4206AB0F5EC
:1041C000803F05D16868A16820F40030084368602A
:1041D000D4E908010843696821F474110843686050
:1041E000C6F86090FFF7B0FC044606E025E000BF8B
:1041F000FFF7AAFC001B022809D828688001F7D520
:104200001BE000BFFFF7A0FC001B022802D903201F
:10421000BDE8F88F28688001F4D40EE00128F7D0BB
:104220006868226A00F48031914204D1616A00F426
:104230007010884201D00120EAE70020E8E7000082
:1042400000100240000042428004424274000020FC
:10425000007000407047000038B5044600684268AE
:104260008168C9434B0606D5CB0704D1D3435B060F
:1042700001D4216C05E08B0708D4D3431B0605D479
:10428000616C01B02046BDE8304008478B0601D57F
:104290004B0646D4D3439B0643D44B060AD494F82A
:1042A0005130032B3ED0636D43F004036365C36854
:1042B00083680093890609D4616D41F0010161654D
:1042C00081680091016821F040010160606D002863
:1042D00027D02068416821F0E0014160012084F886
:1042E0005100900722D02068416821F0030141600D
:1042F000104DE06C40B14563E06CFFF725F818B154
:10430000606D40F040006065A06C002809D04563F6
:10431000A06CFFF719F8002803D0606D40F0400052
:10432000606538BDC1688068009038BD2046FFF7E1
:1043300091FF38BD4956000870B5040009D0606A85
:10434000002540B125616561A56294F8510040B136
:104350000CE0012070BD6068B0F5827FF4D0E561AB
:10436000F2E784F85050204600F040F8022084F82C
:1043700051002068016821F040010160A088218976
:1043800000F4827001F404410843A18901F4006142
:104390000843217C01F002010843217D01F0010165
:1043A0000843218B01F400710843217F01F038019B
:1043B000084394F8201001F080010843218D01F496
:1043C0000051084321680860A069042101EA1040F7
:1043D000216848602068C16921F40061C161656598
:1043E000012084F85100002070BD000030B585B078
:1043F00000240094019402940394006818498842B0
:104400002BD11848816941F480518161816901F49F
:1044100080510491816941F0040181618069124DEC
:1044200000F004000490A0200090022001900320DE
:10443000039069462846FFF77DFA4020CDE9000445
:10444000694628460294FFF775FA002205212320C9
:10445000FFF742FC2320FFF731FC05B030BD000020
:104460000030014000100240000801402DE9FF4FDC
:1044700081B01D46934604464FF001090E9EFFF79A
:1044800063FB074694F851006168012806D0B1F536
:10449000827F3CD1A168C9BB042838D1029800288A
:1044A00071D0BBF1000FFBD0002DF9D094F8500073
:1044B00001282CD04FF0010A84F850A094F8510044
:1044C000042802D0052084F851004FF00008C4F8F9
:1044D0005480C4F838B0E587A58702992163E58642
:1044E000A586C4F84080C4F8448020680168490665
:1044F00003D4016841F040010160E068B0F5006F4D
:10450000606808D0F0B3012D49D081E0FFE70220B8
:1045100005B0BDE8F08F08B1012D39D1206B2168BD
:104520000088C860206B801C2063E08E401EE086FF
:104530002EE02068816889070FD5E18E69B1B9F155
:10454000010F0AD1216B0988C160206B801C206398
:10455000E08E401EE0864FF0000920688168C907A0
:104560000CD0E18F51B1C068A16B0880A06B801C9A
:10457000A063E08F401EE0874FF00109FFF7E4FAE7
:10458000C01B01E00BE067E0B04201D3701C50D1CA
:10459000E08E0028CDD1E08F0028CAD13EE0206B0C
:1045A000216800780873206B401C2063E08E401E59
:1045B000E0862DE02068816889070FD5E18E69B11A
:1045C000B9F1010F0AD1216B09780173206B401CEE
:1045D0002063E08E401EE0864FF00009206881686D
:1045E000C9070CD0E18F51B1C068A16B0870A06BF6
:1045F000401CA063E08F401EE0874FF00109FFF7E9
:10460000A3FAC01BB04202D3701C01D011E086B1E6
:10461000E08E0028CED1E08F0028CBD13A4631463B
:10462000204601F019F850B12020606584F85080D0
:1046300012E084F851A084F85080032068E7A06855
:1046400018B92068C1688068009084F851A084F887
:104650005080606D0028F1D0012059E7704710B5F7
:1046600004460068406994F84110C0F3C010212945
:1046700011D180B12068143050E8001F21F0800172
:1046800040E80012002AF5D1A06B08B1FEF738FE11
:10469000204601F0BDF92068406994F84210C0F34B
:1046A0008010222911D180B12068143050E8001FF9
:1046B00021F0400140E80012002AF5D1E06B08B17A
:1046C000FEF71EFE204601F07CF9002010BD704769
:1046D000F8B5016804460868CA684B6910F00F0F06
:1046E0004FF0000559D003F0010602F490773743EC
:1046F00065D0C10705D0D10503D5616C41F001013A
:104700006164410705D5D90703D0616C41F002010E
:104710006164810705D5D90703D0616C41F00401BC
:104720006164010707D502F02001314303D0616CB9
:1047300041F008016164616C00293AD0800604D51B
:10474000900602D5204601F071F920684069616C3D
:10475000C0F38010090700D460B3204601F031F99E
:1047600020684069400621D52068143050E8001FB9
:1047700021F0400140E80012002AF5D1E06BA8B119
:104780006D494163E06BFEF7DFFD002811D0E06B5F
:10479000416B01B0BDE8F040084783060FD5930692
:1047A0000DD52046BDE8F84001F040B92046FFF79E
:1047B0008EFFF8BD2046FFF78AFF6564F8BD266BC3
:1047C0002023012E7CD1C6067AD5D60678D5086876
:1047D0004868009048694FF00206400640D5E16BFA
:1047E000086840680004000CE8D0A28D8242E5D938
:1047F000E085886920282DD020680C3050E8001F03
:1048000021F4807140E80012002AF5D120681430AC
:1048100050E8001F21F0010140E80012002AF5D104
:104820002068143050E8001F21F0400140E80012D9
:10483000002AF5D184F84230256320680C3050E816
:10484000001F21F0100140E80012002AF5D1E06BB2
:10485000FEF756FD6663A08DE18D401A81B22AE015
:10486000A08DE18D401A81B2E08D0028A6D00029EC
:10487000A4D022680C3252E8000F20F4907042E875
:104880000007002FF5D12068143050E8002F22F0E7
:10489000010240E80027002FF5D184F8423025635B
:1048A00020680C3050E8002F22F0100240E800236E
:1048B000002BF5D166632046FFF7D0FEF8BDFFE779
:1048C00005062BD5150629D594F841002128F5D1E8
:1048D000A068B0F5805F01D12069B0B1206A411CA9
:1048E0002162216800784860E08C401E0004000CC2
:1048F000E084E3D12068C16821F08001C1602068B4
:10490000C16841F04001C160D8E7206A0088C0F367
:1049100008004860206A801C2062E5E74006CDD58B
:104920005006CBD5CA68204622F04002CA6084F8FF
:10493000413000F015FAC1E77958000870B504005D
:1049400004D094F84100002510B106E0012070BDAC
:1049500084F84050204600F023F8242084F84100D9
:104960002068C16821F40051C160204601F0C0F800
:104970002068016921F4904101612068416921F0BA
:104980002A0141612068C16841F40051C160656439
:10499000202084F8410084F842006563002070BD47
:1049A0002DE9F04786B00025009501950295039505
:1049B0000446DFF85082D0F800C093480221032259
:1049C000924B102680274FF48069C4455AD1D0F805
:1049D00018C04CF4804CC0F818C0D0F818C00CF4C3
:1049E000804CCDF810C0D0F818C04CF0040CC0F8C2
:1049F00018C08069039200F0040004900802CDE919
:104A00000001694698461846FEF794FFCDE90095E7
:104A1000694640460295FEF78DFFDFF8F8817C4934
:104A20004046B946C0E90015C0E90257C8F8105021
:104A3000C8F81450C8F81850C8F81C50FEF740FECB
:104A400008B1FEF7B9FB734F7148C4F83C80443796
:104A50001438C8F824403860C7E90165C7E90395F0
:104A60007D61BD613846FD61FEF72AFE08B1FEF7A3
:104A7000A3FBA7630022052125207C62FFF72CF908
:104A8000252061E0DFF890814FF0200AC44560D115
:104A9000D0F81CC04CF4003CC0F81CC0D0F81CC0BE
:104AA0000CF4003CCDF810C0D0F818C04CF0040C49
:104AB000C0F818C08069039200F00400049004203C
:104AC000CDE90001694698461846FEF733FF0820F5
:104AD000CDE90005694640460295FEF72BFFDFF859
:104AE00034814B4908F1880840461431C0E900156B
:104AF000C0E90257C8F81050C8E9055AB946C8F8C5
:104B00001C50FEF7DDFD08B1FEF756FB414F404853
:104B1000C4F83C80CC372830C8F824403860C7E956
:104B20000165C7E903957D61BD613846FD61FEF70A
:104B3000C7FD08B1FEF740FBA76300220521262030
:104B40007C62FFF7C9F82620FFF7B8F806B0BDE889
:104B5000F087324B9C45F9D1C36943F48023C3618C
:104B6000C36903F480230493836943F008038361DA
:104B70008069CDE9009100F00800CDE90320DFF85D
:104B8000A08069464046FEF7D5FE4FF40060CDE9AF
:104B90000005694640460295FEF7CCFEDFF88480AA
:104BA0001B4940462839C0E90015C0E90257C8F83A
:104BB0001050C8E9055AB946C8F81C50FEF780FDE8
:104BC00008B1FEF7F9FA174F1148C4F83C80443792
:104BD0003C38C8F824403860C7E90165C7E9039547
:104BE0007D61BD613846FD61FEF76AFD08B1FEF7E3
:104BF000E3FAA7630022052127207C62FFF76CF807
:104C00002720A1E7003801400010024000080140C1
:104C1000580002401C0300200044004000480040AF
:104C2000000C01402C04002090F84230202B01D0D1
:104C30000220704721B11AB10023036300F0B4BF12
:104C400001207047704770472DE9F843044690F8FB
:104C50004100984616460D46202802D00220BDE8A5
:104C6000F88385B17EB100206064212084F8410082
:104C7000FEF76AFFA6848146E684A0682027B0F587
:104C8000805F02D003E00120E9E7206910B12E46E1
:104C900000250EE000260CE08021204600F0CCFF2D
:104CA000A8B9C6B116F8010B21684860E08C401E17
:104CB000E084E08C4B464FF00002CDF800800028E5
:104CC000EAD14FF04001204600F0B6FF40B184F831
:104CD00041700320C3E735F8020BC0F30800E3E797
:104CE00084F841700020BAE770B5044690F841009E
:104CF000202801D0022070BD49B342B32162A284B2
:104D0000E28400206064212384F84130A56B114BBC
:104D1000AB62A56B104BEB62A56B104B2B63A36BC7
:104D20005863256813462A1DA06BFEF707FD21680E
:104D30006FF0400008602068143050E8001F41F018
:104D4000800140E80012002AF5D1002070BD01204A
:104D500070BD000077590008B9590008895800084B
:104D60000549884201D1002003E00449884202D16C
:104D700001200FF005BF70478C020020D4020020F4
:104D80007047000001A0FEF7E9F9FEE76861726470
:104D90006661756C740000001D4808B5416941F0FA
:104DA000010141614069002200F0010000900521ED
:104DB0000C20FEF791FF0C20FEF780FF002205215A
:104DC0000D20FEF789FF0D20FEF778FF0022052158
:104DD0000E20FEF781FF0E20FEF770FF0022052156
:104DE0000F20FEF779FF0F20FEF768FF0022052154
:104DF0001020FEF771FF1020FEF760FF0022052152
:104E00001120FEF769FFBDE808401120FEF756BFEC
:104E1000001002407CB509F077FC0FF095FD60B101
:104E2000CF2271A176A002F0BDFD502080F3118841
:104E3000BFF34F8FBFF36F8FFEE775A002F0A2FDA7
:104E400003220021012010F0C1FD754C0022042135
:104E5000A060062010F0BAFD20600022042102208C
:104E600010F0B4FD6F4E002560600421002208465A
:104E700010F0ACFD46F825006D1C042DF5D3A0689C
:104E800038B32068002831D0606800283BD000206B
:104E900056F82010002943D0401C0428F8D360495C
:104EA00001202831CDE900010023C0225EA1614824
:104EB00011F074FB012840D0E0224BA150A002F079
:104EC00071FD502080F31188BFF34F8FBFF36F8FB8
:104ED000FEE7D92244A14AA002F064FD502080F3ED
:104EE0001188BFF34F8FBFF36F8FFEE7DA223EA129
:104EF00043A002F057FD502080F31188BFF34F8F7D
:104F0000BFF36F8FFEE7DB2237A13DA002F04AFD21
:104F1000502080F31188BFF34F8FBFF36F8FFEE7F0
:104F2000DD2231A136A002F03DFD502080F3118832
:104F3000BFF34F8FBFF36F8FFEE739490520143160
:104F4000CDE9000100234FF400723BA13C4811F071
:104F500025FB01280CD0E22223A129A002F022FD8A
:104F6000502080F31188BFF34F8FBFF36F8FFEE7A0
:104F70002B4904200C31CDE900014FF4C07400230B
:104F8000224630A1314811F009FB01280CD0E4225F
:104F900015A11BA002F006FD502080F31188BFF37D
:104FA0004F8FBFF36F8FFEE71D4902201031CDE90F
:104FB00000010023224626A1274811F0EFFA01281C
:104FC0000CD0E52208A10EA002F0ECFC502080F3EA
:104FD0001188BFF34F8FBFF36F8FFEE7BDE87C40B2
:104FE0001EA002F0CFBC00002E2E2F436F72652F43
:104FF0005372632F6672656572746F732E6300005F
:10500000636F6E6669672D6173736572740000006B
:10501000756172742D7472616E732D696E6974009E
:1050200000000020D001002064656661756C745436
:1050300061736B00455700084E6574506F6C6C00CF
:10504000715200085561727452780000695D000861
:10505000436F6E6669670000D52F00087461736B3B
:10506000732D637265617465640000002DE9F04181
:1050700086B000242C480094019402940394816922
:1050800041F010018161816901F010010491816991
:1050900041F020018161816901F020010491816961
:1050A00041F004018161816901F004010491816989
:1050B00041F00801816180691C4F00F008004FF445
:1050C00000550490002229463846FEF737FDDFF8E8
:1050D0006080002202214046FEF730FD0095022646
:1050E00001250396CDE9015469463846FEF722FCB6
:1050F00010480095CDE9010469464046FEF71AFCC8
:10510000CDE90065CDE9024669464046FEF712FC4E
:10511000062100220846FEF7DFFD0620FEF7CEFD41
:1051200006B0BDE8F0810000001002400010014010
:10513000000C014000002110084810B5064901602C
:105140000421416040F6FF718160FEF703FD0028F5
:1051500000D0012010BD000000300040E001002020
:10516000104810B50E4901604FF482714160002172
:1051700002228160C0E9031201224261520282616F
:105180001022C0E90721416281620A21C162FFF752
:10519000D3F8002803D0BDE81040FEF70DB810BDCD
:1051A00000300140EC0100200C4810B50A490160B4
:1051B0004FF4E1314160002181600C22C160C0E9FF
:1051C00004128161C161FFF7B9FB002803D0BDE87B
:1051D0001040FDF7F1BF10BD00380140440200202F
:1051E0000C4810B50A4901600B490C22096841605E
:1051F00000218160C160C0E904128161C161FFF7D3
:105200009DFB002803D0BDE81040FDF7D5BF10BDC1
:10521000004400408C020020540000200C4810B5CF
:105220000A4901600B490C224968416000218160F4
:10523000C160C0E904128161C161FFF77FFB0028F2
:1052400003D0BDE81040FDF7B7BF10BD00480040D7
:10525000D40200205400002001A0FDF77FFFFEE7EC
:105260006D656D6D616E616765000000FEE70000B1
:105270001FB56AA002F0D9FB01F0C6FC04466CA081
:1052800002F0D3FB6FA002F0D0FB002108460EF025
:1052900051FF73A002F0C9FB32200FF057FF76A038
:1052A00002F0C3FB2189A27A48BA000440EA022333
:1052B000E07A4DBA2D04034345EA02251B06ADB240
:1052C00043EA05234DBA49BA0904EDB241EA022185
:1052D00043EA0523014343EA11600190A189A27BBF
:1052E00048BA000440EA0223E07B4DBA2D04034390
:1052F00045EA02251B06ADB243EA05234DBA49BA79
:105300000904EDB241EA022143EA0523014343EADD
:1053100011600290218AA27C48BA000440EA02236C
:10532000E07C4DBA2D04034345EA02251B06ADB2CD
:1053300043EA05234DBA49BA090441EA0221EDB214
:10534000014343EA0523514E43EA116001270390CC
:10535000376000200FF0E0FC01464DA002F04EFB4C
:1053600052A002F062FB03AA02A901A805F098FC72
:105370000720306054A002F058FB10F049FA804634
:1053800010F040FA054600200FF0C6FC2B46544DA5
:10539000CDF800800246296852A002F02FFB286851
:1053A000012805D04FF47A7420460FF0CFFEFBE7BA
:1053B00059A002F03AFB5D4D2F605DA002F035FB75
:1053C00000F05EFF10F024FA074610F01BFA0146C9
:1053D0003A4660A002F012FB67A002F026FBB0463E
:1053E0004FF00809694F00E02EB9C8F8009068A096
:1053F00002F01BFB012600F0F3FE10B1204606F080
:1054000039F90221386810F021FF28680028EBD014
:1054100003F062FC03F05CFBE6E700005B4E4554E2
:105420005D207461736B2D656E7472790D0A0000D6
:105430005B4E45545D20636F6E6669672D6F6B0D23
:105440000A0000005B4E45545D2074637069702D46
:10545000696E697420656E7465720D0A0000000043
:105460005B4E45545D2074637069702D696E69747C
:1054700020657869740D0A005B4E45545D20706F9D
:1054800073742D64656C61790D0A00003C00002086
:105490005B4E45545D206E657469662D63616C6C6E
:1054A0002068776D3D256C750D0A00005B4E4554F4
:1054B0005D206E657469662D696E697420656E7411
:1054C00065720D0A000000005B4E45545D206E655C
:1054D0007469662D696E697420657869740D0A00B7
:1054E000500000205B4E45545D20706F73742D6931
:1054F0006E6974206F6B3D256C642068776D3D2567
:105500006C7520667265653D256C75206D696E3D14
:10551000256C750D0A0000005B4E45545D207072CD
:10552000652D72656164790D0A0000003800002065
:105530005B4E45545D2073746172742D6E65747793
:105540006F726B2D7461736B732063616C6C0D0AE9
:10555000000000005B4E45545D20706F73742D7227
:105560006561647920667265653D256C75206D699D
:105570006E3D256C750D0A005B4E45545D206E65D1
:105580007469662D72656164790D0A000800002057
:105590005B4E45545D206C6F6F702D656E74657247
:1055A0000D0A000000F078BC2DE9F04107460B48D9
:1055B00015460E460078532801D000F06DFCEFF33D
:1055C0001184202080F311882A463146384600F0A5
:1055D00007F8E1B281F31188BDE8F081D4A700207B
:1055E00070B50E46144900EB400001EBC0051446AF
:1055F000E86A183520B101280FD0022805D113E040
:10560000284600F07BFCA04201D2002411E0224693
:105610003146284600F0AAFC0BE0284600F06EFC5C
:10562000A042F4D20446F2E73146284600F071FC6D
:105630000446204670BD0000D4A700200148FEF7B4
:105640000BBE0000EC01002010B5406A0021C187AC
:10565000C186FEF7FFFD10BDF8B515460E460B4698
:10566000009204460122022100F010F840B93346AE
:10567000002280212046009500F008F8002804D080
:10568000606D40F0200060650320F8BD2DE9F8430F
:105690001E46914688460446089DFEF755FA401B73
:1056A000351AFEF751FA074625480068C0F3CB309B
:1056B000684338E0701C37D0FEF746FAC01BA8429A
:1056C00003D215B1009860B32CE02068416821F046
:1056D000E00141606068B0F5827F0BD1A068B0F551
:1056E000004F02D0B0F5806F04D12068016821F02E
:1056F00040010160A06AB0F5005F09D1206801682F
:1057000021F4005101602068016841F400510160FA
:10571000012084F85100002084F850000320BDE8E7
:10572000F8830025401E00902068816838EA010057
:1057300004D000214945BDD10020F0E70121F9E75F
:1057400074000020002411A002F01CF9FFF7F4FC03
:10575000124E4FF4005548B111A002F066F92946E7
:105760003046FEF7E3F9012C08D00AE012A002F05F
:105770005CF9012429463046FEF7D8F91448FEF7B3
:1057800018FA4FF4FA700FF0E1FCE8E7646566611F
:10579000756C742D7461736B000000000010014083
:1057A0005B424F4F545D20697764672D696E697461
:1057B0002D6661696C0D0A005B424F4F545D206994
:1057C0007764672D737461727465640D0A0000005C
:1057D000E001002010B511F023F8012803D0BDE846
:1057E000104010F085B810BD30B58FB02821684644
:1057F000FBF7D8F914210AA8FBF7D4F909200121F5
:1058000000904FF48030002404910691CDE901040A
:105810000225CDE907504FF4E01009906846FEF7E5
:1058200089FB60B90F20CDE90A056802CDE90C407B
:1058300002210AA80E94FEF781FA002801D0FDF794
:10584000BBFC0FB030BD704704480168C90703D0E6
:10585000016821F001010160FEF7B2B910080040B3
:10586000022009F03DBD032009F03ABD00200DF0F3
:10587000F9B901200DF0F6B910B5406A0021C185D3
:10588000C184FEF724FF10BD70B5446A20684069EA
:1058900094F84110C0F3C0100025212904D118B19B
:1058A000E584204600F0B4F82068406994F842107E
:1058B000C0F38010222904D118B1E585204600F0FC
:1058C00080F8606C40F0100060642046FEF7FFFE38
:1058D00070BD10B50146406A096809684FF00002C2
:1058E00089062ED4C28501680C3151E8003F23F4AB
:1058F000807341E80034002CF5D10168143151E87F
:10590000003F23F0010341E80034002CF5D1016889
:10591000143151E8003F23F0400341E80034002CEB
:10592000F5D1202180F84210016B012909D10168CD
:105930000C3151E8003F23F0100341E80034002C03
:10594000F5D14263016B012902D0FFF77BF910BD4D
:10595000818DFEF783FE10BD10B5406A01214163C1
:10596000016B012902D0FFF76EF910BD818D490846
:10597000FEF774FE10BD10B50146406A096809685B
:10598000890616D40021C1840168143151E8002F22
:1059900022F0800241E80023002BF5D101680C3190
:1059A00051E8002F42F0400241E80023002BF5D1DE
:1059B00010BDFFF7D5F910BD10B5406AFFF7E0F94B
:1059C00010BD01680C3151E8002F22F4907241E8BB
:1059D0000023002BF5D10168143151E8002F22F08B
:1059E000010241E80023002BF5D1016B012909D107
:1059F00001680C3151E8002F22F0100241E8002329
:105A0000002BF5D1202180F842100021016370475E
:105A100001680C3151E8002F22F0C00241E8002358
:105A2000002BF5D1202180F84110704708B590F87F
:105A30004210222901D0022008BD82684FF4805311
:105A40009A4201D1016921B1816A9A421BD04AB1BF
:105A50000AE00268816A5268C2F308020A80816A19
:105A6000891C08E0026972B10268526802F07F0284
:105A70000A70816A491C8162C18D491E0904090CA2
:105A8000C18503D01BE002685268F1E70168CA686B
:105A900022F02002CA600168CA6822F48072CA60DB
:105AA00001684A6922F001024A61202180F842100F
:105AB00000214163026B012A03D0FFF7C3F80020E5
:105AC00008BD016301680C3151E8002F22F010027B
:105AD00041E80023002BF5D101680A68D20602D5FF
:105AE0000A6849680091818DFEF7B8FDE7E700007C
:105AF00070B5044600680169E26821F44051114321
:105B000001612169A0680843616908432168CA6886
:105B100041F20C639A430243CA6020684169A2695A
:105B200021F44071114341611E492068884202D12D
:105B3000FEF7CAF901E0FEF7B7F900EBC00101EB8F
:105B40000012606864218000B2FBF0F3B3FBF1F354
:105B50006FF018067343B2FBF0F5B2FBF0F605EBFD
:105B60008305322303EB0515B5FBF1F5B6FBF1F622
:105B700005F0F00505EB0615B2FBF0F6B2FBF0F010
:105B8000B0FBF1F06FF01802504306EB800003EB1E
:105B90000010B0FBF1F0216800F00F00284488608D
:105BA00070BD00000038014038B58162044682852E
:105BB000002013466064222284F84220E56B1B4AD1
:105BC000AA62E56B1A4AEA62E56B1A4A2A63E26B3B
:105BD00050630A462168E06B091DFDF7AFFD2068A0
:105BE000016840680090206948B120680C3050E896
:105BF000001F41F4807140E80012002AF5D12068AE
:105C0000143050E8001F41F0010140E80012002A62
:105C1000F5D12068143050E8001F41F0400140E801
:105C20000012002AF5D1002038BD0000D35800082A
:105C300059590008895800082DE9F8439846174635
:105C40000D460446089E24E0701C22D0FDF77CFF20
:105C5000A0EB0800B0421AD8CEB12068C16849074D
:105C600017D5802D15D0402D13D00168C9430907E1
:105C70000FD401680025406800902046FFF7A1FE80
:105C80000820606484F840500120BDE8F8830320B8
:105C9000FBE72068006835EA000004D00020B84225
:105CA000D2D00020F1E70120F9E70000084808B54C
:105CB00000680168C943C90604D4016840680090BF
:105CC00001F0D6FDBDE808400148FEF701BD000027
:105CD000440200201CB5002000900D4800680168B7
:105CE000C943C90610D40168406801906946002084
:105CF0000EF050FE009838B106494FF08050086011
:105D0000BFF34F8FBFF36F8F0148FEF7E1FC1CBD5F
:105D10008C02002004ED00E01CB5002000900D482E
:105D200000680168C943C90610D401684068019041
:105D3000694601200EF02EFE009838B106494FF05A
:105D400080500860BFF34F8FBFF36F8F0148FEF79D
:105D5000BFFC1CBDD402002004ED00E0014AC2E9F2
:105D60000001704754000020C6B000244294ADF8F2
:105D70000C418DF810410EF097FE28B136A0FDF7CA
:105D8000EDF900200FF052FC37A001F0FBFD3B4D78
:105D90004FF0FF360A2341AA31460020419410F00B
:105DA000DFFD012814D14198C00702D0002007F080
:105DB000D7FC4198800702D5012007F0D1FC41981B
:105DC000C10501D585F81043800501D585F8244625
:105DD00044AA43A942A80EF0F7FE294F0AE04598CD
:105DE0004290ADF80C418DF8104144AA43A942A855
:105DF0000EF0EAFE429830B9002245A9386810F04A
:105E000055F90128EBD000F0FFFE8079012810D071
:105E100000200EF0ABFC01200EF0A8FC002003F0E7
:105E200049FE012003F046FEB4E7694600200EF06B
:105E300085FB694600200EF0DBFA0028F5D103E06F
:105E4000694601200EF07AFB694601200EF0D0FA77
:105E50000028F5D1E2E70000756172742D7374615A
:105E600072742D6661696C00756172742D74617352
:105E70006B2D7374617274656400000048C8002063
:105E80000000002001A0FDF769F9FEE77573616766
:105E9000656661756C74000010B5134C482120468E
:105EA000FAF780FE01202061606110A0A06104F17A
:105EB0004800E0614FF4006020620020A062606250
:105EC000E0620AA1216304F6480161631021A16325
:105ED0002064E06360640849C0F10F028A5C2254C8
:105EE000401C1028F8D310BDD4A700205465726D53
:105EF000696E616C00000000B37001080269C1683E
:105F00008A4203D88068401A104400E0501A401EAC
:105F100070472DE9F047C4681746894606464FF09A
:105F200000083069A04201D9051B02E0B168201ABF
:105F30000D1AB0686D1E001BA84200D80546BD4270
:105F400000D33D4670682A4620444946FAF7BBFD17
:105F5000B0687F1B2C44A844A944A04200D100246F
:105F6000F460002FDDD14046BDE8F0872DE9F04117
:105F700004468846D4E90207C51BE16860681646F6
:105F80000844B54206D94146FAF79DFDB819E060CC
:105F9000BDE8F0812A464146FAF795FD761B08EBED
:105FA000050132466068FAF78EFDE660F0E74900C9
:105FB00050EAC12018BF04204A0D18BF40F001006C
:105FC00040F2FF72B2EB515F08BF40F002000128BF
:105FD00008BF052070470907090E002804DB00F1FF
:105FE000E02080F80014704700F00F0000F1E0207E
:105FF00080F8141D704730380A2801D201207047FC
:106000000020704700207047FEE70020704748F2EC
:106010000101884209D0A0F50041023905D0A0F560
:106020000041033901D00020704701207047000073
:1060300010B50C4618B10AA1FAF706FE10B14FF0E0
:10604000FF3010BD600702D548F2020010BD2007E6
:1060500002D548F2030010BD48F2010010BD000057
:106060003A7474004FF0FF307047A0F50043023BD4
:1060700006D0A0F50043033B02D04FF0FF3070473D
:1060800000207047704700002DE9F0470F460400DC
:106090006FF0050556D014F1100F53D02169002977
:1060A00050D004F110066FF00C08002F3CD02AB13C
:1060B00040F22D2231A13AA004F0A8FE2078A16A76
:1060C00005F06CFC05004FF0FF393FD06F6008F021
:1060D0006DFC384609F01CF82946304608F031FDC1
:1060E00098B36C680021204608F0CCFF00212046C0
:1060F0000CF0CCF9002120460CF05AFD002211468C
:1061000020460BF055FC0021204609F0CFFE00266A
:1061100005F10C0004466E6008F0F1FC04B1EE607D
:10612000284605F09DFD1FE0404604F04BFD01466A
:10613000304608F006FD28B9A36A1BB100221146BB
:10614000204698472846BDE8F0870FE0404604F017
:1061500039FD0146304608F0F4FC28B9A36A1BB1AA
:1061600000221146204698474846ECE7A36A1BB137
:1061700000221146204698470020E4E72E2E5C447A
:106180007269766572735C4C7749505C7372635CBC
:106190006170695C6170695F6D73672E63000000F8
:1061A000657870656374206E6577706362203D3D2D
:1061B000204E554C4C206F7220657272203D3D2060
:1061C0004552525F4F4B0000014900204863704721
:1061D00000000020014900200863704700000020F3
:1061E0000148406B70470000000000200148006B30
:1061F00070470000000000200648D0E90612114355
:10620000026A406A1143014301D000207047012017
:10621000704700000000002010B504460EF01EFE7E
:10622000104900208A69944201D188610DE0CA6951
:10623000944201D1C86108E00A6A944201D108621F
:1062400003E04A6A944200D14862D1E906231A4326
:106250000B6A1A434B6A1A4300D1C862BDE810406A
:106260000EF02CBE00000020014901204863704759
:106270000000002001490120086370470000002051
:106280002DE9FC476C4FF86A08B16CA002E0386B4E
:1062900020B173A0BDE8FC4701F0C7BB00F0B4FC1F
:1062A00004460FF0B5FA05460FF0ACFA01462A464F
:1062B00076A001F0A3FB207F04254FF4007900288D
:1062C00024D05D4800231830CDE900504A467CA117
:1062D0007E4810F063F906460FF09AFA80460FF0F8
:1062E00091FA02464346314679A001F087FB012E20
:1062F0000FD0472282A188A001F054FB502080F3E8
:106300001188BFF34F8FBFF36F8FFEE786A001F0B8
:106310008CFB94F82800002824D0474800231C3028
:10632000CDE900504A4687A1894810F037F9064662
:106330000FF06EFA80460FF065FA0246434631468A
:1063400084A001F05BFB012E0FD052226CA172A041
:1063500001F028FB502080F31188BFF34F8FBFF36B
:106360006F8FFEE787A001F060FB94F834000028EF
:1063700024D0314800232030CDE900504A4688A17E
:106380008A4810F00BF906460FF042FA80460FF0EB
:1063900039FA02464346314685A001F02FFB012E13
:1063A0000FD05D2256A15CA001F0FCFA502080F3D2
:1063B0001188BFF34F8FBFF36F8FFEE788A001F006
:1063C00034FB94F84000002824D01B4800232430DC
:1063D000CDE900504A4689A18B4810F0DFF8044609
:1063E0000FF016FA05460FF00DFA02462B4621462D
:1063F00086A001F003FB012C0FD0682240A146A02B
:1064000001F0D0FA502080F31188BFF34F8FBFF313
:106410006F8FFEE789A001F008FB0120F8620FF002
:10642000F7F904460FF0EEF902B02246BDE8F04756
:10643000014689A001F0E2BA000000205B4E4554FD
:106440005D2073746172742D6E6574776F726B2D3D
:106450007461736B7320616C72656164790D0A00FD
:106460005B4E45545D2073746172742D6E65747754
:106470006F726B2D7461736B732073746F702D70FA
:10648000656E64696E670D0A000000005B4E45543E
:106490005D2073746172742D6E6574776F726B2DED
:1064A0007461736B7320656E7465722066726565C6
:1064B0003D256C75206D696E3D256C750D0A0000DB
:1064C0005463705372765331000000006D58000819
:1064D0005B4E45545D206372656174652054637042
:1064E00053727653312072633D256C642066726569
:1064F000653D256C75206D696E3D256C750D0A0036
:106500002E2E2F436F72652F5372632F667265654F
:1065100072746F732E630000636F6E6669672D611E
:1065200073736572740000005B4E45545D20736B9D
:10653000697020546370537276533120656E3D301C
:106540000D0A00005463705372765332000000004D
:10655000735800085B4E45545D2063726561746535
:106560002054637053727653322072633D256C64FD
:1065700020667265653D256C75206D696E3D256CE4
:10658000750D0A005B4E45545D20736B6970205495
:106590006370537276533220656E3D300D0A0000F1
:1065A000546370436C694331000000006158000877
:1065B0005B4E45545D206372656174652054637061
:1065C000436C6943312072633D256C6420667265BB
:1065D000653D256C75206D696E3D256C750D0A0055
:1065E0005B4E45545D20736B697020546370436C3F
:1065F00069433120656E3D300D0A000054637043DD
:106600006C69433200000000675800085B4E455437
:106610005D2063726561746520546370436C6943E7
:10662000322072633D256C6420667265653D256C81
:1066300075206D696E3D256C750D0A005B4E4554E5
:106640005D20736B697020546370436C6943322022
:10665000656E3D300D0A00005B4E45545D2073743D
:106660006172742D6E6574776F726B2D7461736BCC
:1066700073206578697420667265653D256C7520A8
:106680006D696E3D256C750D0A00000010B508B1EE
:10669000012200E0002210210348FDF74FFABDE877
:1066A0001040022000F031B8000801401CB5002065
:1066B00000900190022000F0F8F92C21012000F058
:1066C0008DFAFF217E2000F089FA0321392000F0A5
:1066D00085FA80212D2000F081FA1F21312000F061
:1066E0007DFA684600F0D3F90021532000F076FAD5
:1066F00080211D2000F072FAAD217F2000F06EFA9B
:106700001121052000F06AFA1CBD08B5002808D048
:1067100000EBC000009001E000BF0846411E009160
:10672000FAD208BD10B5012000F0BEF8C0F3801009
:1067300010BD000070B505465FF0000404F11000C4
:10674000C0B200F0B1F82855641CE4B2062CF5D3B1
:1067500070BD10B52A2000F0A7F804462B2000F0E9
:10676000A3F844EA002010BD2C2000F09DB810B51D
:10677000282000F099F80446292000F095F844EA12
:10678000002010BDF0B585B000241B480094019492
:1067900002940394816941F004018161816901F0EF
:1067A00004010491816941F0080181618069134FFE
:1067B00000F008000490012210213846FDF7BEF9D0
:1067C000102001250326CDE90005CDE902466946E2
:1067D0003846FDF7AFF80A4F012202213846FDF78F
:1067E000ADF90220CDE90005CDE9024669463846FB
:1067F000FDF7A0F805B0F0BD001002400008014010
:10680000000C014010B542F21070FFF77EFF00202F
:1068100000F0A0F840F6B830FFF777FF012000F055
:1068200099F8BDE810404CF25030FFF76EBF10B53C
:10683000062100220846FDF74FFABDE81040062069
:10684000FDF73CBAF8B50D46040021D0002D1FDD40
:106850000020FFF71BFF722000F04AF9ADB2642759
:106860000FE0402D01D9402600E02E463346224657
:10687000084909480097FDF7F9FD20B9A81B3444E1
:1068800085B2002DEDD1BDE8F8400120FFF7FEBE36
:10689000F8BD00000E6F0108EC010020702000F030
:1068A00014B8712000F011B810B504460020FFF7AD
:1068B000EDFE204600F01CF9002000F019F9044616
:1068C0000120FFF7E3FE204610BD10B5044600206E
:1068D000FFF7DCFE204600F00BF9002000F008F97D
:1068E00004460120FFF7D2FE204610BD38B50C004B
:1068F000054601D0002020700120FFF7D5FFC0071A
:1069000021D0FFF7CBFFFFF7CCFF00281BD00128D9
:1069100016D104216846FFF795FF14B19DF80100D8
:1069200020709DF80000BDF80240012808D19DF8B4
:106930000100800604D1122C02D3B4F5C06F03D934
:1069400000F050F8002038BD21462846FFF77AFFB6
:10695000201F38BD08B1012200E0002202210148B9
:10696000FDF7ECB8000C0140002803D0007A0028A5
:1069700000D00120704770B504467E20FFF794FFD9
:106980000546ACB125700120FFF78EFF60705320E3
:10699000FFF78AFFA0701D20FFF786FFE070002040
:1069A00020716071A071E0716078C0F38010207276
:1069B00029467E2000F012F9284670BDFFF796BFE9
:1069C00000F02DB810B504460520FFF76DFF34B177
:1069D00040F00101BDE81040052000F0FFB820F0B4
:1069E0000101F7E710B50520FFF75EFF044600F050
:1069F000FE01052000F0F2F80121552000F0EEF82C
:106A00000221012000F0EAF80D217E2000F0E6F8D6
:106A100044F00101BDE81040052000F0DFB870B57A
:106A20000D46002400F0A2F84FF4805605E0641CE7
:106A3000B44202D34FF0FF3070BD0220FFF734FFA5
:106A4000C007F4D1E9B27C2000F0C8F8290A7D2003
:106A500000F0C4F800F002F8002070BD10B502206C
:106A6000FFF722FF40F00101BDE81040022000F0D6
:106A7000B5B870B50546002404F11000295DC0B218
:106A800000F0ACF8641CE4B2062CF5D370BD70B510
:106A90000546002404F11600295DC0B200F09EF8FE
:106AA000641CE4B2082CF5D370BD10B500210C466F
:106AB00020B1012806D002280DD108E04FF48851FA
:106AC000412408E04FF4445140F2011403E04FF434
:106AD000805140F2E114002000F062F821460420C9
:106AE00000F05EF80021BDE810401F2000F076B8ED
:106AF00001B582B000208DF80400642000900123CD
:106B000001AA02A90448FDF7B1FC08B100200EBD9E
:106B10009DF804000EBD0000EC010020084810B5EF
:106B200002210122C0E9041209028161FDF704FC7F
:106B3000002803D0BDE81040FCF73EBB10BD0000AC
:106B4000EC01002010B5084C01E034B1641E0B20AC
:106B5000FFF7AAFEC007F8D110BD00210B2000F0FE
:106B60003DF84FF0FF3010BDA086010070B50D4616
:106B7000060014D0002D12DD0020FFF787FDF8205D
:106B8000FFF7B6FF002403E0305DFFF7B1FF641CA0
:106B9000AC42F9DBBDE870400120FFF777BD70BD66
:106BA00010B50C4640F040010C2000F017F8E1B29F
:106BB0000D2000F013F8210A0E2000F00FF80A2132
:106BC0000B2000F00BF8FFF7BDFF002805D10021D6
:106BD000BDE810400B2000F001B810BD70B50446B0
:106BE0000D460020FFF752FD44F08000FFF780FFC4
:106BF0002846FFF77DFFBDE870400120FFF746BD46
:106C0000582102F05DBA0000004870472CB0002007
:106C100010B5044601F0B6FF002804D102484169CE
:106C20002160008BA08010BD2CB00020022802D370
:106C30004FF4E1307047024901EB8000C06C7047AF
:106C40002CB0002010B502F059FABDE8104000F059
:106C500027B800001CB5C3788278CDE900230C4624
:106C60004378027802A12046F9F7FAFB1CBD000028
:106C700025752E25752E25752E25750038B1012810
:106C800007D0022807D0032807D000207047102023
:106C90007047202070470120704702207047000095
:106CA00010B55C210C4802F033FA78B90A4C0B4954
:106CB000206888420AD1A088032807D12046FFF720
:106CC0009FFFA16D884201D1002010BD00F0CEFCD5
:106CD0004FF0FF3010BD00002CB000205550435441
:106CE0007FB50C46817845790379C2788DE82E000E
:106CF0004378027802A12046F9F7B2FB7FBD00007D
:106D0000253032583A253032583A253032583A2513
:106D10003032583A253032583A2530325800000087
:106D200010B50146046800E0641C20782028FBD0E0
:106D30000928F9D010F0FF0F4FF0000201D02046D3
:106D400003E000200A6010BD401C03782BB12C2BFF
:106D5000FAD100F8012B086000E00A6020460DF02F
:106D60000DFB204610BD00002DE9F0478A46D4B047
:106D7000914601469F2213A8F9F73BFF00268DF8A4
:106D8000EB6013A80DF0FAFA13A807F031FE0178B2
:106D9000412901D061297DD14178542901D074293C
:106DA000F9D1817811B12B29F5D101E0E9A221E0D7
:106DB000C01C0746E9A100F0B1FE20B9E8A13846A1
:106DC00000F0ACFE30B14946504602F041FA54B0F2
:106DD000BDE8F087E4A1384600F0A0FE78B100F0ED
:106DE00031FC30B1E2A249465046F9F74FFB04208E
:106DF000EDE7E5A249465046F9F748FBD6E2E9A19E
:106E0000384600F08BFE012418B1E8480470E8A26F
:106E1000F0E7ECA1384600F081FE18B100F026FC46
:106E2000EAA2E7E7EFA1384600F078FEEF4D30B177
:106E3000AB79EFA249465046F9F728FBB6E2F0A13C
:106E4000384600F06BFE40B1286D0090EEA2494636
:106E50005046EB6CF9F71AFBA8E253AAF1A13846A9
:106E600005F0AEFD90B32F2268465399F9F7C1FEA5
:106E70008DF82F60CDF838D00EA8FFF751FF30B352
:106E80000746EAA100F04AFE30B9E9A1384600F011
:106E900045FE00E059E108B1344609E0E6A1384674
:106EA00000F03CFE20B9E5A1384600F037FE70B195
:106EB0000EA8FFF735FF38B10CAB4FF461224FF449
:106EC000966105F0AAFD20B1DEA286E206E0E4A20A
:106ED00083E205EB84010C98C864B4E253AAE6A1EE
:106EE000384605F06DFD58B16B46012200215398DC
:106EF00005F093FD08B1E1A26FE20098A871A2E24B
:106F0000E4A1384600F00AFE08B3B84803A90830E7
:106F1000FFF7A0FEB5480CA90C30FFF79BFEB34865
:106F20003BA91030FFF796FE10A8FFF771FE07A9E6
:106F300010A8FFF7D5FE07AA3BA90CA88DE807000B
:106F400003ABD6A249465046F9F7A0FA2EE253AA5F
:106F5000DCA1384605F034FD00283CD05F223BA878
:106F60005399F9F746FE3BA805908DF84B6105A8AB
:106F7000FFF7D6FE18B103A900F000FC08B1D2A2B9
:106F80002BE205A8FFF7CCFE18B104A900F0F6FB30
:106F900008B1D4A221E205A8FFF7C2FE18B106A9E4
:106FA00000F0ECFB08B1D7A217E205A8FFF7B8FE86
:106FB00018B101A900F016FC08B1DAA20DE203989D
:106FC000A8600498E8600698286101986861BDF897
:106FD0000800288337E2DAA1384600F09FFDE8B3C5
:106FE00000243BAE04EB440005EB800006EB0411EB
:106FF0002030FFF72FFE641C042CF3D395F84100DA
:107000001C3502F0B5FD0746687E02F0B1FD04466E
:10701000687B02F0ADFD8046687802F0A9FD01466C
:10702000A88DEB8C47AACDE910200F9312972A8CDC
:1070300095F8240043ABCDE90B32CDE90D406A8BC6
:107040002B7EAC8ACDE90932CDE907483FA8EA8911
:107050002B7BCDE90520CDE9031300E00BE0288967
:1070600069880091CDE901602B78B74A49465046BE
:10707000F9F70CFA9AE153AAB4A1384605F0A0FC3E
:10708000002862D05F223BA85399F9F7B2FD3BA8D4
:1070900009908DF84B6109A8FFF742FEA0B307469F
:1070A000ACA100F03BFD08B1002713E0AAA13846CF
:1070B00000F034FD08B101270CE0A8A1384600F02B
:1070C0002DFD08B1022705E0A5A1384600F026FDF8
:1070D000D0B1032709A8FFF723FEC0B106AB0122F8
:1070E000002105F09AFC00287FF405AF09A8FFF7FE
:1070F00017FE38B14FF6FF7807AB4246012105F085
:107100008CFC08B397A268E1FFE79CA265E107EB5E
:10711000470005EB800404F120000AA9FFF79AFD5F
:10712000607F02F025FD8FB1012F10D0022F0FD00C
:10713000032F0ED099A3A18CE28BCDE903100AADE9
:10714000CDE90125207F2BE13EE184E130E132E110
:1071500034E136E14F4B0D0A000000003F00000013
:10716000515545525900000053415645000000005A
:107170004552524F523A2053617665206661696CE0
:1071800065640D0A000000004F4B3A20436F6E66A5
:10719000696775726174696F6E2073617665640DDD
:1071A0000A0000005245534554000000B801002079
:1071B0004F4B3A20526573657474696E672E2E2E9C
:1071C0000D0A000044454641554C54004F4B3A20AF
:1071D00044656661756C747320726573746F726553
:1071E000640D0A004D55583F000000002CB00020EF
:1071F0002B4D55583A25750D0A4F4B0D0A000000CE
:10720000424155443F0000002B424155443A55301D
:107210003D256C752C55313D256C750D0A4F4B0D78
:107220000A000000424155440000000055300000B3
:10723000554152543200000055310000554152541E
:10724000330000004552524F523A20496E76616C2D
:1072500069642062617564726174650D0A000000E2
:107260004552524F523A20496E76616C69642055FE
:107270004152540D0A0000004D5558004552524FDE
:10728000523A20496E76616C69642076616C75654E
:107290000D0A00004E45543F000000002B4E45549F
:1072A0003A49503D25732C4D41534B3D25732C4796
:1072B000573D25732C4D41433D25730D0A4F4B0D12
:1072C0000A0000004E4554004552524F523A2049A0
:1072D0006E76616C696420495020666F726D6174CE
:1072E0000D0A00004552524F523A20496E76616CA9
:1072F0006964206D61736B20666F726D61740D0A35
:10730000000000004552524F523A20496E76616C9F
:107310006964206761746577617920666F726D6159
:10732000740D0A004552524F523A20496E76616CF4
:107330006964204D414320666F726D61740D0A00CF
:107340004C494E4B3F000000C87401084C494E4B5D
:1073500000000000533100005332000043310000B0
:10736000433200004552524F523A20496E76616CCA
:10737000696420706F72740D0A0000004552524F0C
:10738000523A20496E76616C696420726F7574653B
:10739000206669656C640D0A000000003F00000073
:1073A000009030A249465046F9F770F800200EE5EB
:1073B000AFF26003BFE6AFF26003BCE6AFF2640376
:1073C000B9E6AFF26403B6E609A8FFF7A9FC18B165
:1073D00005A900F0D3F930B130A249465046F9F77B
:1073E00055F80220F3E409A8FFF79AFC00283FF4BF
:1073F00089AE08AB4246002105F00FFB00287FF460
:1074000081AE09A8FFF78CFC00283FF47EAE8046D1
:10741000AFF2E81100F082FB08B1344606E0AFF2AB
:10742000E811404600F07AFB0028EED007EB470059
:1074300005EB8000069901770799C18305990162E0
:10744000089981844477AFF2F42249465046F9F70F
:107450001DF80520BBE41AA249465046F9F716F874
:107460000320B4E42B4C494E4B3A25732C454E3D3A
:1074700025752C4C504F52543D25752C5249503D8A
:1074800025732C52504F52543D25752C5541525462
:107490003D25730D0A4F4B0D0A0000004552524F17
:1074A000523A20496E76616C69642072656D6F7422
:1074B0006520495020666F726D61740D0A000000EE
:1074C0004552524F523A20556E6B6E6F776E206365
:1074D0006F6D6D616E640D0A0000000010B500282C
:1074E00010D009494C6889780268A2420AD0046029
:1074F000084607F0AFF922460146BDE8104003A058
:1075000000F07CBA10BD0000B80100205B43464784
:107510005D2072782D726F7574652D6661696C20BF
:1075200072633D257320636E743D256C750D0A00F2
:10753000F0B504460079ADF5077D0E46002778B317
:107540002078042801D0082827D1C0B2082841D0CB
:107550005FF00005ADF814720846F9F795FA83B2AA
:1075600040F2062285A903A88DE80700207832465C
:1075700000210CF019FF78B3BDF8142203A92846A6
:107580000DF01CFA002808D00DF06AFA0246BDF88A
:107590001432294615A000F031FA0DF5077DF0BD33
:1075A000FFE71C4C012060701B4D2868C16821F06A
:1075B0001001C1603046F9F767FA82B2C82331463C
:1075C0002846FDF741FB2868C16841F01001C16001
:1075D0006770E2E70125BDE7FFE73046F9F754FAA7
:1075E000024621780DA000F009FAD6E75B43464732
:1075F0005D20726573702D74782D6661696C2063EF
:10760000683D25752072633D2573206C656E3D25B0
:10761000750D0A00B8010020440200205B43464774
:107620005D20726573702D656E632D6661696C20D7
:107630007372633D307825303258206C656E3D257D
:10764000750D0A0010B5084C064820600320A08084
:107650002046FFF7D5FAA0652046BDE810405C2122
:1076600001F068BD555043542CB000202DE9FC4179
:1076700015A04FF00008056814A05C21066814A04E
:1076800007681448CDF80480F9F78CFA114C1248B9
:1076900020600320A08004F1080084F8068080E8C0
:1076A000E001BDF80400208307F050F94FF4E13009
:1076B000E064206540F6B83060652046FFF7A0FA28
:1076C000A065BDE8FC810000C0A81F64FFFFFF00AB
:1076D000C0A81F012CB000205550435410B50EA077
:1076E00000F0A3F912480068C16841F01001C160C0
:1076F000A02210490E48FDF797FA38B10EA000F00D
:1077000094F9BDE8104012A0FBF728BDBDE8104079
:1077100014A000F08AB900005B4346475D207278F0
:107720002D737461727420656E7465720D0A0000A9
:107730004402002088B000205B4346475D207278F9
:107740002D7374617274206661696C0D0A0000000B
:107750006366672D72782D73746172742D6661692A
:107760006C0000005B4346475D2072782D737461A6
:10777000727420657869740D0A00000010B586B037
:107780000C4604AA03A9CDE9001202AB05AA12A176
:10779000F9F732F801464FF0FF30042919D1059965
:1077A000FF2916D8029A002A13DBFF2A11DC039A5C
:1077B000002A0EDBFF2A0CDC049A002A09DBFF2AD0
:1077C00007DC2170029860700398A0700498E07044
:1077D000002006B010BD000025642E25642E25640F
:1077E0002E2564002DE9F04F8BB00DF1240808AF71
:1077F00007AE06AD8DE8E00104AC8946834622461B
:1078000011A1231DF8F7F8FF4FF0FF3A062809D021
:107810008DE8E001231D04AA10A15846F8F7ECFFFB
:10782000062805D15FF0000054F82010FF2903D985
:1078300050460BB0BDE8F08F09F80010401C062838
:10784000F2DB0020F5E7000025783A25783A257824
:107850003A25783A25783A257800000025782D25B4
:10786000782D25782D25782D25782D257800000078
:107870007FB51E4DE86B006840681D4C80B2C0F1BA
:10788000A00081B200200390607800282CD189B13B
:107890001848006870B1184BCDE9003103AA0023E5
:1078A00002921A46194606F0A1FF18B1A07060684E
:1078B000401C60600D48FCF7D2FE104E4FF0805423
:1078C00050B9A0220C490948FDF7AEF920B128684B
:1078D000C16821F01001C1600398002804D0346011
:1078E000BFF34F8FBFF36F8F7FBD000044020020B6
:1078F000B80100200400002088B0002004ED00E062
:10790000012801D0042070470820704730B50B4B88
:107910000B4C002108460022C50702D083EA500024
:1079200000E04008521C082AF6D344F82100491C04
:10793000FF29EFD903490120087030BD2083B8ED3D
:10794000C8B30020C001002070B5060016D0307802
:10795000002813D03046F9F797F8094C05462068FF
:10796000401C20602A4631460020FDF71DFEA8423B
:1079700004D26068401C60602068A06070BD000098
:107980005C00002000B902A0014603A000F036B858
:10799000286E756C6C2900005B424F4F545D2025AA
:1079A000730D0A00F0B585B017460C4605460DF07C
:1079B0002FFF06460DF026FF01460B4882684368FC
:1079C0000068CDE90203CDE9001604920CB122460D
:1079D00000E006A20DB1294600E004A13B4605489F
:1079E00000F00CF805B0F0BD5C000020286E756C4E
:1079F0006C290000D0710108FDF7D4BD0FB400B5AB
:107A0000C1B0429A002A0DD043AB4FF48071684652
:107A1000F8F700FD0021002804DB8DF8FF10684610
:107A2000FFF792FF41B05DF814FB002801D0FFF78B
:107A30008BBF704770B505460C46880705D04FF4DC
:107A4000B67207A10EA003F0E1F907F010F8E9689B
:107A500009682160E9680C60BDE8704007F029B84A
:107A60002E2E5C447269766572735C4C7749505C6B
:107A70007372635C636F72655C6D656D702E63001D
:107A80006D656D705F667265653A206D656D20701D
:107A9000726F7065726C7920616C69676E656400E5
:107AA00070B5044606F0E3FF0546E068046874B16B
:107AB00021680160A00705D04FF48C7206A10EA0CA
:107AC00003F0A4F9284606F0F4FF204670BD2846CE
:107AD00006F0EFFF002070BD2E2E5C4472697665C3
:107AE00072735C4C7749505C7372635C636F726550
:107AF0005C6D656D702E63006D656D705F6D616CA2
:107B00006C6F633A206D656D702070726F70657276
:107B10006C7920616C69676E6564000010B50FE0D8
:107B2000A3F16104401C491C192C01D8203BDBB295
:107B3000A2F16104192C01D8203AD2B2934207D1A4
:107B400003781BB10A78002AEAD101E0087808B16D
:107B5000002010BD012010BD2DE9F0410F460400AA
:107B600005D140F2BB123DA145A003F04FF906F04C
:107B70007EFF00266660277294F8201041F0010114
:107B800084F820106578667006F093FFA36A7BB1D5
:107B90000022042120469847A36A4BB100221146D7
:107BA00020469847A36A1BB100220221204698472D
:107BB000384603F007F8804614F10C0F06D0E06851
:107BC00020B1414604F10C0006F0BBFF14F1100F88
:107BD00006D0206920B1414604F1100006F0B1FF43
:107BE000012D0ED0042D0CD0032D0AD0606A002880
:107BF00031D0BDE8F0414FF4FD7218A124A003F08C
:107C000005B994F82000C0F3800100F0FB0084F86F
:107C1000200000291FD1606A28B940F2E9120FA1A3
:107C200022A003F0F3F8606A042D06D00771606AA1
:107C3000456A25B1286810B107E00671F7E74FF4EF
:107C4000F97206A120A003F0E1F828466662BDE8BB
:107C5000F04106F0B0BFBDE8F08100002E2E5C447C
:107C60007269766572735C4C7749505C7372635CC1
:107C70006170695C6170695F6D73672E63000000FD
:107C8000636F6E6E20213D204E554C4C000000006D
:107C9000636F6E6E2D3E63757272656E745F6D7389
:107CA00067203D3D204E554C4C000000636F6E6ECA
:107CB0002D3E63757272656E745F6D736720213D32
:107CC000204E554C4C000000696E76616C69642052
:107CD0006F705F636F6D706C657465645F73656D05
:107CE000000000002DE9F74F84B04FF00A0B00248C
:107CF0000646DA465F46D94602940194CDF8004024
:107D00004F4804EB440100EBC108039198F814506C
:107D10000A2F1CD0002D2BD0012D07D0022D05D20B
:107D20004FF4927247A151A003F070F89EB13168F0
:107D3000D8F8040081420ED1069820B1D8F8081076
:107D40000698814207D1204607B0BDE8F08F002D8C
:107D5000E2D127460CE0012D18D0022D08D3052DC5
:107D600006D2B8F812000099884201D3A2460090CA
:107D7000641C24B20A2CC3DB059881074FF0FF3046
:107D8000E2D40A2F16D018DA3C463CE02C4803997E
:107D900050F831000028B8F8120005D00299884246
:107DA000E6D3A1460290E3E701998842E0D3A346D7
:107DB0000190DDE70599C907C6D05146BAF10A0F0F
:107DC0000DDA0C461E4801EB440150F8310078B141
:107DD0004FF4B7721BA135A003F018F808E059461C
:107DE000BBF10A0F03DB4946B9F10A0FACDA0C46C6
:107DF0000A2C05DB4FF4C07212A132A003F006F882
:107E0000204600F07FF80A2C05DB4FF4C2720DA16A
:107E10002CA002F0FBFF0A4804EB440100EBC10573
:107E2000287D28B140F2851206A12BA002F0EEFFBA
:107E30000EB130686860002068820698A86082E70A
:107E4000989A00202E2E5C447269766572735C4CA1
:107E50007749505C7372635C636F72655C697076BE
:107E6000345C6574686172702E63000073746174B1
:107E700065203D3D204554484152505F5354415484
:107E8000455F50454E44494E47207C7C20737461C9
:107E90007465203E3D204554484152505F53544143
:107EA00054455F535441424C450000006172705F7D
:107EB0007461626C655B695D2E71203D3D204E559D
:107EC0004C4C000069203C204152505F5441424CD0
:107ED000455F53495A4500006172705F7461626C7E
:107EE000655B695D2E7374617465203D3D2045546A
:107EF000484152505F53544154455F454D50545989
:107F00000000000070B50B4D00EB4006002455F852
:107F1000360018B101F05CF945F8364005EBC600B3
:107F2000054904754482846044600A68C260898897
:107F3000018270BD989A00209D7001082DE9F047DC
:107F400086B00D0080460AD0D8F804404FF48079FE
:107F50002088484540D1207906283DD105E020A061
:107F6000F8F772FA06B0BDE8F0876079042833D1DB
:107F70006088082830D1D4F80E100491A26968688E
:107F800018B1824204D1012603E00026374608E0FA
:107F90000026814201D1012700E000270EB1012314
:107FA00000E0022304F10802924604A9284600F0EA
:107FB0002BFBE08848450FD176B16FB9022204ABA4
:107FC000CDE90232291DCDE9001A05F12603194633
:107FD0005246284600F036FA404605F0DDF8C1E783
:107FE0006E6574696620213D204E554C4C000000A2
:107FF000FEB515460E46040005D140F21F3241A1E0
:108000004AA002F003FF2EB94FF448723DA14BA0E5
:1080100002F0FCFE2DB940F221323AA14AA002F052
:10802000F5FE2146286801F068FB08B14A4B3FE0A5
:108030002868C0F303110E2925D0A168636800EAFF
:1080400001020B409A4208D080B2A0F57E41A939C6
:1080500003D0E068B0B304F10C05404B40481A78F7
:1080600002EB420100EBC1010F7D022F2ED38F687E
:10807000A7422BD12F6849688F4227D1314620462D
:1080800000F070F8FEBD01208DF8040000208DF88E
:1080900005005E208DF80600687801AB00F07F00D7
:1080A0008DF80700A8788DF80800E8788DF80900A9
:1080B0004FF40060009004F126023146204600F0A3
:1080C00099FBFEBDFFE76FF00300FAE75FF00002E7
:1080D00002EB420100EBC1010F7D022F08D38F6834
:1080E000A74205D12F6849688F4201D11A70C5E7B0
:1080F000521CD2B20A2AEBD332462946204600F05F
:108100009BF8DEE72E2E5C447269766572735C4CD8
:108110007749505C7372635C636F72655C697076FB
:10812000345C6574686172702E6300006E657469FA
:108130006620213D204E554C4C0000007120213D11
:10814000204E554C4C00000069706164647220211F
:108150003D204E554C4C00009770010894010020C2
:10816000989A00202DE9F8430646154688461B4894
:1081700002EB450100EBC104207D022805D240F24C
:10818000EF2217A120A002F041FE144A05EB4501A1
:10819000207D02EBC1050C35022813D1608A03272C
:1081A000B0F58E7F04D9211D304600F0E5F907E0D7
:1081B000B0F5877F06D32A46211D304600F0E2F94C
:1081C00000B927754FF4006000902B4606F1260297
:1081D0004146304600F00EFBBDE8F883989A002037
:1081E0002E2E5C447269766572735C4C7749505CE4
:1081F0007372635C636F72655C697076345C65741E
:10820000686172702E6300006172705F7461626CED
:10821000655B6172705F6964785D2E73746174650B
:10822000203E3D204554484152505F5354415445EF
:108230005F535441424C45002DE9F74F82B08946C7
:1082400002984FF0FF3B26300190086814465E46C6
:108250004FF00008029901F050FAA0B9D9F80000D7
:10826000C0F303110E290ED0B9F1000F0BD050B19D
:1082700001214846029AFFF735FD050006D540B2B8
:1082800005B0BDE8F08F6FF00F00F9E77F2D05D343
:1082900040F2C2324AA154A002F0B8FD05F0FF0A34
:1082A00055480AEB4A0700EBC705287D68B101284D
:1082B00007D0022805D240F2CE3241A14FA002F0F1
:1082C000A5FDB8F1000F08D106E04FF0010885F8D0
:1082D00014800298A86000E07CB94946029800F03A
:1082E0004BF9060007D1287D012804D1B8F1000F11
:1082F00001D100206882002C5FD0287D3E490228F1
:108300000ED348494FF4006005F10C0381F800A03A
:108310000090DDE90120214600F06CFA06464CE0B1
:108320008846012849D1254640F2FA3668892989CC
:10833000884206D1286820B1324621A13AA002F035
:1083400065FD287B400607D522464FF420710E209C
:1083500004F07CFD044605E02D68002DE6D12046A2
:1083600005F030F844B3072003F062F908B30021A8
:10837000C0E9001458F837104246B9B1012301E0B2
:1083800021465B1C0C68002CFAD10860032B0BD330
:1083900052F83740206848F83700606804F0FCFE67
:1083A0002146072003F000F9002606E048F83700D0
:1083B000FAE7204604F0F0FE5E46304660E7000033
:1083C0002E2E5C447269766572735C4C7749505C02
:1083D0007372635C636F72655C697076345C65743C
:1083E000686172702E63000074797065206F766525
:1083F00072666C6F77000000989A00206172705F5F
:108400007461626C655B695D2E7374617465203D97
:108410003D2050454E44494E47206F7220535441F1
:10842000424C4500940100206E6F207061636B65C3
:10843000742071756575657320616C6C6F77656408
:10844000210000002DE9FF4F81B09846DDE90FA91A
:10845000DDF838B006004FF0000705D14FF48C620C
:1084600029A133A002F0D2FC4FF420721C210E206F
:1084700004F034FB050044D068891C2805D240F282
:108480006B4221A12EA002F0C1FC6C68119801F092
:10849000C7FCE08096F82C00062805D040F2724216
:1084A00019A1344802F0B2FCD8F80010A160B8F865
:1084B0000400A081DAF80010C4F81210BAF8040021
:1084C000E082DBF80000C4F80E00D9F80000A061DB
:1084D0004FF48070208008206080062020710420E6
:1084E000607140F60600DDE902230090294630461F
:1084F00000F080F9284604F04FFE384605B0BDE88C
:10850000F08F4FF0FF30F9E72E2E5C4472697665EC
:1085100072735C4C7749505C7372635C636F726515
:108520005C697076345C6574686172702E630000FB
:108530006E6574696620213D204E554C4C0000004C
:10854000636865636B207468617420666972737414
:1085500020706275662063616E20686F6C642073A2
:108560007472756374206574686172705F68647298
:108570000000000040740108014A00F003B8000048
:10858000977001087FB5064D031D0124CDE9003524
:10859000CDE9021422331946FFF754FF04B070BD31
:1085A0009D70010870B5174D002400BF04EB440016
:1085B00005EBC002117D01B305291ED0508A401C75
:1085C00080B25082B0F5967F0AD2012906D00329E5
:1085D0000AD004290AD001290BD00EE0052808D3BF
:1085E0002046FFF78FFC08E0042000E00220107511
:1085F00003E0111D9068FFF7BFFF641C0A2CD5DB58
:1086000070BD0000989A00202DE9F84F054690F8BB
:108610002C001E4691460C46062805D04FF4D57214
:108620002EA138A002F0F2FBA4B1206890B1294637
:1086300001F063F870B92078C0F303100E2809D058
:108640002A4631462046FFF74DFB002805DA40B2A6
:10865000BDE8F88F6FF00F00FAE7334C710706D5CD
:1086600000EB400204EBC2020521117508E000EBAB
:10867000400104EBC1010A7D052A13D002220A75CC
:1086800000EB400604EBC6004FF400688560D9F8A3
:108690000020C260B9F8041001820021418205F176
:1086A000260A14E06FF00500D2E7086844F83600A7
:1086B00007204F6802F078FF4B465246394628465D
:1086C000CDF8008000F096F8384604F065FD54F8C7
:1086D00036100029E9D10020BAE700002E2E5C44B4
:1086E0007269766572735C4C7749505C7372635C37
:1086F000636F72655C697076345C65746861727012
:108700002E6300006E657469662D3E68776164644F
:10871000725F6C656E203D3D204554485F4857416F
:108720004444525F4C454E00989A002070B50C4668
:10873000050004D146221EA127A002F067FB24B940
:1087400047221BA127A002F061FB68890E2803D2F3
:10875000284604F021FD18E06868808901F060FB7C
:10876000B0F5006F13D0A0F500600638F0D194F892
:108770002D000007ECD50E21284604F053FE0028FA
:10878000E6D121462846FFF7D9FB002070BD94F8BA
:108790002D0010F0180FDBD00E21284604F042FE09
:1087A0000028D5D121462846BDE8704000F0BCBF66
:1087B0002E2E5C447269766572735C4C7749505C0E
:1087C0007372635C6E657469665C65746865726E0D
:1087D00065742E63000000007020213D204E554C32
:1087E0004C0000006E6574696620213D204E554C9A
:1087F0004C0000002DE9F0471E46DDF8209017469A
:108800000D465FEA000804D129221FA128A002F02A
:10881000FDFA25B92A221CA129A002F0F7FA27B9EE
:108820002B2219A129A002F0F1FA26B92C2216A1B7
:1088300029A002F0EBFA4FF420720E21002004F080
:108840004DF904001CD0294604F0EEFA6568306842
:108850002860B088A8803868C5F80600B8886881A4
:10886000484601F0DDFAA881D8F818204046214694
:1088700090470546204604F08FFC2846BDE8F08767
:108880004FF0FF30FAE700002E2E5C4472697665E7
:1088900072735C4C7749505C7372635C6E6574698B
:1088A000665C65746865726E65742E630000000016
:1088B0006E6574696620213D204E554C4C000000C9
:1088C0007020213D204E554C4C00000073726320F7
:1088D000213D204E554C4C0064737420213D204EA8
:1088E000554C4C0010B586B004000DD00021605CE2
:1088F00038B12046FEF7BDF8204600F069FB06B00F
:1089000010BD491C0629F2D303A8FDF713FF03A8E5
:1089100000F05EFB9DF80F009DF811209DF81010EF
:108920008DE807009DF80E309DF80D209DF80C1085
:1089300001A0FFF763F8E2E75B4554485D207573DB
:108940006520696E7465726E616C206D61633D2592
:108950003032583A253032583A253032583A25309C
:1089600032583A253032583A253032580D0A000034
:1089700070B543B1184C1D6844F83E5F9B88A380D6
:10898000164C0023237068B161B15AB113460A46F0
:1089900001461148183003F0CFFF010002D010A0AB
:1089A000FFF72CF80C4800221549183003F0B6FFE9
:1089B000010002D013A0FFF721F8074800221A494E
:1089C000183003F0ABFF010004D0BDE8704017A0E1
:1089D000FFF714B870BD0000889B0020A80100209C
:1089E0005B4554485D207365742D61646472206634
:1089F00061696C206572723D25640D0A00000000FB
:108A0000D1C700085B4554485D20726573796E6379
:108A10002D64656661756C74206661696C20657291
:108A2000723D25640D0A000061C800085B4554488A
:108A30005D20726573796E632D7570206661696C57
:108A4000206572723D25640D0A00000070B5094C66
:108A5000606818B14FF0FF310DF0F8FBFDF779FEBB
:108A60000546606820B100231A4619460DF0D4F877
:108A7000284670BDA801002070B5094C606818B187
:108A80004FF0FF310DF0E2FBFDF76EFE054660682A
:108A900020B100231A4619460DF0BEF8284670BDD5
:108AA000A801002070B5094C606818B14FF0FF3183
:108AB0000DF0CCFBFDF75BFE0546606820B100239E
:108AC0001A4619460DF0A8F8284670BDA8010020E6
:108AD00070B50B4C606818B14FF0FF310DF0B6FB6C
:108AE000FDF720FEC5B2606820B100231A46194682
:108AF0000DF092F82846BDE8704000F075BA00000D
:108B0000A801002010B50CF0A9F9034900208870D5
:108B1000BDE810400CF0D2B9889B00202DE9FC4143
:108B2000074600201C4615460E468DF80400FFF748
:108B3000E9FF01A8009023462A463146384600F056
:108B400089F8054800F059F901469DF8042003A072
:108B5000FEF754FFBDE8FC819C9B00205B45544818
:108B60005D207265632066756C6C206E3D256C75AA
:108B7000206C696E6B3D25750D0A0000002000F029
:108B800033BA000040B105494A782AB18A680260C8
:108B9000898981800120704700207047A80100204A
:108BA0002DE9F041040005D140F2F92212A11CA0E8
:108BB00002F02CF9042002F01BFB05004FF0FF37F8
:108BC00017D000262E601AA0C4E90750652084F84B
:108BD0002E006E2084F82F00184860611848A061AC
:108BE000204600F0CFFF002804D0284602F0F0F91C
:108BF000E6613846BDE8F0812E2E5C4472697665E8
:108C000072735C4C7749505C7372635C6E65746917
:108C1000665C65746865726E657469662E630000D3
:108C20006E6574696620213D204E554C4C00000055
:108C3000746370327561727400000000F17F000887
:108C4000059D0008024890F82D00C0F38000704791
:108C5000A09B00202DE9F0471D4C8146089E6068CE
:108C60001F461546884618B14FF0FF310DF0EEFA59
:108C7000FDF754FFFDF7C6FDFDF718FD3846FFF779
:108C800031FE0220FDF711FF0120FDF79BFE114888
:108C900000F098F8607810B10D4B083300E0002325
:108CA0002A4641464846FFF763FEFDF73BFDC5B245
:108CB000606820B100231A4619460CF0ADFFFDF79D
:108CC000B6FD06B135702846BDE8F04700F08CB916
:108CD000A8010020A09B0020FEB5314D0424686847
:108CE00010B1611F0DF0B2FA0020009001900290C7
:108CF0006846FDF740FE686820B100231A46194611
:108D00000CF08AFF9DF8000010F00C0F15D0254ED6
:108D100001270CF0A3F8B56830466D1CB5600178EA
:108D2000012900D207700CF0C9F8284600F048F974
:108D300018B129461CA0FEF761FE00F069F8022870
:108D400009D09DF80000800605D56846FDF70CFEA9
:108D5000C0B200F049F9134E18361248183000F02E
:108D600083FF050017D00F4932691831904710B1C1
:108D7000284604F011FA641E14F0FF04EDD100F04F
:108D800047F800BF0E494FF080500860BFF34F8F87
:108D9000BFF36F8FFEBD00F03BF8002CF2D0FEBD9C
:108DA000A8010020889B00205B4554485D20727814
:108DB000206F7666206E3D256C750D0A0000000060
:108DC00004ED00E070B5040016D0062084F82C00F5
:108DD00004F126000546FDF7ADFC284600F0F8F842
:108DE00040F2DC50A0841A2084F82D00E0690028AD
:108DF00002D000210180817070BD70B505460CF075
:108E00002DF82C68641C2C600CF058F8204670BDBE
:108E1000F0B585B000278DF804700CF01FF8584E9F
:108E2000707860BB357855B33770012070700CF0E6
:108E300045F835B3022D26D0524C606810B1791E2A
:108E40000DF004FAFDF7CEFD606820B100231A464C
:108E500019460CF0E1FE4A481030FFF7CEFF0446F9
:108E600000F0AEF818B1214647A0FEF7C7FD0BF0A1
:108E7000F5FF77700CF022F8284605B0F0BD0CF035
:108E80001DF80020F9E7FDF7BFFE0189044648BA46
:108E9000A27A000440EA0223E07A91FA91FC4FEAB8
:108EA0000C4C03434CEA022C1B061FFA8CFC43EAD1
:108EB0000C2391FA91FC49BA09040CF0FF0C41EA29
:108EC000022143EA0C23014343EA11600290A18985
:108ED000A27B48BA000440EA0223E07B91FA91FCAD
:108EE0004FEA0C4C03434CEA022C1B061FFA8CFC85
:108EF00043EA0C2391FA91FC49BA09040CF0FF0CE7
:108F000041EA022143EA0C23014343EA1160039042
:108F1000218AA27C48BA000440EA0223E07C91FA4C
:108F200091FC4FEA0C4C03434CEA022C1B061FFA3F
:108F30008CFC43EA0C2391FA91FC49BA09040CF029
:108F4000FF0C41EA022143EA0C23014343EA11608A
:108F50000490FFF7D7FD01A8009004F1140304AAC0
:108F600003A902A8FFF776FE05481430FFF745FF76
:108F700001469DF804200AA0FEF740FD77E70000B7
:108F8000889B0020A80100205B4554485D20726545
:108F900063207278206E3D256C750D0A000000007C
:108FA0005B4554485D207265632066756C6C206E6D
:108FB0003D256C75206C696E6B3D25750D0A0000B2
:108FC000032803D9800601D0002070470120704794
:108FD000044920B102688A60808888810120487035
:108FE00070470000A8010020F0B5064689B0264869
:108FF00005F0B5FD254C264D94F82D00C0F38007F3
:109000004FEA4070AEB100280EDB204603F006FCAC
:10901000287848B994F82D00C00705D0211D2046B6
:10902000FFF7AAFA01202870174805F0A9FD0120D2
:109030000AE0002804DA154803F0D0FB002028706D
:10904000114805F09DFD0020B8421BD094F828007F
:1090500004AD94F82B3094F82A2094F8291085E870
:109060000F00A07994F8273094F82620E1798DE854
:109070000F00637922790EB106A100E006A108482D
:10908000FEF7BCFC09B0F0BDA4010020A09B0020AD
:10909000A801002075700000646F776E000000006A
:1090A0008474010800B585B0002102900120009170
:1090B000039004A96846FAF78BFB05B000BD0000D9
:1090C00070B505460B480E464FF0FF34007808B9DE
:1090D000FEF71CFC0022084807E0A95C6140C9B209
:1090E000521C50F8211081EA1424B242F5D3E04317
:1090F00070BD0000C0010020C8B30020034810B5B7
:10910000007808B9FEF702FC002010BDC001002065
:1091100010B54FF0FF3218B111B1B1F5806F01D920
:10912000104610BD0A460249F7F7CDFC002010BDDD
:1091300000FC05082DE9F0470F4606004FF0FF3808
:1091400032D08FB3B7F5806F2ED8FAF7DFFB58BB5C
:10915000174C2046FFF7A6FF18B100BFFAF78CFBAB
:1091600022E0A1462546002413E0305D611CB9428F
:1091700004D23119497840EA012201E040F47F42EB
:10918000294600230120FAF781FB0028E6D1A41C20
:10919000AD1CBC42E9D3FAF76FFB3A46314648466C
:1091A000F7F746FC002800D04046BDE8F0870000F5
:1091B00000FC05088A68002A01DCF8F767BF521E28
:1091C0008A604A68C0B2531C4B6010707047000040
:1091D00070B5040006D1BDE8704097220BA115A020
:1091E00001F014BE2546D5E9004020B99B2207A115
:1091F00013A001F00BFE686803F0CEFF294607209C
:1092000002F0D2F9002CEDD170BD00002E2E5C448E
:109210007269766572735C4C7749505C7372635CFB
:10922000636F72655C697076345C657468617270D6
:109230002E6300007120213D204E554C4C00000053
:10924000722D3E7020213D204E554C4C00000000F8
:109250002DE9F047BEB0894682462FA93848FDF770
:10926000F9FC374833A9001DFDF7F4FC344837A951
:109270000830FDF7EFFC3BA8FDF7CAFC2AA93BA884
:10928000FDF72EFD2E4C00251AAE083C05EB4500DF
:1092900004EB800006EB05112030FDF7DBFC6D1CB4
:1092A000042DF3D394F84100183400F061FC80469B
:1092B000607F00F05DFC0746607C00F059FC0546CD
:1092C000607900F055FCD4E90D2314F812CCCDE9F7
:1092D0001823CDE9168C218EB4F82AC094F82830D2
:1092E00026AACDE91421CDE9123CA18CE38B0E9383
:1092F00022AA1197CDE90F21217F228B1EABCDE948
:109300000C51CDE90A32628A217CA38907AD06930C
:1093100085E80700E08821790596CDE9031033A997
:1093200000912AAA37A8CDE901022FAB054A494688
:109330005046F7F7ABF83EB00020BDE8F0870000DC
:1093400034B00020947501080A46032100F0E8B803
:109350002DE9FE4F8A464D4904468E683078000755
:10936000850E142D4ED360890428FBD360680078E5
:10937000002847D0082845D1486901F11409C0F3F5
:1093800003120E2A7DD08846096800F0B6F900283D
:1093900077D12089082874D3204600F03FF90028AF
:1093A0006FD105F10E010F46204603F054FB002853
:1093B0002ED02089411989B2884262D84FF4207298
:1093C0000E2003F08BFB07005BD0798905F10800C4
:1093D000814214D32A4631467868F7F774FB294650
:1093E000384604F01FF828B1B62229A132A001F0B6
:1093F0000DFD04E02146384603F05AFD18B1384609
:1094000003F0CAFE3DE0204603F0C6FE3C460AE0FB
:109410003946204604F006F828B1C7221CA133A023
:1094200001F0F4FC2DE029462046676803F013FBA9
:1094300038BB6668D9F800004FF6F771F060D8F8CD
:10944000100030614FF0000887F80080788888426B
:1094500001D9093000E008307880FF203072A6F88A
:109460000A802946304600F0D3F870810121CDE909
:109470000081FF230022CDF808A04946204600F0D5
:1094800027FA2046BDE8FE4F03F086BEE0620020CA
:109490002E2E5C447269766572735C4C7749505C21
:1094A0007372635C636F72655C697076345C696368
:1094B0006D702E630000000069636D705F696E70EF
:1094C00075743A206D6F76696E6720722D3E7061FB
:1094D000796C6F616420746F2069636D70206865BA
:1094E00061646572206661696C65640069636D70B2
:1094F0005F696E7075743A20726573746F72696E0D
:1095000067206F726967696E616C20702D3E7061B3
:10951000796C6F6164206661696C656400000000AD
:109520002DE9FF47074600891C24924689461C28DE
:1095300000D2044604F10805A9B24FF4207222209B
:1095400003F0CCFA060036D07089A84205D240F26A
:109550006D121AA123A001F059FC7568D7F8048098
:10956000082385F8009085F801A04FF00009C5F8A0
:10957000049022463946304603F010FDD8F80C001E
:10958000039003A800F060FA040011D0A5F802903F
:109590004F467189284600F03BF86880012000970B
:1095A000CDE90104FF2303AA0021304600F090F921
:1095B000304603F0F1FDBDE8FF8700002E2E5C442D
:1095C0007269766572735C4C7749505C7372635C48
:1095D000636F72655C697076345C69636D702E636D
:1095E00000000000636865636B2074686174206626
:1095F0006972737420706275662063616E20686F93
:109600006C642069636D70206D65737361676500BC
:1096100000B501F029FCC04380B200BD70B5002642
:109620003446054612E06989686801F01DFC204453
:1096300081B201EB1044A87AC00706D08EB1002693
:10964000E0B2C4F3072141EA00242D68002DEAD1DD
:1096500026B1E0B2C4F3072141EA0024E04380B21E
:1096600070BD0126ECE730B41B68029D9CB204EB90
:1096700013442B689DB22C4404EB13439CB204EBBF
:1096800013439CB204EB134330BCAFF300802DE9CD
:10969000F0411C4690460F460026054612E06989B7
:1096A000686801F0E1FB204481B201EB1044A87A24
:1096B000C00706D0FEB10026E0B2C4F3072141EA9C
:1096C00000242D68002DEAD126B1E0B2C4F30721B1
:1096D00041EA0024384600F0A3FB0444404600F071
:1096E0009FFB204481B201EB104000EB1040C043CF
:1096F00080B2BDE8F0810126DEE7421C12D088B1BD
:1097000091F82D2092070BD54B68834208D08968C9
:1097100000EA01020B409A4202D10143491C01D0E8
:1097200000207047012070472DE9F0474568074643
:109730000E4628780421B1EB101F03D0384603F001
:109740002BFDA8E000074FEA9068688800F068FBEE
:1097500004463889A04203D92146384603F0A4FDC7
:1097600079894145EAD33889A042E7D34046B8F128
:10977000140FE3D301462846FFF74AFF0028DDD146
:109780002969DFF81891C1F303100E28C9F81410E5
:10979000EA68C9F8102005D0304600F083F850B1CF
:1097A000344619E096F82D00C00702D070680028F2
:1097B000F6D1002410E099F8140000247F280BD083
:1097C0003748046806E0B44203D0204600F06AF847
:1097D00010B92468002CF6D13146D9F81000FFF7F3
:1097E0008CFF0028AAD199F810104846C1F3031144
:1097F0000E29A3D0002CA1D0E98831F0C0019DD161
:109800008560C0E900462978CA460907890EA9F88B
:109810000C103146384604F05FFD814601282DD0FA
:109820004146384603F0FEFD687A012811D006282B
:109830000AD0B9F1020F1ED055462146DAF81400BD
:10984000FFF75BFF50B116E03146384606F060FC8A
:1098500014E031463846FFF77BFD0FE0287DC0F36A
:1098600003100E2807D04146384603F005FD0221BB
:109870003846FFF769FD384603F08EFC0021CAF830
:109880000010CAF80410CAF80810AAF80C10CAF898
:109890001010CAF814100020BDE8F087E062002024
:1098A0003801002010B590F82D10C9070CD0416880
:1098B00051B1064A52698A4204D001461046FFF768
:1098C0001CFF08B1012010BD002010BDE062002087
:1098D000FEB5DDE90954089E1AB109B10F6807B950
:1098E000211D0096CDE9015400F002F8FEBD0000F4
:1098F0002DE9F84F0546DDE90A87807BDDF830B0B9
:10990000994616468A46012805D040F2763234A19F
:109910003CA001F07BFA6FF00104002E4ED0142120
:10992000284603F098F800284BD168896C68142801
:1099300005D240F2AA322AA135A001F067FA84F8D4
:109940000890390247EA0920677241EA102031681D
:1099500021618AB2104400EB1140452121704FEA89
:10996000082248F48A4142EA112184F801800F1844
:10997000288900F055FA00EB07086080304F00207E
:10998000E080388800F04CFAA08039884044491CB7
:109990003980BAF1000F0ED0DAF80010E1608AB217
:1099A000104400EB114081B201EB104000EB10407D
:1099B000C04360810CE023490968EFE768891428F7
:1099C00002D22046BDE8F88F68686E4600690090B4
:1099D000DBF814305846324629469847F2E7000033
:1099E0002E2E5C447269766572735C4C7749505CCC
:1099F0007372635C636F72655C697076345C697006
:109A0000342E6300702D3E726566203D3D2031008E
:109A1000636865636B20746861742066697273742F
:109A200020706275662063616E20686F6C642073BD
:109A300074727563742069705F686472000000005E
:109A4000960100209070010870B50146144813E09B
:109A500090F82D20D3070FD053070DD543685BB185
:109A600084680D68234005EA04069E4216D09207DA
:109A700002D4C268954211D000680028E8D1094894
:109A8000006850B190F82D20D30706D0520704D5B6
:109A9000426812B109787F2900D1002070BD000012
:109AA000380100203C01002038B5049C0094FFF7E9
:109AB000DAFD38BD2DE9F0418046C52148432349F0
:109AC00001EB800494F8100310B10020BDE8F08190
:109AD000B4F80C13B4F80A034FF4807204F09AFD42
:109AE0000028F3D00546802800D98025B4F80C63FF
:109AF000002009E0A1192218761C91F80412401CDC
:109B000082F88410F6B280B2A842F3D32A4604F158
:109B100084012068FBF7E8F80021012768B1A4F868
:109B20000E1394F8110330B92A46414608A0FDF7F8
:109B300065FF84F811730320C8E7A4F80C63A4F848
:109B40000E5384F8107384F81113BEE748C8002040
:109B50005B554152545D206B69636B2D6661696C86
:109B60002063683D2575206C656E3D25750D0A00E6
:109B7000012801D00248704701480C3070470000AE
:109B80002C7200082DE9F0410746FDF73DF81F4D06
:109B90000446686828B901200BF00CFF68600028B3
:109BA00030D0FCF7EFFDFCF7B9FFFCF72BFEFCF71C
:109BB0007DFD0520FCF778FE06463920FCF774FE93
:109BC00005467F20FCF770FE014633462A4610A06A
:109BD000FDF714FF1D20FCF767FE05465320FCF738
:109BE00063FE01462A4616A0FDF708FF04F11400A3
:109BF000FEF778FE3846FFF7E5F8FCF718FE002080
:109C0000BDE8F0814FF0FF30FAE70000A801002026
:109C10005B4554485D2063666720696D723D30780E
:109C20002530325820696E7463723D3078253032A9
:109C300058207263723D3078253032580D0A00008A
:109C40005B4554485D206263206263617374637294
:109C50003D307825303258206D6172373D3078259F
:109C60003032580D0A0000002DE9F843DFF88C80EF
:109C7000C669D8F8040018B14FF0FF310CF0E6FACD
:109C800069461F48FCF79AFE9DF80010B1703080BD
:109C900048B381B24FF4C172002002F01FFF0500EB
:109CA00016D0DFF85C900027044609EB07016289B3
:109CB0006068F6F708FF60892468384487B2002C92
:109CC000F3D1B078800603D0284603F065FA00256A
:109CD000D8F8040020B100231A4619460BF09CFF67
:109CE0002846BDE8F883D8F8040020B100231A46BE
:109CF00019460BF091FF0020F3E70000A8010020B7
:109D0000D49B00202DE9F047294E0F46706818B10A
:109D10004FF0FF310CF09AFA00253C464FF4C06832
:109D2000DFF8909017E06289501940450AD97068B1
:109D300020B100231A4619460BF06EFF6FF00100A8
:109D4000BDE8F08709EB05006168F6F7BCFE6089A5
:109D50002468284485B2002CE5D139891548FCF7E0
:109D60002FFE0446706820B100231A4619460BF0F6
:109D700053FFCCB10BF072F80F4C6068401C606070
:109D8000A078FF2801D2401CA070C5B20BF096F855
:109D90002A460AA06168FDF731FE062D01D3FCF7C3
:109DA00063FA6FF00200CBE7FEF7ACFE0020C7E7D6
:109DB000A8010020D4A10020889B00205B455448C6
:109DC0005D2074782074696D656F7574206E3D2513
:109DD0006C752073747265616B3D256C750D0A009E
:109DE00010B504464068804704F0CDFE094A21685A
:109DF00052688B181A1AB2F1004F03D30844224656
:109E0000054902E0044922461846BDE8104004F026
:109E100031BF000088010020E19D000800BA7047B2
:109E200040BA704710B504F069FE01F099F901F0ED
:109E3000D9FB02F055FC06F05FF9BDE8104004F0D4
:109E400079BF0021017101684868002806D00978AF
:109E50000122B2EB111F01D105F018B9704710B5FE
:109E6000026804466FF00501506830B1127802F0C4
:109E7000F002102A08D0402A02D00846207110BDF6
:109E8000A16804F013FAF9E7A289A16805F082F944
:109E9000F4E7000070B5016804466FF00A024B68F1
:109EA0004878002B49D00B780125B5EB131F44D11E
:109EB000237A032B01D002283FD003283DD001286C
:109EC00038D0D80702D0084601F067FE2068406A03
:109ED00028B140F2C7721AA122A000F097FF2168B2
:109EE00004204870206800214462206800F04EF889
:109EF000002821D020684078042805D040F2CC7298
:109F00000FA11FA000F082FF1F4804F039FE0021BE
:109F1000606A04F0B1FD1C4804F021FE206840781E
:109F2000002809D0BDE870404FF4FA6204A114A0E3
:109F300000F06CBFFB20207170BD227170BD00006D
:109F40002E2E5C447269766572735C4C7749505C66
:109F50007372635C6170695C6170695F6D73672EB9
:109F600063000000616C72656164792077726974C6
:109F7000696E67206F7220636C6F73696E67000093
:109F80007374617465210000A40100202DE9F05F65
:109F90008B46040005D140F2A6326AA172A000F0FF
:109FA00035FF20780121B1EB101F05D040F2A73218
:109FB00064A171A000F02AFF6078042805D04FF456
:109FC0006A7260A174A000F021FF606828B940F2B5
:109FD000A9325CA179A000F019FF606A28B940F2AB
:109FE000AA3258A17AA000F011FF606AD4F8048068
:109FF000007A00F0010900F0020703280FD0B9F140
:10A00000000F07D098F81400052808D0062806D0BD
:10A01000082804D04FB198F81A00C00605D50126CB
:10A020000021404605F02EF800E0002698F81400C4
:10A0300001281DD0B9F1000F07D00021404608F0DB
:10A0400025FA0021404604F04CFF1FB10021404694
:10A0500008F0AEFD96B100221146404607F0A8FC7C
:10A060000021404605F022FF404605F02DFB0AE0A6
:10A070000021404604F035FF002EF5D13A4649460E
:10A08000404608F0EFFE050013D0681C11D1A0690E
:10A0900044F6206A002800DD824604F074FD616AFF
:10A0A000C968411A51450DDB1EB1404604F016FF48
:10A0B0000025606AD0F8248005710020606260701D
:10A0C0002DB11CE098F81400012821D026E036B10B
:10A0D0006060A36A1BB10022042120469847B9F1B1
:10A0E000000F05D0A36A1BB10022114620469847F5
:10A0F0002FB1A36A1BB10022022120469847BBF171
:10A10000000F02D0404604F056FD0020BDE8F09F4D
:10A1100040F245420BA135A000F078FE1FB13C494A
:10A12000404608F045FD01223A49404607F040FC10
:10A130003949404605F0BAFE2146404604F0A2FFE8
:10A140002846E3E72E2E5C447269766572735C4C98
:10A150007749505C7372635C6170695C6170695FC0
:10A160006D73672E63000000696E76616C69642010
:10A17000636F6E6E0000000074686973206973205D
:10A18000666F7220746370206E6574636F6E6E7399
:10A19000206F6E6C79000000636F6E6E206D7573BA
:10A1A0007420626520696E207374617465204E4569
:10A1B00054434F4E4E5F434C4F53450070636220F3
:10A1C000616C726561647920636C6F736564000013
:10A1D000636F6E6E2D3E63757272656E745F6D7324
:10A1E0006720213D204E554C4C000000436C6F739E
:10A1F000696E672061206C697374656E207063629C
:10A20000206D6179206E6F74206661696C21000099
:10A21000B1E80008C5D60008597B000810B504460F
:10A22000006842686AB1017801F0F001102910D08D
:10A23000402909D033A0F6F707F96FF00500207127
:10A2400010BD6FF00E00FAE71046A16804F037F871
:10A25000F5E74178032903D029B16FF00900EEE753
:10A260006FF00800EBE704F0A1FB2068A289A16869
:10A2700040682A4B05F064FB0028E0D121680322E6
:10A2800091F820004A70C0F340000028206810F8C0
:10A29000201F05D041F0040101706FF00400CEE7EB
:10A2A00001F0FB01017020684462206840780328B7
:10A2B00005D040F274521AA122A000F0A7FD234855
:10A2C00004F05EFC2068C169606A04F0D5FB401CA4
:10A2D00009D120684178032905D100214162206815
:10A2E0004170FD202071194804F039FC2068407845
:10A2F0000328A5D1BDE8104040F27E5208A111A06C
:10A3000000F084BD496E76616C6964206E6574638B
:10A310006F6E6E20747970650000000051A3000814
:10A320002E2E5C447269766572735C4C7749505C82
:10A330007372635C6170695C6170695F6D73672ED5
:10A34000630000007374617465210000A4010020A3
:10A3500070B50026154604000BD06078032805D0A0
:10A3600040F2275222A12BA000F050FD606A18B1E4
:10A370000EE06FF0050070BD94F8200040070AD48D
:10A380004FF4A5621AA12BA000F040FD606A10B145
:10A390000571606A466A20780121B1EB101F03D174
:10A3A00015B9204604F002FB94F8200040F3800524
:10A3B00000F0FB0084F820006D1C00D046B955EA7F
:10A3C000060005D040F2345209A12AA000F01EFD7B
:10A3D000002060626070A36A1BB100220221204647
:10A3E000984715B1304604F0E6FB002070BD000030
:10A3F0002E2E5C447269766572735C4C7749505CB2
:10A400007372635C6170695C6170695F6D73672E04
:10A4100063000000636F6E6E2D3E7374617465207F
:10A420003D3D204E4554434F4E4E5F434F4E4E45AB
:10A430004354000028636F6E6E2D3E637572726523
:10A440006E745F6D736720213D204E554C4C292062
:10A450007C7C20636F6E6E2D3E696E5F6E6F6E5FEB
:10A46000626C6F636B696E675F636F6E6E6563745A
:10A4700000000000626C6F636B696E6720636F6E33
:10A480006E656374207374617465206572726F7297
:10A490000000000070B5044600684578B5B100784A
:10A4A0000121B1EB101F05D040F2624233A13CA064
:10A4B00000F0ACFC022D09D0032D04D1206890F8E7
:10A4C0002000400702D4FB20207170BD00252571BB
:10A4D000206801F062FB2168486850B10A7802F0F8
:10A4E000F002102A15D0402A01D103F0A3FF206802
:10A4F00045602068836A002BE7D000221146984708
:10A500002068836A002BE0D0BDE870400022022161
:10A510001847486A28B14FF4936218A125A000F0AB
:10A5200075FC2168042048700320207220680021F7
:10A5300044622068FFF72AFD0028C6D020684078D2
:10A54000042805D040F29E420CA121A000F05EFC40
:10A55000214804F015FB0021606A04F08DFA1E48C2
:10A5600004F0FDFA206840780028AED0BDE87040C5
:10A5700040F2A24201A116A000F048BC2E2E5C447D
:10A580007269766572735C4C7749505C7372635C78
:10A590006170695C6170695F6D73672E63000000B4
:10A5A0006E6574636F6E6E2073746174652065727E
:10A5B000726F7200616C7265616479207772697480
:10A5C000696E67206F7220636C6F73696E6700003D
:10A5D0007374617465210000A4010020F8B502685D
:10A5E00004466FF00A01506848B113780125B5EBB5
:10A5F000131F5DD15278002622B1022A43D08DF874
:10A60000001051E0017D21B15FF0FA008DF80000EB
:10A610004AE0217A6A4606F06DFA050044D02068C7
:10A6200010F10C0F09D0C16839B10C3004F067FA91
:10A63000206810F10C0F00D0C6608DF80060206813
:10A6400010F1100F01D0016929B90621103004F072
:10A6500069FA8DF800009DF8000028B1284605F041
:10A6600033F8206846601FE02168022048702168A6
:10A6700028464D60216804F005FD20680D494068BA
:10A6800004F02FFC10E08DF80060007D012805D05B
:10A690004FF4BE6208A111A000F0B8FB207A00B907
:10A6A00001202168496808779DF800002071F8BDF5
:10A6B000F020ABE7896000082E2E5C447269766555
:10A6C00072735C4C7749505C7372635C6170695C57
:10A6D0006170695F6D73672E630000007063622DA7
:10A6E0003E7374617465203D3D204C495354454E82
:10A6F000202863616C6C656420666F722077726FCE
:10A700006E67207063623F29000000000021017124
:10A7100001684968002901D102F0CCBE70472DE9DB
:10A72000F04104460020207120684168002915D0BE
:10A7300000780121B1EB101F10D1A5680F044FF66E
:10A74000FF78BD4201D3404600E0284686B220682B
:10A750003146406807F0F6FEAD1BF2D1BDE8F0814E
:10A7600010B50446006801F06BFA00284BD1206850
:10A7700001210278B1EB121F43D142780AB1881F40
:10A7800041E04268002A39D041702068406A28B10F
:10A7900040F22D721DA126A000F038FB606928B997
:10A7A00040F22E7219A129A000F030FB2068002190
:10A7B0004462206800F05AF8002825D020684078CC
:10A7C000012805D040F2327210A125A000F01EFB36
:10A7D000254804F0D5F90021606A04F04DF92248BB
:10A7E00004F0BDF92068407801280DD1BDE8104083
:10A7F00040F2367205A11AA000F008BB6FF00A0003
:10A8000001E06FF00500207110BD00002E2E5C44A9
:10A810007269766572735C4C7749505C7372635CE5
:10A820006170695C6170695F6D73672E6300000021
:10A83000616C72656164792077726974696E6720F2
:10A840006F7220636C6F73696E6700006D73672DA4
:10A850003E6D73672E772E6C656E20213D20300093
:10A860007374617465210000A40100202DE9F34F89
:10A8700081B004004FF0000A05D140F27D628AA148
:10A8800092A000F0C3FA6078012805D040F27E6201
:10A8900085A192A000F0BAFA606A28B940F27F62FE
:10A8A00081A196A000F0B2FA606828B94FF4D06296
:10A8B0007DA199A000F0AAFA606A8169406981428D
:10A8C00005D340F2816278A199A000F09FFA606AF6
:10A8D000808928B940F2836273A1A5A000F096FA9E
:10A8E000606A077F94F82000800701D4780701D5BB
:10A8F000012000E000208046A0696FF0060BD0B177
:10A9000004F041F90146606A026A891AA26991421B
:10A9100011DB8069002878D00025606A416A0571E2
:10A92000002060626070029810B1084604F043F99C
:10A930000020BDE8FE8F616A4FF48039886809699C
:10A9400002680A4400924268551A4D4504D34FF6F6
:10A95000FF7647F0020700E0AEB26068B0F864002E
:10A96000B0420DD20646B8F1000F07D046B9606A72
:10A97000806908B100254FE05D464DE047F00207D1
:10A980008819904205D940F2AD6247A182A000F03B
:10A990003DFAA6F57F40FF3801D14D4506D2A8B259
:10A9A000B04208D1606A8089012804D94FF00109BA
:10A9B00047F0020701E04FF000093B46324660686D
:10A9C000009908F011FF050019D1606A81693144CE
:10A9D0008161606A016931440161606A826852681C
:10A9E00091420CD18189491E0904090C8181606A58
:10A9F00005D0816808318160616A00200861B9F181
:10AA0000000F03D0002D96D001E04BE00DB1681C83
:10AA100083D1B8F1000F11D0606A81694069814229
:10AA20000CD2A36A1BB1002203212046984794F858
:10AA3000200040F0100084F820000FE06068B0F8BB
:10AA40006410B1F5866F03D3B0F86600052805D30E
:10AA5000A36A1BB100220321204698475DB1681C00
:10AA6000D6D1606806F0F0F9011D19D0B8F1000FD9
:10AA700013D0606A4DE7606A81694069814202D003
:10AA8000B8F1000F01D04FF0010A606806F0DCF960
:10AA9000011D05D0BAF1000FBAD14FF0FF3048E7E1
:10AAA00005463AE75D4638E72E2E5C4472697665C6
:10AAB00072735C4C7749505C7372635C6170695C63
:10AAC0006170695F6D73672E63000000636F6E6E67
:10AAD00020213D204E554C4C00000000636F6E6EEF
:10AAE0002D3E7374617465203D3D204E4554434FA7
:10AAF0004E4E5F575249544500000000636F6E6E22
:10AB00002D3E63757272656E745F6D736720213DB3
:10AB1000204E554C4C000000636F6E6E2D3E7063EE
:10AB2000622E74637020213D204E554C4C00000075
:10AB3000636F6E6E2D3E63757272656E745F6D73BA
:10AB4000672D3E6D73672E772E6F66667365742072
:10AB50003C20636F6E6E2D3E63757272656E745F1E
:10AB60006D73672D3E6D73672E772E6C656E0000DA
:10AB7000636F6E6E2D3E63757272656E745F6D737A
:10AB8000672D3E6D73672E772E766563746F725FE7
:10AB9000636E74203E2030006C7769705F6E657460
:10ABA000636F6E6E5F646F5F77726974656D6F72ED
:10ABB000653A20696E76616C6964206C656E6774B5
:10ABC0006821000010B510F10F0F12D010F10E0F18
:10ABD0000CD010F10D0F07D020B17D2206A10FA0DF
:10ABE00000F014F9002010BD104810BD0F48401CA3
:10ABF00010BD0E48801C10BD2E2E5C447269766517
:10AC000072735C4C7749505C7372635C6170695C11
:10AC10006170695F6D73672E63000000756E686117
:10AC20006E646C6564206572726F720094700108C6
:10AC300070B50C00054604D185220CA114A000F0CB
:10AC4000E5F81648854201D1F3200AE01348401C7C
:10AC5000854201D1F22004E01048801C854203D1D6
:10AC6000F1202070012070BD002070BD2E2E5C44AC
:10AC70007269766572735C4C7749505C7372635C81
:10AC80006170695C6170695F6D73672E63000000BD
:10AC900065727220213D204E554C4C009470010885
:10ACA0002DE9FE4F2D4D00238C462B602C4E6FF06E
:10ACB000004131602B4F3960DFF8AC90C9F80010CB
:10ACC000DFF8A8A0CAF80010294C02212160032156
:10ACD0002160DFF8A4802749CDE9003802911346AE
:10ACE00001466246254801F0FDFD010031604FF04C
:10ACF000FF3602D02E6022A023E004202060002234
:10AD000027491E4801F00AFE0100396002D02E607A
:10AD100024A016E000222B49184801F0FFFD010095
:10AD2000C9F8001002D02E6027A00AE000222F49A7
:10AD3000124801F0F3FD0100CAF8001006D02E60A1
:10AD40002BA003B0BDE8F04FFCF758BE05202060F3
:10AD50000620206001202860BDE8FE8F5000002002
:10AD60004000002044000020480000204C0000204B
:10AD70003C00002029420108A18B0008A09B002074
:10AD80005B4554485D206E657469662D616464207E
:10AD90006661696C206572723D25640D0A000000D1
:10ADA000D1C700085B4554485D207365742D646508
:10ADB0006661756C74206661696C206572723D25F0
:10ADC000640D0A00DDC700085B4554485D207365CB
:10ADD000742D6C696E6B2D646F776E206661696C83
:10ADE000206572723D25640D0A00000061C80008EC
:10ADF0005B4554485D207365742D757020666169EC
:10AE00006C206572723D25640D0A000001B908A12D
:10AE100000B907A013460A46014607A0FCF7EEFD5D
:10AE2000502080F31188BFF34F8FBFF36F8FFEE781
:10AE3000286E756C6C2900005B4641554C545D20B2
:10AE40006C7769702D617373657274206D73673DE3
:10AE500025732066696C653D2573206C696E653DC0
:10AE600025640D0A0000000018B50022ADF800208E
:10AE700010F001030CD000290ADD10F8014B8DF809
:10AE80000140491E04E000BF30F8024B891E2244F5
:10AE90000129F9DC002902DD00788DF80000BDF8F9
:10AEA0000000104481B201EB104081B201EB104070
:10AEB00023B1C1B2C0F3072040EA012080B218BD1F
:10AEC000F8F786FEFCF798FD26A0FCF75BFDFAF785
:10AED0008BFC27A0FCF756FDFAF7C8F8F9F75CFFE2
:10AEE000FAF762F9FBF7AEFE0120FBF79FFE04467E
:10AEF0000020FBF79BFE2146FAF730FFFAF770F9C6
:10AF0000FAF78CF9FAF72CF91DA0FCF73BFD0122AA
:10AF100051032048F8F712FE1F4C00220221204660
:10AF2000F8F70CFE0120F8F741FC0122022120462F
:10AF3000F8F704FE3220F8F739FC012210211748F7
:10AF4000F8F7FCFD16A0FCF71DFD01F00BFDF9F76D
:10AF500061FF17A0FCF716FD19A0FCF713FD01F027
:10AF600013FDFEE768616C2D696E697400000000D6
:10AF7000636C6F636B2D636F6E6669670000000022
:10AF80007065726970686572616C732D7265616459
:10AF90007900000000100140000C01400008014051
:10AFA000636F6E6669672D726561647900000000E9
:10AFB0006672656572746F732D696E697400000046
:10AFC0007363686564756C65722D73746172740067
:10AFD0002DE9F041002860D0810704D040F27322AF
:10AFE0002FA137A00DE03F4DA0F1080429688C4245
:10AFF00003D369680C30884206D940F27F2228A129
:10B0000039A0FFF703FF2FE03648083003F0A7FD13
:10B01000207900282ED02888201A86B2208803F0B4
:10B0200085F80746608803F081F821884FF4E053E3
:10B03000002299420DD8618899420AD8B14202D0C3
:10B040000088B04205D16868874218D07888B0423D
:10B0500015D040F2952212A12AA000BFFFF7D6FE1C
:10B060002048083003F08CFD03F001FDBDE8F041FD
:10B0700003F01FBD4FF4237209A12FA0EEE7227148
:10B08000E868844200D2EC60204602F06BFABDE82A
:10B09000F0411448083003F073BDBDE8F0810000B2
:10B0A0002E2E5C447269766572735C4C7749505CF5
:10B0B0007372635C636F72655C6D656D2E63000017
:10B0C0006D656D5F667265653A2073616E6974794E
:10B0D00020636865636B20616C69676E6D656E7473
:10B0E00000000000F80000206D656D5F6672656508
:10B0F0003A20696C6C6567616C206D656D6F727963
:10B10000000000006D656D5F667265653A20696CD0
:10B110006C6567616C206D656D6F72793A206E6F3A
:10B120006E2D6C696E6B65643A20646F75626C6538
:10B1300020667265650000006D656D5F667265650D
:10B140003A20696C6C6567616C206D656D6F727912
:10B150003A20646F75626C65206672656500000058
:10B1600070B51248124C20F003014FF4E0552160F5
:10B170000D80002048800871284602F0D7FF012189
:10B1800060600171058045802068E06004F108007E
:10B1900003F0EAFC002807D0BDE8704040F21F220F
:10B1A00004A10CA0FFF732BE70BD0000FB620020BE
:10B1B000F80000202E2E5C447269766572735C4C38
:10B1C0007749505C7372635C636F72655C6D656D2B
:10B1D0002E6300006661696C656420746F20637281
:10B1E00065617465206D656D5F6D757465780000CF
:10B1F0002DE9F04700280ED0C41C4FF6FC710C401E
:10B200004FF4E0590C2C01D20C2401E04C4501D83C
:10B21000844202D20020BDE8F087414803F09FFC41
:10B220003F48C4F5E0570838824681890288891A68
:10B230008EB26FE0304602F079FF054600790028B3
:10B2400065D12888801B0838A04260D3288804F183
:10B250001401801B08384FF0010888421CD33019B4
:10B26000083087B24F4505D140F287322DA135A075
:10B27000FFF7CCFD384602F059FF00210171298803
:10B28000018046802F8085F804800088484505D0DD
:10B2900002F04CFF478001E085F80480DAF80C00EA
:10B2A0005646854203D013E0008802F03FFF017943
:10B2B00011B171688842F7D1F0607168884207D097
:10B2C000007928B140F2B53216A123A0FFF79EFD08
:10B2D000134803F055FC281971680830884205D9D5
:10B2E00040F2B9320FA123A0FFF790FDA8070BD0C1
:10B2F00040F2BB320BA12BA0FFF788FD40F2BD321C
:10B3000008A134A0FFF782FD05F1080083E7DAF811
:10B310000000865BB7428DD8014803F031FC79E725
:10B32000000100202E2E5C447269766572735C4CBD
:10B330007749505C7372635C636F72655C6D656DB9
:10B340002E630000696E76616C6964206E657874A6
:10B3500020707472000000006D656D5F6D616C6C33
:10B360006F633A20216C667265652D3E7573656466
:10B37000000000006D656D5F6D616C6C6F633A205D
:10B38000616C6C6F6361746564206D656D6F72795B
:10B39000206E6F742061626F76652072616D5F65EB
:10B3A0006E642E006D656D5F6D616C6C6F633A202D
:10B3B000616C6C6F6361746564206D656D6F72792B
:10B3C0002070726F7065726C7920616C69676E6550
:10B3D000642E00006D656D5F6D616C6C6F633A206B
:10B3E00073616E69747920636865636B20616C6951
:10B3F000676E6D656E74000002490988401A80B25C
:10B4000070470000F80000202DE9F05F0646CC1CD4
:10B410004FF6FC7004404FF4E05A0C2C01D20C247F
:10B4200001E054452DD88C422BD3434F38688642D7
:10B4300002D37868864205D340F2D1223FA147A0CB
:10B44000FFF7E4FC3868864202D379688E4204D361
:10B4500003F00DFB03F02DFB18E0A6F10805BB4639
:10B46000281A87B22888C01B08381FFA80F94C4573
:10B4700005D94FF4397231A13EA0FFF7C7FC4C4506
:10B4800003D94FF00000BDE8F09F01D13046FAE744
:10B49000294800F1080003F062FB288802F046FE0C
:10B4A0008046007948B304F11400484520D8381983
:10B4B000083084B22888504505D140F216321FA1C9
:10B4C00034A0FFF7A3FC204602F030FEDBF80C208E
:10B4D000904201D2CBF80C00002101712988018033
:10B4E00047802C800088504502D002F01FFE448027
:10B4F0001148083003F044FBC8E72888504505D1BF
:10B5000040F2F5220DA123A0FFF780FC3819083086
:10B51000DBF80C10B8F8009084B2414504D1204605
:10B5200002F004FECBF80C00204602F0FFFD0021E3
:10B530000171A0F80090D3E7F80000202E2E5C44A3
:10B540007269766572735C4C7749505C7372635CA8
:10B55000636F72655C6D656D2E6300006D656D5F78
:10B560007472696D3A206C6567616C206D656D6FF2
:10B57000727900006D656D5F7472696D2063616E34
:10B58000206F6E6C7920736872696E6B206D656DCB
:10B590006F727900696E76616C6964206E6578748B
:10B5A00020707472000000000B2802D305A0F4F78D
:10B5B0004BBF002904D00A4A52F82000FCF73ABADF
:10B5C000704700006D656D705F667265653A207446
:10B5D000797065203C204D454D505F4D415800002D
:10B5E0000070010830B5064D002400BF55F8240056
:10B5F00000F008F8641CA4B20B2CF7D330BD000097
:10B6000000700108C268002111608168C91C21F026
:10B610000301002207E0C368521C1B680B60C3686B
:10B62000196083881944C3889342F4DC7047000092
:10B6300010B50B2804D306A0F4F706FF002010BDB8
:10B640000B4951F82000BDE81040FCF729BA000072
:10B650006D656D705F6D616C6C6F633A20747970AD
:10B6600065203C204D454D505F4D41580000000085
:10B67000007001082DE9F0410446008986B041BA06
:10B680000A04A17A45BA42EA0123E27A2D0413435F
:10B6900045EA01251B06ADB243EA052345BA40BA87
:10B6A0000004EDB240EA012043EA0523104343EAD7
:10B6B00010600290A08941BA0A04A17B45BA42EA0F
:10B6C0000123E27B2D04134345EA01251B06ADB29D
:10B6D00043EA052345BA40BA0004EDB240EA01202E
:10B6E00043EA0523104343EA10600390208A41BADD
:10B6F0000A04A17C45BA42EA0123E27C2D041343EB
:10B7000045EA01251B06ADB243EA052345BA40BA16
:10B710000004EDB240EA012043EA0523104343EA66
:10B7200010600490FDF72AFA214E00203060FAF7ED
:10B73000A1FD02E0142009F009FDFAF75DFD0028E3
:10B74000F8D0322009F002FD4FF4FA7009F0FEFC47
:10B7500004F1140304AA03A902A8FDF7DFF9FDF719
:10B76000A1F90546FDF772F90446FDF785F907468C
:10B77000B5F5E05F03D1A4F5114051380CD00AF0C3
:10B7800047F880460AF03EF8CDE900083B462246DD
:10B7900029460848FCF732F9FAF71CFD0120306011
:10B7A000FAF76EFDFAF710FD06B00120BDE8F08152
:10B7B00038000020D876010810B56FF00F0450B1A2
:10B7C00059B162B143687BB15B680B6040684089E6
:10B7D0001080002010BD06A002E00CA000E013A025
:10B7E000F4F732FE204610BD6FF0010010BD0000DE
:10B7F0006E65746275665F646174613A20696E7625
:10B80000616C696420627566000000006E65746298
:10B8100075665F646174613A20696E76616C696413
:10B820002064617461707472000000006E6574625F
:10B8300075665F646174613A20696E76616C6964F3
:10B84000206C656E0000000010B504000CD020686C
:10B8500020B101F0A1FC0020606020602146BDE81D
:10B8600010400420FFF7A0BE10BD000010B54FF03F
:10B87000FF3438B14168096839B14160086830B1B6
:10B88000002010BD03A0F4F7DFFD204610BD01200D
:10B8900010BD00006E65746275665F6E6578743AFF
:10B8A00020696E76616C6964206275660000000034
:10B8B00070B58CB00D0004466FF00F0616D0002056
:10B8C0002860ACB1204600F0BBF98DF800000028DC
:10B8D0001CD114F1100F6FF00E063AD02069002829
:10B8E00037D094F82000C10733D105E01AA000E05A
:10B8F00021A0F4F7A9FD2CE0810704F1100007D581
:10B900000BA903F0A3F8401C08D1C01F0CB070BDF8
:10B910000BA9E26903F074F8401C0DD0A36A1BB1B7
:10B92000002201212046984769460B98FFF780F9CD
:10B9300028B19DF90000E9E76FF00200E6E70B9CF3
:10B940003CB101A91448019400F088F800202C6053
:10B95000DCE73046DAE700006E6574636F6E6E5F99
:10B960006163636570743A20696E76616C69642006
:10B97000706F696E746572006E6574636F6E6E5F72
:10B980006163636570743A20696E76616C696420E6
:10B99000636F6E6E00000000439E00082DE9F041C9
:10B9A00007460E460520FFF743FE041E1DD0002566
:10B9B0002572277007F0F000656010280AD0402833
:10B9C00006D040F2EB2212A11AA0FFF71FFA07E0FF
:10B9D000042100E0062104F10C0003F0A3F830B1CB
:10B9E00021460520FFF7E0FD0020BDE8F08114F1BD
:10B9F000100F00D025616570C4E909564FF0FF3083
:10BA0000C4E90505E56184F820502046EDE7000013
:10BA10002E2E5C447269766572735C4C7749505C7B
:10BA20007372635C6170695C6170695F6D73672ECE
:10BA3000630000006E6574636F6E6E5F616C6C6FA7
:10BA4000633A20756E646566696E6564206E657420
:10BA5000636F6E6E5F7479706500000070B50546A7
:10BA6000FA200C4608710021084602F0F3FB02465A
:10BA700060622146284608F0E5FB002801D194F9D0
:10BA8000040070BD00B58BB008B139B107E008A063
:10BA9000F4F7DAFC6FF00F000BB000BD0B49029118
:10BAA0000090ADF80C2069460948FFF7D7FFF3E78F
:10BAB0006E6574636F6E6E5F62696E643A20696E64
:10BAC00076616C696420636F6E6E0000907001088F
:10BAD0005F9E0008032100F001B8000000B58BB0A4
:10BAE00058B100908DF8081003F04DF803906946A6
:10BAF0000548FFF7B3FF0BB000BD04A0F4F7A4FCAA
:10BB00006FF00F00F7E70000959E00086E65746304
:10BB10006F6E6E5F636C6F73653A20696E76616CF1
:10BB2000696420636F6E6E0000B58BB008B139B1E7
:10BB300007E008A0F4F788FC6FF00F000BB000BD21
:10BB40000C4902910090ADF80C2069460A48FFF7B5
:10BB500085FFF3E76E6574636F6E6E5F636F6E6E85
:10BB60006563743A20696E76616C696420636F6EF8
:10BB70006E000000907001081DA2000870B505005D
:10BB800004D000F09BF9040002D004E0002070BD56
:10BB9000284600F065F8204670BD2DE9FC410446BA
:10BBA00010F10C0F4FF0000721D0E06804F10C05F4
:10BBB000E8B101266946284602F048FF401C11D032
:10BBC0002078B6EB101F09D101A90098FFF730F8D3
:10BBD0000028EFD1009801F0DFFAEBE70098FFF7BB
:10BBE00033FEE7E7284602F08AFF05B1E76014F16B
:10BBF000100F23D02069002820D004F110056946D9
:10BC0000284602F023FF401C12D001A90098FFF73C
:10BC10000FF80028F3D1009E3046FFF7BEFF706892
:10BC200010B103F05BF97760304600F019F8E6E7F1
:10BC3000284602F064FF002D00D02761BDE8FC819A
:10BC400070B5040009D002F012FF94F908500021E9
:10BC5000217202F02EFF284670BD002070BD00004A
:10BC600010B50446406828B14FF448720FA118A0DF
:10BC7000FFF7CCF814F10C0F07D0E06828B140F2C0
:10BC800027320AA11EA0FFF7C1F814F1100F07D048
:10BC9000206928B140F22A3204A128A0FFF7B6F8A3
:10BCA0002146BDE810400520FFF77EBC2E2E5C44E7
:10BCB0007269766572735C4C7749505C7372635C31
:10BCC0006170695C6170695F6D73672E630000006D
:10BCD000504342206D757374206265206465616C09
:10BCE0006C6F6361746564206F757473696465203B
:10BCF000746869732066756E6374696F6E00000006
:10BD0000726563766D626F78206D757374206265FD
:10BD1000206465616C6C6F63617465642062656644
:10BD20006F72652063616C6C696E672074686973FB
:10BD30002066756E6374696F6E00000061636365F1
:10BD400070746D626F78206D757374206265206405
:10BD500065616C6C6F6361746564206265666F72A7
:10BD6000652063616C6C696E672074686973206616
:10BD7000756E6374696F6E0000B58BB040B1009052
:10BD80008DF8081069460548FFF768FE0BB000BD46
:10BD900003A0F4F759FB6FF00F00F7E7DDA50008EB
:10BDA0006E6574636F6E6E5F6C697374656E3A2056
:10BDB000696E76616C696420636F6E6E00000000CE
:10BDC00030B50D468BB01146FFF7E8FD04002ED0CC
:10BDD0008DF80850694617480094FFF73FFE002889
:10BDE00025D0606820B1A32213A11CA0FFF70EF894
:10BDF00014F10C0F01D0E06820B9A4220EA120A0FC
:10BE0000FFF704F814F1100F06D0206920B1A62224
:10BE100009A121A0FEF7FAFF04F10C0002F06FFE69
:10BE200021460520FFF7C0FB00200BB030BD2046A7
:10BE3000FBE700000DA700082E2E5C4472697665B2
:10BE400072735C4C7749505C7372635C6170695CBF
:10BE50006170695F6C69622E6300000066726565DF
:10BE6000696E6720636F6E6E20776974686F757492
:10BE70002066726565696E6720706362000000006D
:10BE8000636F6E6E20686173206E6F2072656376DB
:10BE90006D626F7800000000636F6E6E2D3E61630F
:10BEA000636570746D626F782073686F756C646E13
:10BEB00027742065786973740000000000B58BB0AA
:10BEC000002807D0009002F05EFE03906946024809
:10BED000FFF7C4FD0BB000BD95A40008F8B50E0037
:10BEE00007466FF00F041AD000253560CFB13878BF
:10BEF0000121B1EB101F2DD104200095FFF798FB15
:10BF0000040013D000226946384600F005F9070006
:10BF10000FD021460420FFF747FB3846F8BD11A09B
:10BF200000E018A0F4F790FA2046F8BD4FF0FF307B
:10BF3000F8BD009828B940F2793219A121A0FEF786
:10BF400065FF0098206000986060A581A5600020D2
:10BF50003460F8BD31463846BDE8F840002200F0B4
:10BF600037B800006E6574636F6E6E5F72656376DE
:10BF70003A20696E76616C696420706F696E7465D1
:10BF8000720000006E6574636F6E6E5F726563763B
:10BF90003A20696E76616C696420636F6E6E000092
:10BFA0002E2E5C447269766572735C4C7749505CE6
:10BFB0007372635C6170695C6170695F6C69622E49
:10BFC000630000007020213D204E554C4C000000C5
:10BFD0007CB504464FF000000D006FF00F06009096
:10BFE00013D028609CB114F10C0F6FF00A0612D028
:10BFF000E06880B194F8201004F10C008B0712D493
:10C00000520710D4C9070ED10BE028A000E02FA0E2
:10C01000F4F71AFA15E02046FFF712FE002811D1B6
:10C020000FE0217A91B1694602F010FD401C13D156
:10C030002046FFF705FE002804D194F82000C00731
:10C0400001D030467CBD6FF006007CBD6946E269D8
:10C0500002F0D6FC401C10D020780121B1EB101F5B
:10C0600010D101A90098FEF7E3FD48B19DF9040045
:10C0700010F10F0FE9D100207CBD6FF002007CBDF4
:10C08000009809E0009828B940F2912216A11FA05B
:10C09000FEF7BCFE00980068A36A028913B1012173
:10C0A0002046984700982860E5E700006E657463B5
:10C0B0006F6E6E5F726563763A20696E76616C6949
:10C0C0006420706F696E7465720000006E65746341
:10C0D0006F6E6E5F726563763A20696E76616C6929
:10C0E0006420636F6E6E00002E2E5C44726976656C
:10C0F00072735C4C7749505C7372635C6170695C0D
:10C100006170695F6C69622E630000006275662071
:10C11000213D204E554C4C00F0B58BB00D460446E9
:10C12000174610F10C0F0AD0E06840B194F82000D7
:10C13000010608D500F07F0084F8200021E06FF0B0
:10C140000A000BB0F0BD29462046FFF741FF06006C
:10C15000F7D12D68380707D40DB1298900E00121F6
:10C160006A46204600F024F80DB13046E9E7F806AB
:10C1700007D514F8200F40F0800020706FF0060003
:10C18000DFE7A36A1BB100220121204698476068BF
:10C1900030B101212046FFF7A1FC6FF00E00D0E77F
:10C1A0002046FFF74DFD0028CBD16FF00D00C8E70A
:10C1B00010B520B103780124B4EB131F05D007A0FC
:10C1C000F4F742F96FF00F0010BD91601060BDE808
:10C1D000104011460A48FFF741BC00006E657463C9
:10C1E0006F6E6E5F726563765F7463705F706275A9
:10C1F000663A20696E76616C696420636F6E6E00CA
:10C200001FA7000810B50021084602F023F80028F7
:10C2100014D00068002811D00021084602F01AF856
:10C2200004000BD002F0B1FC2046FEF7D1FE002244
:10C23000BDE810401146104609F04EB910BD00008F
:10C2400010B50021084602F005F810B1006800287A
:10C2500028D10420FEF7CCFF040009D000200146BD
:10C260002060204602F09BFCB0B12046FEF7B0FEF5
:10C270000021084601F0EEFF30B10021084601F030
:10C28000E9FF006800280DD1BDE810404FF4A96215
:10C2900005A10EA0FEF7BABD00212246084609F00E
:10C2A0001BF9E5E710BD00002E2E5C44726976652F
:10C2B00072735C4C7749505C7372635C6170695C4B
:10C2C0006170695F6C69622E630000004C574950D1
:10C2D0005F4E4554434F4E4E5F5448524541445F74
:10C2E00053454D5F414C4C4F432829206661696C92
:10C2F000656400003EB5069C0094CDE90112012260
:10C3000001A900F001F83EBD2DE9F0418AB0109D71
:10C3100050B1047801266FF00508B6EB141F0BD05E
:10C320002CA0F4F791F83CE033A0F4F78DF86FF00F
:10C330000F000AB0BDE8F08190F82040A40701D4B6
:10C340005C0703D5846901261CB903E084690026D3
:10C350000CB101262DB30024274607E001EBC70CE2
:10C36000DCF804C06444A4451BD87F1C9742F5DB6D
:10C37000ACB1B4F1004F02D39DB16FF00044029113
:10C3800000210090ADF80C2004918DF81C30CDE90F
:10C390000541806938B102F0F6FB089004E0002006
:10C3A000C7E74046C5E7089169461A48FFF756FBBC
:10C3B00007000CD10DB10698286046B90698A04236
:10C3C00005D04FF4866214A11CA0FEF71FFD38466D
:10C3D000AFE700006E6574636F6E6E5F77726974AD
:10C3E000653A20696E76616C696420636F6E6E2DAC
:10C3F0003E747970650000006E6574636F6E6E5FE9
:10C4000077726974653A20696E76616C696420633D
:10C410006F6E6E0061A700082E2E5C44726976650F
:10C4200072735C4C7749505C7372635C6170695CD9
:10C430006170695F6C69622E63000000646F5F77F2
:10C4400072697465206661696C656420746F207719
:10C450007269746520616C6C206279746573000088
:10C460002DE9F0470400DDE90970089D02D01FB1F5
:10C4700031B106E030A000E036A0F3F7E5FF1CE0A4
:10C480003D4902B93C4A03B93B4B00266660A660B1
:10C49000DFF8E8C0C4F814C0E660A68484F82D6014
:10C4A000E561374D95F800C084F830C02061204622
:10C4B00000F05EF92046B84710B10020BDE8F087D3
:10C4C000B2464FF4CE784FF4CF7900BF94F83000E5
:10C4D000FF2801D184F830A000276E681CE0A64236
:10C4E00004D1424627A130A0FEF790FC7F1CFF2F0D
:10C4F00004DD4A4623A131A0FEF788FC96F83000FF
:10C5000094F83010884206D1C8B2401C84F830003C
:10C51000002EDBD102E03668002EE0D194F8300026
:10C52000FE2806D0401C28706868206020466C6099
:10C53000C4E785F800A0F7E76E657469665F61641B
:10C54000643A20696E76616C6964206E6574696610
:10C55000000000006E657469665F6164643A204E95
:10C560006F20696E69742066756E6374696F6E20E2
:10C57000676976656E0000009070010869C7000861
:10C58000340100202E2E5C447269766572735C4C17
:10C590007749505C7372635C636F72655C6E65743F
:10C5A00069662E63000000006E6574696620616C28
:10C5B000726561647920616464656400746F6F20E2
:10C5C0006D616E79206E65746966732C206D61787B
:10C5D0002E20737570706F72746564206E756D6255
:10C5E00065722069732032353500000070B50C4645
:10C5F000054604F05DFB21462846BDE8704001F089
:10C60000E3BE0A68C3689A4204D001B90022C2603E
:10C610000120704700207047F8B516460C0005460B
:10C6200005D14FF4EE7211A119A0FEF7EFFB2EB960
:10C6300040F2DD120DA116A0FEF7E8FB2068696844
:10C64000884211D000906868306069463046FFF734
:10C65000CDFF3CB1206868600121284600F042F817
:10C660000120F8BD0020F6E70020F8BD2E2E5C4426
:10C670007269766572735C4C7749505C7372635C67
:10C68000636F72655C6E657469662E6300000000FE
:10C69000696E76616C696420706F696E7465720092
:10C6A0000A6883689A4204D001B90022826001209E
:10C6B000704700207047000001000CD00748406818
:10C6C00007E000BF90F83020521CD2B28A4203D05B
:10C6D00000680028F6D100207047000034010020D7
:10C6E0007047000070B50D46040005D14FF462722A
:10C6F0000BA114A0FEF78AFB94F82D0041070ED57C
:10C70000C1070CD0E9070AD06168002907D00007EB
:10C7100005D5211D2046BDE87040FBF72DBF70BD3B
:10C720002E2E5C447269766572735C4C7749505C5E
:10C730007372635C636F72655C6E657469662E63A9
:10C74000000000006E657469665F69737375655FEC
:10C750007265706F7274733A20696E76616C696489
:10C76000206E6574696600006FF00B007047000072
:10C770002DE9F84F4FF000091D4616460C00824681
:10C78000C84600D1114C06B9104E05B90F4DACB1D9
:10C79000206898B100274A4631465046FFF780FF8F
:10C7A000424629465046FFF72CFF002F04D16A4627
:10C7B00021465046FFF730FFBDE8F88F01276A4653
:10C7C00021465046FFF728FFE5E70000907001087A
:10C7D00001498860704700003401002040B190F8A2
:10C7E0002D104A0703D501F0FB0180F82D1070478A
:10C7F00001A0F3F729BE00006E657469665F73657A
:10C80000745F6C696E6B5F646F776E3A20696E76E9
:10C81000616C6964206E65746966000050B190F8BF
:10C820002D104A0709D441F0040180F82D1003218E
:10C83000FFF758BF01A0F3F707BE70476E65746934
:10C84000665F7365745F6C696E6B5F75703A2069C3
:10C850006E76616C6964206E657469660000000024
:10C8600050B190F82D10CA0709D141F0010180F8AC
:10C870002D100321FFF736BF01A0F3F7E5BD704788
:10C880006E657469665F7365745F75703A20696E72
:10C8900076616C6964206E65746966000EB500F19E
:10C8A0001401001D0EC98DE80E000FC8FFF7D8FD5A
:10C8B00008B100200EBD6FF00B000EBD10B5014693
:10C8C000C268406812B1BDE81040104789688847C7
:10C8D000002010BD10B5001D0FC8FFF749FF002054
:10C8E00010BD000070B588B0DDE90D540C9E01B993
:10C8F000084902B9074A03B9064B0DF1040C8CE84C
:10C900004F00CDE906546946034807F003FC08B020
:10C9100070BD0000907001089DC8000800B589B086
:10C9200001AB83E807006946024807F0F3FB09B052
:10C9300000BD0000BDC8000800B589B001B90749B5
:10C9400002B9064A03B9054B0DF1040C8CE80F003F
:10C950006946034807F0DEFB09B000BD907001088E
:10C96000D5C80008EFF3058010B16FF005007047DF
:10C970000448016811B14FF0FF3070470121016098
:10C9800000207047C800002010B5EFF3058010B1FB
:10C990006FF0050010BD08480168012902D04FF072
:10C9A000FF3010BD054A002182F8141D02210160EC
:10C9B00008F0D0FD002010BDC80000200BE000E012
:10C9C0002DE9F041044616460D460846F4F75CF89A
:10C9D0000346224611E000BF12F8011B6D1CA1F1B5
:10C9E0006107192F01D82039C9B2A0F16107192FA9
:10C9F00001D82038C0B2814205D128780028EBD177
:10CA0000E05C3D2802D00020BDE8F081E018401C29
:10CA100001F0EEFF30600120F6E72DE9F843914682
:10CA20000E461D4607460A226946F3F7A9FF04464B
:10CA300000984FF0FF38B84207D001F0D9FF0078D6
:10CA400018B9B44201D34C4502D94046BDE8F88339
:10CA500000202C60FAE70022AFF3008070B598B197
:10CA6000B1F5803F22D2B1B104898BB21C44A4B28B
:10CA70009C421BD3057B2D060FD54268511A00F14D
:10CA80001002914212D30BE04FF4F17208A110A0F2
:10CA9000FEF7BCF90AE0002070BD3AB14268511AB5
:10CAA00041604189194441810481F4E7012070BD4E
:10CAB0002E2E5C447269766572735C4C7749505CCB
:10CAC0007372635C636F72655C706275662E63007F
:10CAD0007020213D204E554C4C0000002DE9FC5F9C
:10CAE000054690460F461046012A0ED041280CD02C
:10CAF000B0F5C17F0FD0B2F5207F4FD040F22712A2
:10CB00003DA145A0FEF782F957E00246002000F063
:10CB1000D9F804466EE00024A1460A20FEF788FDFD
:10CB2000060034D005F1030B2BF00300C0F51470A0
:10CB3000B84200D9384682460020CDE900807019FD
:10CB4000133020F0030153463A46304600F09EFB76
:10CB50003079800705D04FF4807227A135A0FEF709
:10CB600055F99421B1EB9B0F05D14FF4817222A1AD
:10CB70003CA0FEF74BF97CB1C9F80060A7EB0A00B6
:10CB80000704B1463F0C4FF00005C6D132E0A4B116
:10CB9000204600F001FB10E03446EFE7E81C20F0EF
:10CBA0000301F81C20F00302881880B200F1100184
:10CBB00089B2824201D88A4202D90020BDE8FC9F96
:10CBC0000846FEF715FB041EF8D00020CDE90080D2
:10CBD0006019133020F003013B461A46204600F04E
:10CBE00055FB2079800705D04FF4917202A12AA04D
:10CBF000FEF70CF92046E1E72E2E5C44726976655B
:10CC000072735C4C7749505C7372635C636F7265DE
:10CC10005C706275662E6300706275665F616C6C35
:10CC20006F633A206572726F6E656F7573207479E9
:10CC300070650000706275665F616C6C6F633A20AE
:10CC40007062756620712D3E7061796C6F61642031
:10CC500070726F7065726C7920616C69676E656463
:10CC600000000000504255465F504F4F4C5F425508
:10CC70004653495A45206D75737420626520626978
:10CC800067676572207468616E204D454D5F414C49
:10CC900049474E4D454E5400706275665F616C6C3D
:10CCA0006F633A20706275662D3E7061796C6F61BA
:10CCB000642070726F7065726C7920616C69676E48
:10CCC000656400002DE9FC4114460E460746412AE2
:10CCD00007D0012C05D04FF4A5720BA112A0FEF7CE
:10CCE00095F80920FEF7A4FC05004FF0000008D0DD
:10CCF000CDE9004033461A463946284600F0C6FAC8
:10CD00002846BDE8FC8100002E2E5C4472697665E1
:10CD100072735C4C7749505C7372635C636F7265CD
:10CD20005C706275662E6300696E76616C69642062
:10CD3000706275665F7479706500000070B50D46AD
:10CD400000B125B9BDE8704011A0F3F77DBB0446E2
:10CD5000006820B121892A8911442181F7E72089BF
:10CD6000618988420DD04FF4597217A11EA0FEF7B9
:10CD70004DF8206828B140F2653213A126A0FEF7D5
:10CD800045F82089298908442081256070BD00006C
:10CD9000286820213D204E554C4C2920262620284D
:10CDA0007420213D204E554C4C29202870726F670D
:10CDB00072616D6D65722076696F6C617465732048
:10CDC00041504929000000002E2E5C4472697665AE
:10CDD00072735C4C7749505C7372635C636F72650D
:10CDE0005C706275662E6300702D3E746F745F6CAC
:10CDF000656E203D3D20702D3E6C656E20286F666F
:10CE0000206C617374207062756620696E2063689F
:10CE100061696E2900000000702D3E6E65787420F7
:10CE20003D3D204E554C4C0010B50C46FFF786FF9B
:10CE30002046BDE8104000F0C5BA002102E0491CC0
:10CE4000006889B20028FAD10846704770B51546C7
:10CE500013890A461946FFF741FE04000BD0294604
:10CE600000F026F828B140F2435204A10BA0FDF7D0
:10CE7000CDFF204670BD002070BD00002E2E5C440A
:10CE80007269766572735C4C7749505C7372635C4F
:10CE9000636F72655C706275662E630070627566A2
:10CEA0005F636F7079206661696C656400000000E3
:10CEB00010B529B10A89BDE81040002300F06EB812
:10CEC00002A0F3F7C1FA6FF00F0010BD7062756633
:10CED0005F636F70793A20696E76616C6964207364
:10CEE0006F757263650000002DE9F0470027164654
:10CEF0008946B84620B1B9F1000F03D0044625E0B9
:10CF000015A000E01CA0F3F79FFA0020BDE8F08711
:10CF10002BB16089984202D8181A83B215E0608953
:10CF2000C01A85B2B54200D9354660682A46C11894
:10CF300009EB0700F3F7C7FD08EB05001FFA80F8BF
:10CF4000781987B2701B86B2002324680EB1002CBA
:10CF5000DED14046DAE70000706275665F636F708D
:10CF6000795F7061727469616C3A20696E76616C88
:10CF70006964206275660000706275665F636F7039
:10CF8000795F7061727469616C3A20696E76616C68
:10CF90006964206461746170747200002DE9F05F4F
:10CFA00090460C0005461E464FF000076FF00F0A32
:10CFB00002D02189414501D233A049E025B1298918
:10CFC00006EB0800814201D23CA041E06FF0050B66
:10CFD0006889811B6089C01B814200D20846414696
:10CFE000804500D20846814660684A46C119686893
:10CFF0003044F3F768FDA8EB09001FFA80F8688950
:10D000004E444F44B04205D240F2F73237A13FA020
:10D01000FDF7FCFE6089B84205D24FF47E7233A161
:10D0200040A0FDF7F3FE6089B84207D824680027C6
:10D0300024B9B8F1000F01D041A009E06889B042DD
:10D040000BD12D68002645B9B8F1000F05D040A0DE
:10D05000F3F7FAF95046BDE8F09F2CB160892189B9
:10D06000884201D1206830B955B168892989884240
:10D0700006D1286820B13AA0F3F7E6F95846EAE766
:10D080005FEA0800A4D1E6E7706275665F636F70BF
:10D09000795F7061727469616C5F706275663A2065
:10D0A000636F70795F6C656E206269676765722077
:10D0B0007468616E20736F75726365007062756667
:10D0C0005F636F70795F7061727469616C5F7062C9
:10D0D00075663A20746172676574206E6F742062A1
:10D0E000696720656E6F7567680000002E2E5C44CE
:10D0F0007269766572735C4C7749505C7372635CDD
:10D10000636F72655C706275662E63006F6666732E
:10D1100065745F746F203C3D20705F746F2D3E6CB2
:10D12000656E00006F66667365745F66726F6D2072
:10D130003C3D20705F66726F6D2D3E6C656E000029
:10D14000705F66726F6D20213D204E554C4C000083
:10D15000705F746F20213D204E554C4C0000000044
:10D16000706275665F636F70795F70617274696118
:10D170006C5F70627566282920646F6573206E6F1E
:10D180007420616C6C6F77207061636B65742071C3
:10D1900075657565732100002DE9F041040007D025
:10D1A0005FF0000501F063FC0746A07B48B10EE08C
:10D1B00040F2DE221AA122A0FDF728FE0020BDE8E1
:10D1C000F08140F2F32216A120A0FDF71FFEA07B04
:10D1D000401EC6B2A673384601F06BFC96B9207BA0
:10D1E000266800F00F0002280ED001280FD098B159
:10D1F00040F211320AA11BA0FDF708FE6D1CEDB232
:10D200003400CFD12846DAE721460A2001E0214642
:10D210000920FEF7C9F9F1E72046FDF7D9FEEDE751
:10D220002E2E5C447269766572735C4C7749505C53
:10D230007372635C636F72655C706275662E630007
:10D240007020213D204E554C4C00000070627566E8
:10D250005F667265653A20702D3E726566203E20DD
:10D2600030000000696E76616C69642070627566DA
:10D2700020747970650000000122AFF3008000295E
:10D2800002DA494200F0CEB8FFF7E8BB70B50024DF
:10D29000DDE90456C0E9004102814381057346730C
:10D2A00001218173C47370BD2DE9F0410D46040066
:10D2B00005D14FF4CC7221A128A0FDF7A7FD20894C
:10D2C000A84238D9401B86B240F2AF170BE0281AAB
:10D2D00085B22089801B2081246824B93A4617A191
:10D2E00024A0FDF793FD6089A842F0D3207B0007BE
:10D2F00019D16089A84216D0A088001B284481B2A9
:10D300002046FEF781F8060005D140F2BD120BA1C0
:10D310001EA0FDF77BFDA64205D040F2BF1207A17B
:10D3200021A0FDF773FD65812581206808B1FFF715
:10D3300033FF00202060BDE8F08100002E2E5C4409
:10D340007269766572735C4C7749505C7372635C8A
:10D35000636F72655C706275662E630070627566DD
:10D360005F7265616C6C6F633A207020213D204EC6
:10D37000554C4C00706275665F7265616C6C6F63D2
:10D380003A207120213D204E554C4C006D656D5F5B
:10D390007472696D2072657475726E656420722096
:10D3A0003D3D204E554C4C006D656D5F7472696D4E
:10D3B0002072657475726E6564207220213D207143
:10D3C0000000000010B5040011D001F050FBA17B5B
:10D3D000491CA17301F06DFBA07B002807D1BDE8BB
:10D3E00010404FF4517202A109A0FDF70FBD10BD0E
:10D3F0002E2E5C447269766572735C4C7749505C82
:10D400007372635C636F72655C706275662E630035
:10D410007062756620726566206F766572666C6FE5
:10D420007700000010B520B1B1F5803F08D301208E
:10D4300010BD40F24E220CA113A0FDF7E7FCF6E769
:10D4400039B143898AB2934205D212A0F2F7FCFFA8
:10D45000EDE7002010BD446821444160991A4181E4
:10D460000189891A0181F4E72E2E5C447269766580
:10D4700072735C4C7749505C7372635C636F726566
:10D480005C706275662E63007020213D204E554C05
:10D490004C000000696E6372656D656E745F6D614E
:10D4A000676E6974756465203C3D20702D3E6C6527
:10D4B0006E00000070B5044600680025406828B181
:10D4C0004FF41A7215A11EA0FDF7A0FC2068007889
:10D4D00000F0F00010280FD0402801D0FA201AE008
:10D4E000217A284600F0A0FF21684860226888B1B0
:10D4F0001B4900F09CFF09E0284603F043FC21682B
:10D500004860216830B1084601F050FA2068406850
:10D51000002801D1FF20207170BD00002E2E5C4438
:10D520007269766572735C4C7749505C7372635CA8
:10D530006170695C6170695F6D73672E63000000E4
:10D540007063625F6E65773A2070636220616C720F
:10D550006561647920616C6C6F636174656400005F
:10D5600065E400082DE9F0412E4D04462868844208
:10D5700005D240F2DF122CA133A0FDF747FC68680A
:10D58000844205D34FF4F07227A135A0FDF73EFC8D
:10D59000207928B140F2E11223A138A0FDF736FC32
:10D5A00020884FF4E058404505D94FF4F2721EA18F
:10D5B00039A0FDF72BFC208800F0B8FD0646B442E8
:10D5C00015D0307998B96868864210D0E868B042C2
:10D5D00000D1EC60308820803088404507D020465C
:10D5E000FDF70AFF0746308800F0A0FD47806088FD
:10D5F00000F09CFDA04212D0017900290FD1E9680A
:10D60000A14200D1E860218801802188414506D0EF
:10D61000FDF7F2FE0546208800F088FD4580BDE854
:10D62000F0810000F80000202E2E5C4472697665BF
:10D6300072735C4C7749505C7372635C636F7265A4
:10D640005C6D656D2E630000706C75675F686F6C54
:10D6500065733A206D656D203E3D2072616D00005E
:10D66000706C75675F686F6C65733A206D656D20CF
:10D670003C2072616D5F656E64000000706C7567C0
:10D680005F686F6C65733A206D656D2D3E757365CF
:10D6900064203D3D20300000706C75675F686F6CE2
:10D6A00065733A206D656D2D3E6E657874203C3D46
:10D6B000204D454D5F53495A455F414C49474E45C2
:10D6C0004400000010B5040005D140F26D1217A10E
:10D6D0001FA0FDF79BFB6078012802D0042805D02D
:10D6E00008E001212046FDF7C1F803E001212046B2
:10D6F000FCF74CFC94F82010C80614D5606890B173
:10D70000B0F86420B2F5866F0DD3B0F86600052836
:10D7100009D201F0EF0084F82000A36A1BB10022B7
:10D72000022120469847002010BD00002E2E5C44A8
:10D730007269766572735C4C7749505C7372635C96
:10D740006170695C6170695F6D73672E63000000D2
:10D75000636F6E6E20213D204E554C4C0000000042
:10D76000C521484370B5174901EB80000168C96BBA
:10D7700009684968C1F1800189B2802900D300217C
:10D78000021D00F5827400BFB0F804338B4217D03D
:10D79000B0F80633B0F808535B1CDBB29D420FD0E3
:10D7A000B0F80453B0F80663AD5C3555A0F8063305
:10D7B000B0F804335B1C03F07F03A0F80433E3E705
:10D7C00070BD000048C800202DE9F041134C0F4601
:10D7D0000546E6682068001D07F050FA681C07D16E
:10D7E00037B12168BDE8F0410D48091D07F02ABB9B
:10D7F00020683544B5424560216805D2A06BBDE87C
:10D80000F041091D07F006BB606B091D07F002FB24
:10D81000A06A854200D2A562BDE8F08178000020B0
:10D82000F40500202DE9F041054607F017FB2E4CCA
:10D83000A068401CA06020682C4F10B1606940B304
:10D840002DE02560A068012829D1002606EB86007E
:10D8500007EB800007F0D0FA761C072EF6D323489A
:10D860008C3007F0C9FA2148A03007F0C5FA1F48EC
:10D87000B43007F0C1FA1D48C83007F0BDFA1B48A4
:10D88000DC3007F0B9FA19488C3060631430A063BB
:10D8900005E02068E96AC06A884200D82560606AAD
:10D8A000401C60626864E86A2169884200D920618E
:10D8B00000EB800007EB8000291D07F0C3FA07F09A
:10D8C000FDFA606900280CD02068E96AC06A8842C5
:10D8D00007D207494FF080500860BFF34F8FBFF366
:10D8E0006F8FBDE8F081000078000020180500204F
:10D8F00004ED00E038B507F0B1FA104C2068C8B963
:10D900000F4807F079FA0E48143007F075FA0C4802
:10D91000E060143020610A4B0020F03B009003F1DE
:10D92000500210210A2008F09BF8206010B105A1D8
:10D9300007F082FBBDE8384007F0C0BAB400002011
:10D94000F8060020546D72510000000030B4026CE3
:10D950000B46002A0BD0C1681144C1608468A14203
:10D9600001D30168C16030BC1846F3F7ACB830BCD5
:10D9700070472DE9F041856B174604460026026C7E
:10D9800082B1C7B1E068F3F79EF8E168206C091A2C
:10D99000E1602268914202D2A168081AE060022F79
:10D9A00016D017E02068A8B9A06809F01FF806464D
:10D9B0000020A0600EE06068F3F785F8216C6068D5
:10D9C00008446060A168884204D32068606001E078
:10D9D00005B16D1E6D1CA5633046BDE8F0810000E9
:10D9E00010B5044690F85D0088B1012812D00228D5
:10D9F00015D040F65D720AA116A0F9F7D3FF5020AA
:10DA000080F31188BFF34F8FBFF36F8FFEE7206B5A
:10DA100007F078FA2046BDE8104007F073BA10BD51
:10DA20002E2E2F4D6964646C6577617265732F5477
:10DA3000686972645F50617274792F4672656552CD
:10DA4000544F532F536F757263652F7461736B73EB
:10DA50002E630000636F6E6669672D617373657274
:10DA60007400000010484FF4AA41420706D0C01DC0
:10DA70000D4920F00700411AC1F5AA410B4A0023C5
:10DA80000144C2E900030839183A21F00701116086
:10DA90004B600B600B1AC0E9001393604FF000401D
:10DAA0005360506170470000E00D0020E40000204A
:10DAB000154E164CA6F1C8074FF08058DFF850906D
:10DAC00012E000BF07F0CAF9F068C568281D07F02A
:10DAD000D5F8A068401EA0606068401E606007F036
:10DAE000EDF92846FFF77CFF60680028EAD1386826
:10DAF000012805D9C9F80080BFF34F8FBFF36F8F9E
:10DB000007F028F9F0E70000E00500207800002089
:10DB100004ED00E0002807D00021816001600B4681
:10DB20000A46C16008F078B87047000070B51D461D
:10DB3000049C51B1C4F80020C4E90F010121204622
:10DB400007F0FEFF84F84C5070BD2460F4E700003D
:10DB50002DE9F05F8846DDE90B9415468346910078
:10DB60009A460A9EA522206BF2F7F2FF6FF003019E
:10DB7000206B01EB8501084420F0070778070DD0E2
:10DB80004FF4597222A12FA0F9F70CFF502080F317
:10DB90001188BFF34F8FBFF36F8FFEE70025B8F1F9
:10DBA000000F0FD05FF00000221818F8001082F864
:10DBB000341018F8001011B1401C1028F4D384F868
:10DBC000435001E084F83450072E00D30626E66265
:10DBD000C4E91365201D07F01AF904F1180007F0D5
:10DBE00016F92461C6F107006462A0616565A56548
:10DBF00084F85C5052465946384600F045FB206098
:10DC0000B9F1000F01D0C9F80040BDE8F09F000055
:10DC10002E2E2F4D6964646C6577617265732F5485
:10DC2000686972645F50617274792F4672656552DB
:10DC3000544F532F536F757263652F7461736B73F9
:10DC40002E630000636F6E6669672D617373657282
:10DC50007400000030B5114900E011460A688242A4
:10DC6000FBD34B685C18844203D140681844486079
:10DC7000084643681C18944209D1084C183C246893
:10DC8000A24209D052681A4442600A6812680260CF
:10DC9000814200D0086030BD0460F9E7E400002054
:10DCA00070B5002441600B4D0061914206D8D11A35
:10DCB0008269914206D2011D286907E09A4203D287
:10DCC000994201D3012403E0011DE86807F0A2F89E
:10DCD000204670BDB400002010B5044607F0BEF821
:10DCE000A06B28B15FF0000407F0E8F8204610BDF3
:10DCF0000124F9E7F8B505461A480E46C068C06821
:10DD0000C468201D06F0BAFF94F8280041071FD50B
:10DD1000A0692B46411932462046FFF7C1FFD8B112
:10DD200000200346014600902A46204609F048F8A4
:10DD300090B90D4940F2112201F13400F9F732FE99
:10DD4000502080F31188BFF34F8FBFF36F8FFEE732
:10DD500020F0010084F82800216A01B02046BDE8C7
:10DD6000F0400847B4000020F8DF000830B589B063
:10DD7000444D7CE00498002806DADDE90601059AA6
:10DD800090470498002872DB069C606910B1201D42
:10DD900006F074FF03A800F0DFF8024604980A2892
:10DDA00065D2DFE800F0050505353B580505353B34
:10DDB00094F8280040F0010084F828000599A06933
:10DDC000059B01442046FFF76BFF00284FD0216AD6
:10DDD0002046884794F82800400748D50020009046
:10DDE0000598A169002342181946204608F0E8FF6B
:10DDF00000283CD14FF44B7223A130A0F9F7D2FD9B
:10DE0000502080F31188BFF34F8FBFF36F8FFEE771
:10DE100014F8280F20F00100207028E094F8280062
:10DE200040F0010084F828000598A06128B181180D
:10DE300013462046FFF734FF19E04FF4517212A148
:10DE40001EA0F9F7AFFD502080F31188BFF34F8F6C
:10DE5000BFF36F8FFEE794F82800810703D42046B4
:10DE600007F050F803E020F0010084F828000022B9
:10DE700004A9286808F01AF900287FF47BAF09B0DC
:10DE800030BD0000B40000202E2E2F4D6964646C5C
:10DE90006577617265732F54686972645F5061724F
:10DEA00074792F4672656552544F532F536F7572B4
:10DEB00063652F74696D6572732E6300636F6E66A0
:10DEC00069672D617373657274000000F8B50D46C3
:10DED000064607F021FC684600F03EF8044600982C
:10DEE00010B108F08BFEF8BD1148ADB101690968A9
:10DEF000D9B10025311B2A46006807F005F908F062
:10DF00007DFE0028EFD10B494FF080500860BFF331
:10DF10004F8FBFF36F8FF8BDA642EBD808F06EFEAF
:10DF200021463046FFF7E6FEF8BD0125E2E7000096
:10DF3000B400002004ED00E00648416B096829B1F7
:10DF4000416BC968C9684968816270474FF0FF3109
:10DF5000FAE700007800002070B5054608F06EFC76
:10DF6000064E0446B068844203D200F009F801204E
:10DF700000E0002028602046B46070BDB40000209E
:10DF8000F8B51C4D20E0C068C4680668201D06F086
:10DF900075FE216A2046884794F82800400713D56B
:10DFA000A0693044B04206D924616060211DE86850
:10DFB00006F030FF08E0002003460146009032469C
:10DFC000204608F0FDFE38B1E86801680029DAD182
:10DFD0002969C5E90310F8BD40F29D3206A113A0DE
:10DFE000F9F7E0FC502080F31188BFF34F8FBFF3A7
:10DFF0006F8FFEE7B40000202E2E2F4D6964646CF5
:10E000006577617265732F54686972645F506172DD
:10E0100074792F4672656552544F532F536F757242
:10E0200063652F74696D6572732E6300636F6E662E
:10E0300069672D617373657274000000002101E04F
:10E04000401C491C0278A52AFAD0C1F38F00704702
:10E050000C484068401C0CD0CA220B490BA0F9F7B1
:10E06000A1FC502080F31188BFF34F8FBFF36F8F57
:10E07000FEE7502080F31188BFF34F8FBFF36F8FFF
:10E08000FEE70000EC00002068720108636F6E6616
:10E0900069672D617373657274000000074CE06856
:10E0A000016841B1C0680021D0F80000FFF70EFF01
:10E0B000FFF75CFEF3E701210020F7E7B400002042
:10E0C0002DE9F041044606F0C9FE94F9455004F1EB
:10E0D000240609E0606A48B1304608F031FD08B115
:10E0E00007F0FAF86D1E6DB2002DF3DC4FF0FF362D
:10E0F00084F8456006F0E2FE06F0B0FE94F9445064
:10E1000004F1100709E0206948B1384608F018FD0D
:10E1100008B107F0E1F86D1E6DB2002DF3DC84F854
:10E120004460BDE8F04106F0C9BE0000014909683D
:10E1300008447047F80000202DE9F041054600270B
:10E1400007F0EAFA3D4E306808B9FFF78BFC7069BA
:10E1500005421BD1D5B10835680713D005F007007B
:10E16000C0F10800054468070CD09722344935A057
:10E17000F9F718FC502080F31188BFF34F8FBFF3DD
:10E180006F8FFEE715B17068854202D908F036FD41
:10E190003EE02A48183001460C6801E020460C4653
:10E1A0006168A94202D221680029F7D131688C4206
:10E1B000ECD007682168016060680837411B1029AE
:10E1C00013D9601942070CD0C4221D491DA0F9F7CC
:10E1D000E9FB502080F31188BFF34F8FBFF36F8F9F
:10E1E000FEE741606560FFF735FD61687068401AC1
:10E1F0007060B268904200D2B06070690143002044
:10E20000C4E90001F068401CF06008F0F7FC0FB9A9
:10E2100006F0A2FD78070DD040F20512084909A0CA
:10E22000F9F7C0FB502080F31188BFF34F8FBFF385
:10E230006F8FFEE73846BDE8F0810000CC0000207B
:10E2400020720108636F6E6669672D617373657272
:10E250007400000002460020012905DA0AB90348CB
:10E26000026802EB8100406D7047000078000020DA
:10E270000449086818B10868026D521C02650868F4
:10E28000704700007800002010B5031F4FF0807425
:10E290001C601B1F21F001011960191F024B0B604C
:10E2A000143940380A6010BD51E0000820B119B19E
:10E2B00009680160002070476FF00500704740B1A9
:10E2C00039B109684160417C41F00101417400208D
:10E2D00070476FF0050070472DE9F84FDFF8BC80FC
:10E2E00082464FF0000BD8F80010D8F81400FBF766
:10E2F00004FA8146DAF80400294E0025477A34688A
:10E3000048E0207CB84243D1217A39B1D8F80420C2
:10E3100092F83020521CD2B2914239D1B9F1000F9B
:10E3200003D04CB1206838B132E02CB1206818B16C
:10E33000D8F8141088422BD1607CC00704D06168E3
:10E34000D8F81000814223D1D4F814C0BCF1000FDA
:10E350001ED0DAF80400114B00904FF0020B10337E
:10E3600052462146A069E04740B125B1E068E86027
:10E370003068E06034600120BDE8F88FDAF80410FE
:10E380000098814204D0C02206A10E48FCF73EFD51
:10E390002546E468002CB4D15846EDE7E062002041
:10E3A000400100202E2E5C447269766572735C4CCD
:10E3B0007749505C7372635C636F72655C726177FE
:10E3C0002E6300002C73010810B5002813D00268DA
:10E3D000002A10D000290ED00A68002A0BD0064A65
:10E3E000126806E013680468A34201D10B68136049
:10E3F000D268002AF6D110BD4001002070B5054654
:10E400000020FDF715F9040009D01C21F2F7CAFB22
:10E410002574FF20E07203480168E1600460204633
:10E4200070BD0000400100200846FFF7E7BFC0E9CB
:10E43000051270470A490A6882420AD1D2680A6006
:10E4400009E0D16821B1814202D1C168D16002E006
:10E450000A46002AF5D101460020FDF7A5B80000C4
:10E46000400100202DE9F0410F4604002CD014F1AA
:10E470000C0F29D0E06800B34FF420710020FEF7A4
:10E48000E5FC060020D00420FDF7D2F8050011D0ED
:10E490000F482E606E600069A860387CA8813689BC
:10E4A000294604F10C0000F04CFB38B12846FDF77A
:10E4B000CBF909E03046FEF76FFE05E0A36A1BB119
:10E4C00032460021204698470020BDE8F081000038
:10E4D000E06200202DE9F0411F4614460E0005467B
:10E4E00005D140F22F1222A12AA0FCF78FFC2DB9F2
:10E4F0004FF498721EA130A0FCF788FC2FB140F2B7
:10E5000031121BA134A0FCF781FC8DB16868B042C8
:10E5100005D04FF49C7216A135A0FCF777FC15F1DD
:10E520000C0F09D0E86838B17CB1214624890EE08F
:10E530006FF00500BDE8F081BCB12189304604F0E0
:10E5400001F82046FEF728FE0FE03149002405F1CE
:10E550000C0000F0F6FA10B14FF0FF30EAE7AB6ABA
:10E560001BB122460021284698470020E2E7000020
:10E570002E2E5C447269766572735C4C7749505CF0
:10E580007372635C6170695C6170695F6D73672E43
:10E5900063000000726563765F746370206D75734D
:10E5A0007420686176652061207063622061726703
:10E5B000756D656E74000000726563765F746370DC
:10E5C000206D757374206861766520616E206172BC
:10E5D00067756D656E74000065727220213D20457F
:10E5E00052525F4F4B20756E68616E646C656400BB
:10E5F000726563765F7463703A2072656376206635
:10E600006F722077726F6E67207063622100000066
:10E6100096700108884201D3401A01E0511A08445B
:10E6200080B2704770B5054608F008F94FEA00045B
:10E6300006F014FC00F070F8064606F03FFC0EB140
:10E64000304670BD3DB1012006F080FD08F0F6F8BF
:10E65000001BA842ECD3002070BD10B55020EFF392
:10E66000118480F31188BFF34F8FBFF36F8F00F0D9
:10E6700053F884F3118810BD10B504001AD006F0C9
:10E68000EDFB0D48002100BF01EB411200EB02122F
:10E69000A24208D101EB411100EB0110002280F8E9
:10E6A0000C22428002E0491C0829EDD3BDE810404D
:10E6B00006F004BC10BD0000C8B7002010B500284B
:10E6C0001ED05021EFF3118281F31188BFF34F8FD9
:10E6D000BFF36F8F0B4B002101EB411403EB0414CC
:10E6E000844208D101EB411103EB0111002081F8B4
:10E6F0000C02488002E0491C0829EDD382F31188FE
:10E7000010BD0000C8B700204FF484510148F2F753
:10E7100049BA0000C8B700200E49002000EB4012A3
:10E7200001EB021292F80C2222B1401C0828F5D30A
:10E730000020704700EB401001EB0010012280F830
:10E740000C2200F10C0181600021418001704170B8
:10E7500001717047C8B7002070B514460D46DDE959
:10E76000041220B119B112B1B2F5007F01D9012014
:10E7700070BD05704470037142808068F2F7A3F9A0
:10E78000002070BD2DE9FE4F9046DDE90C5489460E
:10E790001F468246224629460E9E00F07FF800283A
:10E7A00011D13046FFF73EFF029070B1CDE9005421
:10E7B0003B4642464946FFF7CFFF040007D0029888
:10E7C000FFF75AFF2046BDE8FE8F0220FBE700233B
:10E7D000324602A9504607F01FFA012804D00298D9
:10E7E000FFF74AFF0320EEE70020ECE72DE9FE4F9C
:10E7F0009046DDE90C5489461F468246224629464A
:10E800000E9E00F04BF8002811D13046FFF725FF8F
:10E81000029070B1CDE900543B4642464946FFF7AD
:10E820009BFF040007D00298FFF748FF2046BDE891
:10E83000FE8F0220FBE70023324602A9504607F074
:10E84000D5FA012804D00298FFF738FF0320EEE73D
:10E850000020ECE738B1012807D0022807D00328B0
:10E8600007D005A0704706A0704706A0704707A014
:10E87000704708A070470000756E6B6E6F776E0072
:10E880006F6B0000696E76616C696400706F6F6C0D
:10E8900000000000717565756500000020B119B1B8
:10E8A00012B1B2F5007F01D90120704700207047F6
:10E8B00070B51546040005D06078012809D00428F9
:10E8C0000CD00FE04FF4CB7213A11CA0FCF79EFA02
:10E8D0001FE001212046FBF7C9FF03E0012120468C
:10E8E000FBF754FB6068A0B1B0F86410B1F5866F17
:10E8F0000FD3B0F8660005280BD294F8200000F082
:10E90000EF0084F82000A36A1BB12A4602212046AA
:10E910009847002070BD00002E2E5C447269766519
:10E9200072735C4C7749505C7372635C6170695CB4
:10E930006170695F6D73672E63000000636F6E6EB8
:10E9400020213D204E554C4C0000000010B53021D8
:10E950001448F2F727F9134801231C38002100F866
:10E960001C3F41F69072417042800F4A1468446027
:10E970000173437341F69174C48114680461037692
:10E98000437642F2293343835468C4615C1E048495
:10E9900080F8241080F82510591CC1849168816288
:10E9A000838510BD48B00020C470010810B54468CC
:10E9B0000146204600F066FB0949204603F066FD4B
:10E9C0000849204604F0F4F802220749204602F0E4
:10E9D000EFFF2046BDE81040044901F067BA00008F
:10E9E000D5E40008B1E80008C5D60008597B000846
:10E9F00000E0401C01782029FBD00929F9D070479C
:10EA00002DE9F84316460C46804607F017FF0746E7
:10EA10004FF0FF358EB14FF47A704643B6FBF0F2FB
:10EA20006946D8F8000007F041FB012807D00CB177
:10EA3000002020602846BDE8F8832A46F0E70CB1A4
:10EA40000098206007F0FAFEC01BF4E738B50C46CA
:10EA500000680022694607F029FB012802D04FF028
:10EA6000FF3038BD0CB100982060002038BD10B5D3
:10EA700006F0F4F9002010BD2DE9F0410D460746DF
:10EA800007F0DCFE06464FF0FF3465B14FF47A70B4
:10EA90004543B5FBF0F1386807F0D8FB012804D0F6
:10EAA0002046BDE8F0812146F5E707F0C7FE801B50
:10EAB000F7E706F003BA00002DE9F04100F063F833
:10EAC0000D4C05464FF000472168002911D04868D9
:10EAD0002A1ABA420DD20A682260D1E90262606045
:10EAE00090460820FCF760FD002EEDD04046B04770
:10EAF000EAE7BDE8F081000088010020704710B50A
:10EB00000446006818B910BD012006F01FFB2068FC
:10EB100006F0C8F80028F7D1206806F0A1FA002016
:10EB2000206010BD10B50B46044600220421184693
:10EB300006F04CFF206008B1002010BD4FF0FF3000
:10EB400010BD13B5002300681A4601A907F064F848
:10EB5000012802D04FF0FF301CBD00201CBD006812
:10EB60004FF0FF3107F06ABC10B50446042006F0F0
:10EB700021FF206008B1002010BD4FF0FF3010BD14
:10EB8000006807F04BBA07F059BE10B5044600689C
:10EB9000002803D006F064FA0020206010BD10B5F4
:10EBA0000446FF2006F0BAFE206008B1002010BD28
:10EBB0004FF0FF3010BD002300681A46194607F0D9
:10EBC0002BB83EB500250C460295069902ADCDE95D
:10EBD000001599B213460A460146204607F0DEFCAE
:10EBE000012801D000203EBD02983EBD70B51546FB
:10EBF0000E460446B0F1804F05D340F2291206A11B
:10EC00000EA0FCF703F9FFF7BEFF20442A46314669
:10EC1000BDE8704000F02EB82E2E5C447269766517
:10EC200072735C4C7749505C7372635C636F72659E
:10EC30005C74696D656F7574732E630054696D65DE
:10EC40006F75742074696D6520746F6F206C6F6EC2
:10EC5000672C206D6178206973204C5749505F55AF
:10EC6000494E5433325F4D41582F34206D736563E4
:10EC70007300000070B5044615460E460820FCF7E8
:10EC8000D7FC78B10021C560104A80E852001168B5
:10EC900031B14B68E51A4FF000439D4211D301603A
:10ECA000106070BDBDE87040BE2209A111A0FCF744
:10ECB000ADB85568651B9D4202D30260086070BD07
:10ECC00011460A68002AF8D0F3E700008801002006
:10ECD0002E2E5C447269766572735C4C7749505C89
:10ECE0007372635C636F72655C74696D656F757474
:10ECF000732E63007379735F74696D656F75743A11
:10ED00002074696D656F757420213D204E554C4C03
:10ED10002C20706F6F6C204D454D505F5359535FE1
:10ED200054494D454F555420697320656D70747971
:10ED300000000000034A0449A2F108008068FFF7C0
:10ED400055BF000088700108E19D000810B5084C0F
:10ED5000206848B1FFF717FF21684968081AB0F129
:10ED6000004F00D3002010BD4FF0FF3010BD000059
:10ED7000880100202DE9FF5F8946040003D0207D33
:10ED8000012806D00BE004B037A0BDE8F05FF1F732
:10ED90005BBB4FF410723BA142A0FCF737F8207D1B
:10EDA0000A283DD0216D03910025DFF82C81D4F88D
:10EDB00024B0D4F810A0D4F88C602F4678B34D4618
:10EDC000E78A214608F1180002F060FD012188F869
:10EDD0000010206F08B103F040FEE06E08B103F0B0
:10EDE0003CFE204600F052F955B1208B211D0091C8
:10EDF000CDE9017023465A461846039903F08CFD6D
:10EE0000204601F0BDF8002E2CD004B05046B44688
:10EE1000BDE8F04F6FF00C015DF804EB60470AE0CD
:10EE20002D4821461C3002F031FD04B02046BDE8DB
:10EE3000F05F01F0A5B8E08A0028CAD0D8F8100029
:10EE4000A0420AD1C068C8F8100008E0C168A14219
:10EE500002D1E168C16002E008460028F6D1002036
:10EE6000E060B6E7BDE8FF9F7463705F6162616E4A
:10EE7000646F6E3A20696E76616C696420706362BB
:10EE8000000000002E2E5C447269766572735C4C43
:10EE90007749505C7372635C636F72655C74637016
:10EEA0002E630000646F6E27742063616C6C2074A5
:10EEB00063705F61626F72742F7463705F6162610F
:10EEC0006E646F6E20666F72206C697374656E2D50
:10EED0007063627300000000440100200121FFF70D
:10EEE00049BF002803D0027D012A00D1816170470B
:10EEF00010B50C0005D14FF4447205A10CA0FBF72E
:10EF000085FF2046FFF7EAFF6FF00C0010BD000000
:10EF10002E2E5C447269766572735C4C7749505C46
:10EF20007372635C636F72655C7463702E63000060
:10EF30007463705F6163636570745F6E756C6C3A67
:10EF400020696E76616C6964207063620000000065
:10EF50002DE9F04106460120FCF76AFB454D04000F
:10EF60005BD1A86909E0418BC4680A0704D521F088
:10EF70000801418300F096FC20460028F3D10022CE
:10EF80001146EC68E86906E0036AE31A934201D38C
:10EF90001A460146C0680028F6D111B10846FFF7AD
:10EFA0009DFF0120FCF744FB040036D1092001F04D
:10EFB00051FC0120FCF73CFB04002ED1082001F09D
:10EFC00049FC0120FCF734FB040026D17F2E01D937
:10EFD0007F2001E030001BD0401EC2B20023194642
:10EFE000EC68A8690EE0477D974206D309D1D0F8B6
:10EFF00020C0A4EB0C0C9C4503D3016A3A46631A6B
:10F000000146C0680028EED111B10846FFF766FF3F
:10F010000120FCF70DFB040028D0A021F1F7C2FD70
:10F0200066754FF48660A4F8640060852085FF2132
:10F03000E172411061860621A4F84010E187C91FE2
:10F0400021860121A4F84810E9682162A978A177F6
:10F05000A4F84A000848C4F880000848C4F89000A2
:10F060000748C4F894000920C4F898002046BDE879
:10F07000F081000044010020F524010800DD6D004E
:10F08000F8240100002800D00161704710B5040089
:10F0900005D140F23F120DA114A0FBF7B7FE608B23
:10F0A000800512D5A06F00280FD0407F28B940F20C
:10F0B000431206A110A0FBF7A9FEA16F487F401ED6
:10F0C0004877608B20F40070608310BD2E2E5C4466
:10F0D0007269766572735C4C7749505C7372635CDD
:10F0E000636F72655C7463702E63000070636220EE
:10F0F000213D204E554C4C00616363657074735F15
:10F1000070656E64696E6720213D2030000000004C
:10F1100010B5040005D14FF494720DA114A0FBF7B3
:10F1200075FE608B800512D4A06F00280FD0417F40
:10F13000491C11F0FF01417705D140F22D1204A1C5
:10F140000EA0FBF763FE608B40F40070608310BD7F
:10F150002E2E5C447269766572735C4C7749505C04
:10F160007372635C636F72655C7463702E6300001E
:10F1700070636220213D204E554C4C0061636365F5
:10F180007074735F70656E64696E6720213D203016
:10F19000000000002DE9F0410D0004464FF004038B
:10F1A00000D1294D44B1207D60B128A0F1F74CF980
:10F1B0006FF00500BDE8F0812EA0F1F745F96FF082
:10F1C0000F00F7E7667A700700D5032312B100211C
:10F1D0002E4F2AE001F0DAFD020028D1801EE9E777
:10F1E00057F8210000681DE0B0F816C0944518D10A
:10F1F0005FEA467C04D590F809C05FEA4C7C10D4E5
:10F2000060B1D0F800C0BCF1000F07D035B1D5F81F
:10F2100000E0BEF1000F01D0F44502D16FF007000D
:10F22000C8E7C0680028DFD1491C9942D8DB15B176
:10F23000286800B120601648E2820169E16004613B
:10F2400004F0E6F90020B5E7907001087463705F80
:10F2500062696E643A2063616E206F6E6C79206221
:10F26000696E6420696E20737461746520434C4F2D
:10F27000534544007463705F62696E643A20696E3E
:10F2800076616C6964207063620000007070010830
:10F290004401002070B504464FF47A760FE0322C1A
:10F2A00001D9322500E0254600F012F860B94FF48C
:10F2B0007A706843B0FBF6F005F048FF641B002C41
:10F2C000EDD100F005F808B1002070BD012070BD3F
:10F2D00010B5F6F78BFF002800D0012010BD00000C
:10F2E0002DE9F04786B00446FCF7AAFF022C0AD0AD
:10F2F0005FF000054FF4FA7804EB4406FFF7E8FFEF
:10F3000000287CD10AE00125F4E700BFFFF7E0FF09
:10F310000028F6D1642005F019FF00E05E4F386840
:10F320000028F3D0F9F78EFC0028EFD0F7F76CFC3B
:10F3300000EB8607397F11B1406D30B107E0FFF770
:10F34000C7FF0028DDD1404695E040F6B830814641
:10F3500025B1002551A0F8F768FB8BE0002211468B
:10F360001020FCF72DFD5FEA000AF6D0FA8B6AB197
:10F370005249FCF787FB020008D0FB8B214650A0C6
:10F38000F8F73CFB5046FCF7F9FB73E0388C41BAC8
:10F390000A0497F8221090FA90FC42EA012397F8A9
:10F3A00023204FEA0C4C13434CEA012C1B061FFA96
:10F3B0008CFC43EA0C2390FA90FC40BA000440EA2B
:10F3C00001200CF0FF0C43EA0C23104343EA1060C9
:10F3D0000490CAF81C80BA8C04A95046FCF7A4FB20
:10F3E00002002FD0D01C36D097F82100B7F824C0E7
:10F3F00097F8233097F822108DE80B1000E03FE0DB
:10F4000097F82030214639A0F8F7F8FADAF8040026
:10F41000574680B14448FFF7A2FB786840B1FFF738
:10F420005DFD002078607870214640A0F8F7E6FA8C
:10F430003D48FFF7A5FB3846FCF7A0FBFFF748FF68
:10F44000F0B917E0214640A0F8F7D8FA2146504617
:10F4500000F0A8F8DAE797F82100BB8C97F8232092
:10F4600097F822108DE80F0097F820304246214689
:10F470003CA0C9E74846FFF70DFF00287FF43EAFE8
:10F48000FCF7C0FE07F0C6F9F6F7C6FE002005F04F
:10F49000ABFE06B0BDE8F087380000205B434C4966
:10F4A0005D2043312066697273742D636F6E6E65E3
:10F4B00063742064656665720D0A0000907001082F
:10F4C0005B434C495D206964783D25752062696E17
:10F4D000642D6661696C206572723D2564206C70D4
:10F4E0006F72743D25750D0A000000005B434C49A6
:10F4F0005D206964783D257520636F6E6E65637469
:10F500002D6661696C206572723D25642072697098
:10F510003D25752E25752E25752E25752072706F4B
:10F5200072743D25750D0A00A40100205B434C490F
:10F530005D206964783D25752061626F72742D636A
:10F540006C6F73650D0A00005B434C495D20696474
:10F55000783D257520636F6E6E6563742D6F6B0D3E
:10F560000A0000005B434C495D206964783D2575C5
:10F5700020636F6E6E6563742D74696D656F75744D
:10F58000206D733D2575207269703D25752E25759A
:10F590002E25752E25752072706F72743D25750DA0
:10F5A0000A0000002DE9F04F89B00C468146F7F7BC
:10F5B0002BFB04EB440100EB8100407FF8F7A0F93E
:10F5C00005902046F7F75AFB0A2580466FF00E0B90
:10F5D000C9F81C50FFF77CFE48B907A94846FCF75C
:10F5E0007DFC40B1C11C03D1FFF772FE78B35846D1
:10F5F00009B0BDE8F08F274E03AA06A90798FCF7CB
:10F60000DBF8BDF80C000699CDE900100295022C3C
:10F6100013D006234146059A3068FFF7B3F870B15E
:10F62000FFF718F90246BDF80C3021461AA0F8F78A
:10F63000E5F90798FCF708F9D9E70523EAE7079801
:10F64000FCF714F90028D7DA0798FCF7FDF81D4FEE
:10F650004FF0000A002257F8240008A906F026FD02
:10F660000128B7D1FFF734FE18B10898FFF704F866
:10F67000BDE70898CDF800A001234288816848467C
:10F68000FCF738FE06460898FEF7F6FF002EE1D09C
:10F690003046ADE7000000205B434C495D206964C3
:10F6A000783D25752072782D726F7574652D6661B1
:10F6B000696C2072633D2573206C656E3D25750D68
:10F6C0000A000000D001002010B558B1017D0129C9
:10F6D00003D0418B41F010014183BDE8104001216E
:10F6E00000F012B802A0F0F7AFFE6FF00F0010BDEF
:10F6F0007463705F636C6F73653A20696E76616CDA
:10F700006964207063620000FEB50D46040005D1F7
:10F710004FF4AF7242A14AA0FBF778FB2800504D8E
:10F720004FF000064FF001073DD0207D042801D0A6
:10F73000072838D1606F18B9208DB0F5866F32D0A8
:10F74000A07EC00605D44FF4B27235A145A0FBF7E8
:10F750005DFB228BE18A201D8DE8070023461846B9
:10F76000626A216D03F0D8F8204602F05BF8A869C0
:10F77000A04209D1C068A86108E0C168A14202D1D5
:10F78000E168C16002E008460028F6D13C48E66026
:10F790002F700068A04202D103F0C4FF36E020467B
:10F7A00000F0EEFB32E0207D40B101281AD00228A3
:10F7B0002ED02046BDE8FE4000F074B8E08A002854
:10F7C000EDD02869A04209D1C068286108E0C1686D
:10F7D000A14202D1E168C16002E008460028F6D1EA
:10F7E000E660DCE7204601F075F81D48214614303C
:10F7F00002F04CF8207D012804D1DF22214922A00B
:10F80000FBF704FB21460220FBF7CEFE0020FEBDE5
:10F8100013482146183002F039F82F70BFE7000076
:10F820002E2E5C447269766572735C4C7749505C2D
:10F830007372635C636F72655C7463702E63000047
:10F840007463705F636C6F73655F73687574646F06
:10F85000776E3A20696E76616C696420706362002D
:10F86000440100207063622D3E666C616773202640
:10F870002054465F5258434C4F534544000000000B
:10F8800084010020A0FF00087463705F66726565E4
:10F890005F6C697374656E3A20214C495354454E30
:10F8A0000000000070B5050005D14FF4CE7219A11B
:10F8B00020A0FBF7ABFA287D0526032804D00428F6
:10F8C0000BD007281FD10FE0284603F027F90400CA
:10F8D0000FD12846FFF7DAFB04E0284603F01EF9B3
:10F8E000040006D12E7509E0284603F017F904003C
:10F8F00002D0601C09D004E009202875284601F0D8
:10F90000A3FA204670BD002070BD688B40F008004F
:10F910006883F8E72E2E5C447269766572735C4CDE
:10F920007749505C7372635C636F72655C7463707B
:10F930002E63000070636220213D204E554C4C0028
:10F940002DE9F0479A4690460F4604006FF00F05E8
:10F9500008D04FB1207D60B14DA0F0F775FDA81D16
:10F96000BDE8F08756A000E05CA0F0F76DFD2846EA
:10F97000F6E738686060A4F81880207A10B1FCF7C8
:10F980009BFE02E0201DFAF75FF805006FF003010F
:10F9900010D0206818B9281D0CD000682060E68AB5
:10F9A00056B1607A40072AD5534A022152F8210005
:10F9B00000681FE00846D3E701F0E8F9E082F0B9FB
:10F9C0006FF00100CCE700BFB0F816C0B44510D10D
:10F9D000B0F818C0C4450CD10368D4F800C0634522
:10F9E00007D14368D7F800C0634502D16FF0070024
:10F9F000B6E7C0680028E7D1491C0429D6DB2046B9
:10FA000001F0F4F94FF00008C4F824802065401E8E
:10FA10006064A065E0654FF4866060852085C4F869
:10FA20002C80A4F8600040106086221D294600F05A
:10FA300009F960864FF00109A4F848900221204698
:10FA4000C4F884A000F03CF907001ED102202B4D21
:10FA5000207586B12869A04209D1C068286108E0F4
:10FA6000C168A14202D1E168C16002E008460028F5
:10FA7000F6D1C4F80C80A869E060AC6103F0C8FD61
:10FA800085F80090204601F0DFF9384668E700006D
:10FA90007463705F636F6E6E6563743A2063616E4A
:10FAA000206F6E6C7920636F6E6E65637420667272
:10FAB0006F6D20737461746520434C4F534544004F
:10FAC0007463705F636F6E6E6563743A20696E76FF
:10FAD000616C696420706362000000007463705F91
:10FAE000636F6E6E6563743A20696E76616C6964EB
:10FAF0002069706164647200707001084401002024
:10FB00002DE9F0479A46DDF8208091460D46070022
:10FB100004D1A6222BA134A0FBF778F925B9A7229E
:10FB200028A139A0FBF772F95FEAC87001D004265A
:10FB300000E000260320FBF77BFD04001DD084F8C5
:10FB40000C804FF00008C4E900852889B04204D237
:10FB5000B3221CA135A0FBF759F928891421801B79
:10FB60002081A4F80A802846FCF775FF48B120469A
:10FB700002F065FF0020BDE8F0872846FDF70CFB8A
:10FB8000F8E7606840682061F88AFAF749F9216966
:10FB90000880388BFAF744F9216948805046FAF713
:10FBA0003DF921694860B008000300F5A04040EA33
:10FBB0000900FAF735F92169888121692046A1F801
:10FBC0001280D8E72E2E5C447269766572735C4CA5
:10FBD0007749505C7372635C636F72655C746370C9
:10FBE0005F6F75742E6300007463705F637265618C
:10FBF00074655F7365676D656E743A20696E7661D2
:10FC00006C696420706362007463705F6372656125
:10FC100074655F7365676D656E743A20696E7661B1
:10FC20006C6964207062756600000000702D3E747F
:10FC30006F745F6C656E203E3D206F70746C656EF6
:10FC40000000000070B50C4605462AB940F6CF0208
:10FC500009A111A0FBF7DAF85CB1A18C49B1282900
:10FC600002D928398CB200E00024A54200D22C46EB
:10FC70002546284670BD00002E2E5C4472697665CC
:10FC800072735C4C7749505C7372635C636F72652E
:10FC90005C7463702E6300007463705F6566665FFA
:10FCA00073656E645F6D73735F6E657469663A2029
:10FCB000696E76616C6964206473745F69700000BA
:10FCC0002DE9F843044600250E46880705D140F289
:10FCD00013423AA14248FBF799F82CB940F2154279
:10FCE00036A140A0FBF792F8B00700D50125E80740
:10FCF00000D00420804601464FF420723620FCF7E5
:10FD0000EDFE07004FF0FF3925D07989414505D236
:10FD100040F23D4229A13BA0FBF778F8009532461E
:10FD200039462046E36DFFF7EBFE050013D0287C33
:10FD3000800705D040F2464220A141A0FBF766F8BB
:10FD4000288928B140F247421CA143A0FBF75EF886
:10FD5000E06E38B109E0608B40F080006083484677
:10FD6000BDE8F883E56604E0084601680029FBD198
:10FD700005600020A4F86800B00702D0E06D401CC8
:10FD8000E065F00703D0608B40F020006083686876
:10FD9000FDF753F8B4F8661008440004000CA4F80A
:10FDA000660009D0206F38B9E06E28B940F2694288
:10FDB00002A134A0FBF72AF80020D1E72E2E5C44E4
:10FDC0007269766572735C4C7749505C7372635CE0
:10FDD000636F72655C7463705F6F75742E6300008F
:10FDE000E87301087463705F656E71756575655FB2
:10FDF000666C6167733A20696E76616C6964207025
:10FE0000636200007463705F656E71756575655F30
:10FE1000666C6167733A20636865636B2074686120
:10FE20007420666972737420706275662063616EF7
:10FE300020686F6C64206F70746C656E0000000049
:10FE40007365672D3E746370686472206E6F7420F2
:10FE5000616C69676E6564007463705F656E71756F
:10FE60006575655F666C6167733A20696E76616C73
:10FE70006964207365676D656E74206C656E677468
:10FE8000680000007463705F656E71756575655F0D
:10FE9000666C6167733A20696E76616C6964207183
:10FEA00075657565206C656E6774680070B50D4684
:10FEB00004000AD0207D012805D140F6160203A1D6
:10FEC0000AA0FAF7A3FFC4F88C5070BD2E2E5C4434
:10FED0007269766572735C4C7749505C7372635CCF
:10FEE000636F72655C7463702E630000696E766187
:10FEF0006C696420736F636B6574207374617465DF
:10FF000020666F72206572722063616C6C6261633F
:10FF10006B00000070B5194DA878401CA870AC6942
:10FF200028E0A17FA878814223D0A077608BC10709
:10FF300009D040F002006083204600F085FF608B0E
:10FF400020F00300608380B2010705D520F008008F
:10FF500060832046FFF7A6FCE668606F38B100209A
:10FF60002870204601F0ACFF28780028D7D134460D
:10FF700000E0E468002CD4D170BD000044010020F2
:10FF800010B50446007D012804D1D42204A10CA0A0
:10FF9000FAF73CFF2146BDE810400120FBF704BB07
:10FFA0002E2E5C447269766572735C4C7749505CA6
:10FFB0007372635C636F72655C7463702E630000C0
:10FFC0007463705F667265653A204C495354454EC0
:10FFD000000000002DE9F04799460C460646204FE8
:10FFE00027E02546D5E90040FCF727FFB6F8661064
:10FFF0008046414505D240F264421AA122A0FAF798
:020000040801F1
:1000000005FF36F8661FA1EB080030802889398982
:1000100008443881284602F012FD36F8660940B1DE
:1000200054EA090005D140F26E420EA120A0FAF771
:10003000EDFE8CB120694068F9F7F0FE05462069B5
:100040008089F9F7EDFE800700D00120218928443E
:100050000844B969081AC4D52046BDE8F0870000F5
:10006000640100202E2E5C447269766572735C4CCC
:100070007749505C7372635C636F72655C74637024
:100080005F696E2E630000007063622D3E736E64C4
:100090005F71756575656C656E203E3D207062759B
:1000A000665F636C656E286E6578742D3E702900FE
:1000B0007463705F726563656976653A2076616C1A
:1000C0006964207175657565206C656E677468007C
:1000D0000849C888421CCA800A6912B18B889842B4
:1000E00003D2C9681431085C7047C01AC0B2105CF2
:1000F000704700006401002010B5F0F733F90349A0
:10010000C0F30D0000F54040888010BD4401002080
:100110002DE9FF5F4FF000090500C84604D1832296
:10012000ECA1F5A0FAF772FEF94E6868F0606889F4
:1001300014287DD3F74C21686069F9F7DEFA0028AE
:1001400076D1207DA246C0F303100E2870D004F1B2
:10015000140003900090031F2A890621284601936A
:10016000F9F7A2FC0028EBD1F0688089F9F758FE76
:10017000000B81001429DCD328898842D9D3A1F14E
:10018000140080B27080002232616A898A4204D3EE
:10019000B0802846FDF746F92FE0286820B9C22232
:1001A000CCA1DDA0FAF732FE14212846FDF73AF97A
:1001B0006989B1807088401A84B22846FDF732F907
:1001C00028684189A142B4D3416831612146FDF7D5
:1001D00029F92889001B2881688920B1DF22BDA167
:1001E000D1A0FAF713FE296828890989884204D02A
:1001F000E022B8A1CFA0FAF709FEF0680088F9F76D
:100200000FFE0146F06801804088F9F709FE0146BB
:10021000F06841804068F9F701FE0146F0684160EE
:1002200071618068F9F7FAFD0146F068816000E0CD
:1002300093E0B161C089F9F7F3FD0146F068C1812F
:100240008089F9F7EDFD00F03F0131702889708158
:10025000890704D0411C89B2718188427DD8DFF8BA
:10026000F4B20027DBF800407BE0207D20B9FB22C0
:1002700098A1B9A0FAF7CAFD207D0A2804D1FC2272
:1002800094A1BFA0FAF7C2FD207D012804D1FD2270
:1002900090A1C6A0FAF7BAFD207A38B1DAF80410B6
:1002A00091F83010491CC9B2884258D1F068228BAD
:1002B00001888A4253D1E18A408881424FD16168E6
:1002C000DAF8102091424AD12168DAF8140081420C
:1002D00045D1E068A04205D140F20D127DA1BDA03C
:1002E000FAF794FD37B1E068F860DBF80010E160E0
:1002F000CBF80040E068A04205D140F2151275A18C
:10030000BFA0FAF783FD4CB3DFF820830027C8F8BD
:1003100000702989A8F80810C8F80450F168C8F8D6
:100320001010F761777037813078000703D5687B4C
:1003300040F001006873606F002878D0204601F01B
:10034000BFFD0D3005D0606F002870D07089002887
:100350006DD0608D00286BD0CEE17EE003E02746B3
:10036000E468002C81D1B24840F21F1B5746046854
:1003700026E0207D0A2804D05A4656A1ADA0FAF7FF
:1003800045FD207A30B1796891F83010491CC9B226
:10039000884214D1F068218B028891420FD1E18A02
:1003A000408881420BD160683969884207D1206852
:1003B0007969884203D1204603F044F94DE0E468AE
:1003C000002CD6D1DFF89CB20021B246DBF8000049
:1003D000F3680246D7F804E07C6917E0067A3EB17C
:1003E0009EF830C00CF1010C0CF0FF0C66450BD1EF
:1003F000B0F816C05E88B44506D10668A64208D09B
:1004000000B10EB9804689460146C0680028E5D192
:1004100000E018B95FEA080049460AD021B1C36874
:10042000CB60C260CBF8000000F0ACFA15E01EE033
:1004300019E054469889F9F7F3FC40070DD4E168B8
:1004400001980A8849888DE8070061896069039BE3
:1004500042187868A16902F0DBFA04B02846BDE8CA
:10046000F05FFCF799BE204602F000FB44E1204615
:10047000346201F0E1FA0D3011D070783546000792
:100480000ED5D4F88C201AB16FF00D012069904779
:100490002146304801F0FAF92046FFF771FD2BE1C3
:1004A0002A893AB1E36F23B12146206998470D307C
:1004B0000CD02F81204600F039F938B9E86930B105
:1004C000606F28B14FF4F37202A1CDE014E1EFE0C8
:1004D000CDE000002E2E5C447269766572735C4C30
:1004E0007749505C7372635C636F72655C746370B0
:1004F0005F696E2E630000007463705F696E7075D3
:10050000743A20696E76616C696420706275660069
:1005100064010020E0620020702D3E6E657874203A
:10052000213D204E554C4C00702D3E6C656E203D9B
:100530003D203000702D3E746F745F6C656E203D01
:100540003D20702D3E6E6578742D3E746F745F6C27
:10055000656E00005C0100207463705F696E7075E9
:10056000743A20616374697665207063622D3E730E
:100570007461746520213D20434C4F534544000075
:100580007463705F696E7075743A20616374697624
:1005900065207063622D3E737461746520213D2077
:1005A00054494D452D574149540000007463705F14
:1005B000696E7075743A2061637469766520706342
:1005C000622D3E737461746520213D204C49535463
:1005D000454E00007463705F696E7075743A2070E8
:1005E00063622D3E6E65787420213D207063622029
:1005F000286265666F726520636163686529000023
:100600007463705F696E7075743A207063622D3E1A
:100610006E65787420213D207063622028616674C5
:10062000657220636163686529000000849A002078
:10063000600100207463705F696E7075743A2054B5
:10064000494D452D57414954207063622D3E7374C6
:10065000617465203D3D2054494D452D5741495415
:10066000000000005801002029A0FAF7CFFBA07E6F
:10067000C00606D5E869FCF78FFD2046FEF72EFC84
:100680003AE0D4F880C0BCF1000F05D00023206907
:100690002146EA69E04705E0002321461846EA6959
:1006A00001F028FF10F10D0F26D008B1E86960674E
:1006B0006878800618D5606F20B1417B41F0200139
:1006C000417311E0208DB0F5866F01D0401C20856C
:1006D000D4F880C0BCF1000F06D000231A46214692
:1006E0002069E0470D3007D020462F6200F01EF849
:1006F00010B9204600F0A8FB3762F761D8F8040073
:100700004446002802D0FCF747FD6760BDE8FF9F24
:100710007063622D3E726566757365645F646174B3
:1007200061203D3D204E554C4C00000010B50400AA
:1007300005D140F25A220EA116A0FAF767FB1F4816
:100740004078C00612D5A07EC00606D4D4F88C200E
:100750001AB16FF00E01206990472146184801F048
:1007600095F82046FFF70CFC012010BD002010BDBD
:100770002E2E5C447269766572735C4C7749505CCE
:100780007372635C636F72655C7463705F696E2E15
:10079000630000007463705F696E7075745F6465F8
:1007A0006C617965645F636C6F73653A20696E761E
:1007B000616C6964207063620000000064010020C5
:1007C0005C01002070B504004FF0000505D140F633
:1007D000670210A118A0FAF719FB206D401EF9F767
:1007E0001DFB034600222946204600F081FC05003F
:1007F0000DD0002301461A46204600F0CDFD2246CA
:10080000231D2946BDE87040104600F023BD4FF07F
:10081000FF3070BD2E2E5C447269766572735C4C3D
:100820007749505C7372635C636F72655C7463706C
:100830005F6F75742E6300007463705F6B65657025
:10084000616C6976653A20696E76616C69642070C6
:100850006362000070B50446082807D0092C05D053
:1008600040F2E1620EA116A0FAF7D0FA184B00216F
:1008700008469A69DB6809E0157DA54205D1156A2D
:100880005D1B8D4201D329461046D268002AF3D160
:10089000002804D0BDE870400021FEF76BBA70BD9F
:1008A0002E2E5C447269766572735C4C7749505C9D
:1008B0007372635C636F72655C7463702E630000B7
:1008C000696E76616C696420737461746500000000
:1008D000440100202DE9F041050005D140F211123C
:1008E000134914A0FAF792FA287D012805D04FF495
:1008F00089720F4912A0FAF789FA0126DFF85880A9
:100900005FF0000758F82600046855B9FF2208492F
:1009100012A0FAF77BFA04E0A16FA94200D1A76701
:10092000E468002CF8D1761C042EEBD3BDE8F081EE
:10093000A0FF000870636220213D204E554C4C0002
:100940007063622D3E7374617465203D3D204C4997
:100950005354454E00000000707001087463705FCE
:1009600072656D6F76655F6C697374656E65723AFA
:1009700020696E76616C6964206C697374656E655C
:1009800072000000FEB5464E0546307840071BD485
:100990002DB940F2812243A14BA0FAF737FA307803
:1009A000514FC10611D5F06807F1100207F1140389
:1009B000018840880092CDE901017189706942186F
:1009C0007868B16902F024F8FEBD8007FCD5687F25
:1009D000297F8842F8D2687DFEF7BAFA04004FD02A
:1009E000687F401C6877608B40F400706083786992
:1009F000206038696060E88AE082F06800882083BF
:100A0000032020757069401C6062E062204600F09F
:100A1000EDF9A06520656064E0657069401E606561
:100A20002869A5672061687A00F00C006072287A56
:100A300020722E480168E160046002F0E9FD2C4953
:100A400001200870204600F003FEF068C089A4F879
:100A50006000A4F86200201DF8F7F6FF0146608EE2
:100A6000221DFFF7EFF8608612212046FFF728F9D4
:100A700088B103B02046BDE8F0400021FEF77AB906
:100A8000AB69002BA0D0286903B04FF0FF32BDE85E
:100A9000F040002118472046BDE8FE4000F0D4B9E0
:100AA000640100202E2E5C447269766572735C4C82
:100AB0007749505C7372635C636F72655C746370DA
:100AC0005F696E2E630000007463705F6C697374FD
:100AD000656E5F696E7075743A20696E76616C69D7
:100AE0006420706362000000E06200205C0100206E
:100AF000440100202DE9F04716460F4605004FF04F
:100B0000000407D0287D58B139A0EFF79DFC6FF0A5
:100B10000E0068E044A0EFF797FC6FF00F0062E072
:100B2000687ADFF83491400711D5D9F800000CE05D
:100B3000C18AEA8A914207D101682A68914203D1A9
:100B400000246FF007004EE0C0680028F0D10220BA
:100B5000FAF76EFD04001DD028692061E88AE08262
:100B600001202075687D6075687A6072287A20722D
:100B7000E87AE072A87AA07228682060E88A4FF0CC
:100B80000008A8B1344914390869A8420CD1C068DA
:100B900008610BE04FF0FF3025E0C168A94202D1A7
:100BA000E968C16002E008460028F6D1C5F80C806B
:100BB0002846FFF7E5F92948A06184F81D80207DCB
:100BC000012805D04FF4657225A12DA0FAF71EF972
:100BD00007B901272777D9F80010E160C9F800406C
:100BE00002F016FD002006B130702046BDE8F08707
:100BF0007463705F6C697374656E5F776974685F46
:100C00006261636B6C6F675F616E645F6572723A9D
:100C10002070636220616C726561647920636F6E1D
:100C20006E656374656400007463705F6C697374EF
:100C3000656E5F776974685F6261636B6C6F675F35
:100C4000616E645F6572723A20696E76616C696488
:100C5000207063620000000058010020F1EE0008DF
:100C60002E2E5C447269766572735C4C7749505CD9
:100C70007372635C636F72655C7463702E630000F3
:100C80007063622D3E7374617465203D3D204C4954
:100C90005354454E202863616C6C656420666F7206
:100CA0002077726F6E67207063623F29000000003A
:100CB00070B50D4604001DD0206800281AD00E4ED5
:100CC0002046B16900F01AF82046316900F016F8A4
:100CD000002D0FD0286800280CD006F114000268FF
:100CE00006E010682168884201D128681060D26847
:100CF000002AF6D170BD00004401002070B5050047
:100D00000C4611D140F60A1209A111A0FAF77EF89B
:100D10000AE020682968884205D12046E668FEF787
:100D2000DDF8344600E0E468002CF2D170BD00002C
:100D30002E2E5C447269766572735C4C7749505C08
:100D40007372635C636F72655C7463702E63000022
:100D50007463705F6E657469665F69705F61646417
:100D6000725F6368616E6765645F7063626C69730C
:100D7000743A20696E76616C6964206F6C645F619F
:100D8000646472004020FEF7E3B80000F0B5154D32
:100D9000154A00234FF6FF764FF440474FF4804E3C
:100DA0009088401C80B29080B04200D19780B2F809
:100DB0000440002055F8201009680AE0B1F816C078
:100DC000A44505D15B1C9BB27345E9D30020F0BD5F
:100DD000C9680029F2D1401CC0B20428EAD3A0B2ED
:100DE000F0BD0000707001084401002010B528B962
:100DF00040F6B90204A10CA0FAF708F81149D1E9AC
:100E000002021044886010BD2E2E5C447269766523
:100E100072735C4C7749505C7372635C636F72658C
:100E20005C7463702E6300007463705F6E65787429
:100E30005F6973733A20696E76616C6964207063D0
:100E400062000000440100202DE9F05F040005D19C
:100E500040F2E54286A18FA0F9F7D8FF207D012856
:100E600005D140F2E74282A190A0F9F7CFFF99485F
:100E70000068A04202D10020BDE8F09FB4F86010E5
:100E8000B4F84800814200D20846E56E81466DB153
:100E90002146221D084601F037FD5FEA000A6FF087
:100EA00003012ED054B1206840B10CE0A07E800731
:100EB0007ED52046BDE8F05F01F0D8BD1AF10400F0
:100EC0001FD00068206028694068F8F7A7FF616CB0
:100ED000401A2989421800204A4514D9B4F86020E4
:100EE0004A45E3D1216F0029E0D194F89D100029F3
:100EF000DCD184F89C00012184F89D1084F89E00C8
:100F0000D4E70846B8E784F89D00266F83460EB9FB
:100F10009AE0064630680028FBD194E02869808971
:100F2000F8F77EFF400705D540F23A5250A16AA07B
:100F3000F9F76CFF206FA8B1618B11F0440F11D14C
:100F4000E06E28B102686AB90089628E904209D2C7
:100F5000B4F8640030B1B4F86600082802D211F089
:100F6000A00F7CD0207D022807D01020F8F758FF72
:100F700001462869828911438181524621462846CB
:100F800000F058FA20B1618B41F08001618373E772
:100F9000A5F80AB02868E066207D022803D0608B9F
:100FA00020F00300608328694068F8F737FF00E00D
:100FB00059E0074628698089F8F732FF800700D09A
:100FC0000120298938440844216D091A00D520657B
:100FD00028698089F8F724FF800700D0012029893B
:100FE000C8422CD0C5F800B0206F68B128694068AD
:100FF000F8F714FF074630694068F8F70FFF381A12
:101000001AD504F1700003E0256716E0D8F8000057
:101010008046006850B100694068F8F7FFFE074657
:1010200028694068F8F7FAFE381AEFD4D8F80000BB
:101030002860C8F8005005E035602E4602E02846DA
:1010400001F0FDFCE56E55B128694068F8F7E6FE51
:10105000616C401A2989014449457FF65FAFE06E13
:1010600008B9A4F868B0608B20F08000608302E7C4
:101070002E2E5C447269766572735C4C7749505CC5
:101080007372635C636F72655C7463705F6F7574B9
:101090002E6300007463705F6F75747075743A200E
:1010A000696E76616C69642070636200646F6E279C
:1010B000742063616C6C207463705F6F75747075FD
:1010C0007420666F72206C697374656E2D70636234
:1010D0007300000084010020525354206E6F74206E
:1010E00065787065637465642068657265210000C9
:1010F0002DE9FF411D4616460F46040005D140F27A
:1011000046720CA114A0F9F781FEE08A638D1022CB
:10111000218B8DE80F002B4632463946606A00F07D
:101120002FF8002803D0628D616A1144E16204B097
:10113000BDE8F0812E2E5C447269766572735C4C5A
:101140007749505C7372635C636F72655C74637043
:101150005F6F75742E6300007463705F6F757470D9
:1011600075745F616C6C6F635F6865616465723A2A
:1011700020696E76616C6964207063620000000013
:101180002DE9F05F834688180E46DDE90B98143090
:1011900081B21F464FF420722220DDF828A0FBF711
:1011A0009DFC050029D0698906F11400814205D211
:1011B00040F2277212A11BA0F9F728FE50466C6876
:1011C000F8F72EFE20804846F8F72AFE6080676018
:1011D0005846F8F723FEA060B008000300F5A040D1
:1011E00080B240EA0800F8F71BFEA0810D98F8F7DE
:1011F00017FEE0810020208260822846BDE8F09F33
:101200002E2E5C447269766572735C4C7749505C33
:101210007372635C636F72655C7463705F6F757427
:101220002E630000636865636B20746861742066D8
:101230006972737420706275662063616E20686FD6
:101240006C6420737472756374207463705F686477
:1012500072000000F8B51D4616460C00074605D181
:1012600040F28A720BA114A0F9F7D0FD2A4631464C
:10127000384601F049FB38B100902B4632462146F2
:10128000384600F02FF8F8BD2046FBF785FF6FF0D9
:101290000300F8BD2E2E5C447269766572735C4C57
:1012A0007749505C7372635C636F72655C746370E2
:1012B0005F6F75742E6300007463705F6F75747078
:1012C00075745F636F6E74726F6C5F7365676D6565
:1012D0006E743A20696E76616C696420706275661E
:1012E000000000002DE9FE4398460A9E91460D46F7
:1012F00004462EB940F2A17211A11AA0F9F786FD99
:101300006F68CDF800802A894B4606212846F8F7F9
:10131000CBFB388214B1E37AA07A01E0FF230020EE
:1013200006218DE84300424649462846F8F7D0FAA0
:1013300004462846FBF730FF2046BDE8FE83000048
:101340002E2E5C447269766572735C4C7749505CF2
:101350007372635C636F72655C7463705F6F7574E6
:101360002E6300007463705F6F75747075745F63D3
:101370006F6E74726F6C5F7365676D656E745F6EB0
:10138000657469663A206E6F206E657469662067C1
:101390006976656E0000000070B515460C0005D139
:1013A00040F25A720BA114A0F9F730FD6068EA0709
:1013B00000F1140100D0042210441430884207D0F8
:1013C000BDE8704040F2797202A115A0F9F71EBD88
:1013D00070BD00002E2E5C447269766572735C4CA1
:1013E0007749505C7372635C636F72655C746370A1
:1013F0005F6F75742E6300007463705F6F75747037
:1014000075745F66696C6C5F6F7074696F6E733A48
:1014100020696E76616C69642070627566000000F8
:101420006F7074696F6E73206E6F742066696C6C78
:10143000656400002DE9FE4317460C46050005D102
:1014400040F2BC523EA147A0F9F7E0FC2CB940F2B3
:10145000BD523BA14BA0F9F7D9FC2FB940F2BE52C7
:1014600037A150A0F9F7D2FC284600F0B9F810B126
:101470000020BDE8FE83606AF8F7D0FC2969886027
:10148000608DF8F7CDFC2969C881618D606A0844D8
:10149000E0622E69287B1436C0070AD0221D394627
:1014A0004FF40670FEF7CEFB40F00170F8F7B6FC83
:1014B00001C6B4F930004FF00008002801DAA4F8A2
:1014C0003080606B38B940480068606328694068C4
:1014D000F8F7A4FCA0636968288A8A88801A4A8978
:1014E000121A4A8169680A89101A0881696828698C
:1014F00048602969A1F81080287B2969C00700D0BD
:10150000042014300844B04205D04FF4C4620CA14A
:101510002EA0F9F77BFC201D009068682346062169
:101520000289F8F7C1FA2969221D0882A07A0621EA
:101530008DE88300E37A21466868F8F7C9F998E7EF
:101540002E2E5C447269766572735C4C7749505CF0
:101550007372635C636F72655C7463705F6F7574E4
:101560002E6300007463705F6F75747075745F73C1
:1015700065676D656E743A20696E76616C6964208A
:10158000736567007463705F6F75747075745F73F3
:1015900065676D656E743A20696E76616C6964206A
:1015A000706362007463705F6F75747075745F73DD
:1015B00065676D656E743A20696E76616C6964204A
:1015C0006E65746966000000500100206F707469D8
:1015D0006F6E73206E6F742066696C6C65640000BA
:1015E00010B5040005D140F29E5206A10EA0F9F7F5
:1015F0000DFC6068807B012801D0012010BD002017
:1016000010BD00002E2E5C447269766572735C4CCE
:101610007749505C7372635C636F72655C7463706E
:101620005F6F75742E6300007463705F6F75747004
:1016300075745F7365676D656E745F627573793A13
:1016400020696E76616C6964207365670000000034
:101650002DE9F041060005D140F283721CA125A0BE
:10166000F9F7D4FB2A4C6088002819D00020E080CC
:101670004FF4067510E000BFFEF72AFD00280FD0DA
:10168000012809D002280DD0FEF722FD022807D339
:10169000E1880844801EE080E08861888842EBD3BE
:1016A000BDE8F081FEF714FD0428F9D1E0886188D7
:1016B000801C8842F4D8FEF70BFD0702FEF708FDF8
:1016C0003843A84200D800B928467086E4E70000F5
:1016D0002E2E5C447269766572735C4C7749505C5F
:1016E0007372635C636F72655C7463705F696E2EA6
:1016F000630000007463705F70617273656F707473
:101700003A20696E76616C69642070636200000043
:10171000640100202DE9F05F83460AA85FEA030810
:1017200090E8400615460C460F4604D1EB221EA158
:1017300026A0F9F76BFB26B9EC221BA12CA0F9F728
:1017400065FBAC4214D25FEA897009D4B07E4006D2
:101750000ED4BAF1000F03D0F06E08B9306F38B173
:1017600004F21B2020F00300A84200D80546AFB2C7
:101770004FF4207239465846FBF7B0F9050010D0F7
:10178000286828B14FF4877207A121A0F9F73EFB22
:101790006889001BA8F800002C816C812846BDE8F0
:1017A000F09F0020FBE700002E2E5C4472697665F6
:1017B00072735C4C7749505C7372635C636F7265E3
:1017C0005C7463705F6F75742E6300007463705F88
:1017D000706275665F707265616C6C6F633A2069E8
:1017E0006E76616C6964206F76657273697A6500E4
:1017F0007463705F706275665F707265616C6C6F48
:10180000633A20696E76616C6964207063620000DF
:101810006E65656420756E636861696E65642070CD
:101820006275660070B504001DD0207D002819D0B7
:101830000A2817D0012815D02046FDF727FC606F35
:10184000002510B1FBF7A8FC65674FF0FF3020863C
:10185000E06E01F002F9206F01F0FFF8E566256700
:10186000A4F8685070BDBDE8704001A0EEF7ECBD73
:101870007463705F7063625F70757267653A206948
:101880006E76616C696420706362000070B50C0054
:10189000054605D140F68D0221A129A0F9F7B6FA37
:1018A0002DB940F68E021EA12CA0F9F7AFFA2868D8
:1018B000A04209D1C068286008E0C168A14202D1F5
:1018C000E168C16002E008460028F6D10025204604
:1018D000E560FFF7A7FF207D0A280DD001281BD067
:1018E000608BC10708D040F0020060832046FFF7FC
:1018F000ABFA207D01280FD0E06E28B140F69D02A2
:1019000007A11EA0F9F782FA206F28B140F69E02C7
:1019100003A120A0F9F77AFA2575E58270BD0000D1
:101920002E2E5C447269766572735C4C7749505C0C
:101930007372635C636F72655C7463702E63000026
:101940007463705F7063625F72656D6F76653A2075
:10195000696E76616C696420706362007463705FA5
:101960007063625F72656D6F76653A20696E76614D
:101970006C6964207063626C69737400756E736562
:101980006E74207365676D656E7473206C65616B32
:10199000696E6700756E61636B6564207365676D62
:1019A000656E7473206C65616B696E670000000082
:1019B00070B515460E46040003D0207D012805D0E1
:1019C0000AE0BDE8704006A0EEF73EBD40F64802D2
:1019D00009A111A0F9F71AFAC4F88860657770BDFB
:1019E0007463705F706F6C6C3A20696E76616C69BD
:1019F00064207063620000002E2E5C44726976657C
:101A000072735C4C7749505C7372635C636F726590
:101A10005C7463702E630000696E76616C6964208B
:101A2000736F636B657420737461746520666F7285
:101A300020706F6C6C0000002DE9FE4F040005D192
:101A400040F21F32EDA1F6A0F9F7E0F9FB4D28783E
:101A500041072AD5227D022A05D0616A6869814240
:101A600006D182B115E0206DA969884211D0C2E18A
:101A7000421AFCD4228D1144081AF8D4608B40F02D
:101A800002006083B7E140F23B32DCA1ECA0F9F741
:101A9000BDF9687840F008006870608B20F00100A4
:101AA00060836FF00D00BDE8FE8F800704D5207DB8
:101AB000022801D00328E1D1A07EC00602D4E84864
:101AC000006820624FF0000984F89F9084F89E908F
:101AD0002046FFF7BDFD2A78900704D5207D022817
:101AE00001D00328C3D1DF4B94F814C003F11000D8
:101AF0000421DFF874B3DD4FDD4E1433ACF1020C7A
:101B00004FF0010ABCF1080FB1D2DFE80CF00484F9
:101B1000E8F0EEE8EDECD606A9D5920765D5626C43
:101B2000AE69521CB24260D168690246401C6062D4
:101B30006664E062E868521EC089A4F86000A4F8F8
:101B4000620062652175201DF7F77EFF0146608EF9
:101B5000221DFEF777F841F21C116086B1EB400FB1
:101B600001D2420000E00A46B2EB800F01D98100A9
:101B700003E0B1EB400F00D24100A4F84810B4F8E4
:101B8000660028B940F277329CA1BAA0F9F73EF975
:101B9000B4F86600401EA4F86600256FB5B1286849
:101BA0002067284600F04BFF206FD0B1A4F830909A
:101BB00084F84290D4F88430002B3FF45FAF0022C9
:101BC0002146206998470D3055D057E7E56E2DB96D
:101BD00040F27F3289A1ADA0F9F718F92868E066D4
:101BE000DFE74FF0FF302086E4E7E9680A8849889C
:101BF0008DE807006989686942182046A96900F0E4
